:020000040800F2
:10000000F04D03206D4C00083F0300084103000839
:1000100045030008490300084D03000800000000E4
:10002000000000000000000000000000890200083D
:100030005103000800000000DD0200086D4B0008BD
:10004000874C0008874C0008874C0008874C000844
:10005000874C0008874C0008874C0008874C000834
:10006000874C0008874C0008874C0008874C000824
:10007000874C0008874C0008874C0008874C000814
:10008000874C0008874C0008874C0008874C000804
:10009000874C0008874C0008874C0008874C0008F4
:1000A000874C0008212C0008874C0008874C00086A
:1000B000874C0008874C0008ADC40108874C000835
:1000C000874C0008874C0008874C0008874C0008C4
:1000D000874C000899300008874C0008874C0008BE
:1000E000874C0008874C0008874C0008874C0008A4
:1000F000874C0008874C0008874C0008874C000894
:10010000874C0008874C0008874C0008874C000883
:10011000874C0008874C0008874C0008874C000873
:10012000874C0008874C0008874C0008874C000863
:10013000874C0008874C0008874C0008874C000853
:10014000874C0008874C0008874C0008874C000843
:10015000874C0008874C0008874C0008874C000833
:10016000874C0008874C0008874C0008874C000823
:10017000874C0008874C0008874C0008874C000813
:10018000874C0008874C000800F002F800F06CF87B
:100190000AA090E8000C82448344AAF10107DA45E2
:1001A00001D100F061F8AFF2090EBAE80F0013F0C8
:1001B000010F18BFFB1A43F001031847ACAD07004D
:1001C000CCAD07000A444FF0000C10F8013B13F0CF
:1001D000070408BF10F8014B1D1108BF10F8015BA0
:1001E000641E05D010F8016B641E01F8016BF9D193
:1001F00013F0080F1EBF10F8014BAD1C0C1B09D1EA
:100200006D1E58BF01F801CBFAD505E014F8016B5B
:1002100001F8016B6D1EF9D59142D6D370470000ED
:100220000023002400250026103A28BF78C1FBD8FF
:10023000520728BF30C148BF0B60704764291DF0CA
:100240009F8275291DF09C8263291DF07285732998
:100250001DF07785002070471FB51EF09AFE1DF037
:10026000CBFC1FBD10B510BD1DF08EFD1146FFF774
:10027000F3FF00F0D6FB1DF0ACFD03B4FFF7F2FF77
:1002800003BC04F0E9FC00002A4B19680868B0E8D8
:10029000F04F80F30988BFF36F8F4FF0000080F3B9
:1002A000118870470000000006480068006880F36D
:1002B000088862B661B6BFF34F8FBFF36F8F00DF60
:1002C00000BF00BF08ED00E0DFF80C00016841F45A
:1002D00070010160704700BF88ED00E0EFF3098016
:1002E000BFF36F8F134B1A681EF0100F08BF20ED7D
:1002F000108A20E9F04F106008B44FF0500080F3EE
:100300001188BFF34F8FBFF36F8F19F036FF4FF097
:10031000000080F3118808BC19680868B0E8F04F45
:100320001EF0100F08BFB0EC108A80F30988BFF3ED
:100330006F8F704768020020EFF3058070477047A9
:1003400000BFFEE700BFFEE700BFFEE700BFFEE71D
:10035000704700005F48006840F080505D490860C9
:100360005D48006840F440405B49086059483838AF
:10037000006858493839086008460068086008462F
:10038000006840F4805008605448091F0860081F46
:10039000006840F08070091F086000BF4D48403879
:1003A000006800F000700028F8D040F202704C495C
:1003B000086048483838006820F00300454938395B
:1003C00008600846006840F00200086000BF41482D
:1003D0003838006800F00C000828F8D1704710B5D4
:1003E00000BF00BF00BF00BF3E48006840F470007F
:1003F0003C49086037484038006840F00100354902
:1004000040390860002033493839086031484038A5
:100410000068354908402F49403908603348091DB4
:100420000860081F006820F48020091F0860002071
:10043000284934390860FFF78DFF10BD70B50020E2
:100440000021022200230224224D383D2D6805F0B0
:100450000C0020B1042806D0082829D107E0244D3B
:10046000244E356028E0244D224E356024E0194D9D
:100470003C3D2D68C5F38053164D3C3D2D6805F07D
:100480003F044BB91A4DB5FBF4F5124E3C3E3668AD
:10049000C6F3881605FB06F10E4D3C3D2D68C5F3ED
:1004A00001456D1C6A00B1FBF2F5124E356003E0A8
:1004B0000F4D104E356000BF00BF064D383D2D6812
:1004C000C5F303150D4E705D0A4D2D68C540094EEC
:1004D000356070BD40380240007000401064010774
:1004E000003C024088ED00E0FFFFF6FE10300024E3
:1004F0000024F4000000002000127A000400002014
:100500001CB50121084604F067FF4FF4807000908D
:1005100000208DF8040003208DF8050001208DF8DF
:1005200007006946FE4804F0B7FCFE4801F08DF86C
:10053000FD481BF0D5FF1CBD00B589B00020FB496C
:100540000870FB490870FB490870FB490870FB49BB
:1005500008600021FA4A11605160FA490860F148C8
:1005600001F073F8642017F0EAFFF74802F05AFF31
:100570000A2017F0E4FF01A9F44803F094F9EA48CF
:100580001BF0A6FFE74800F089FEF148007830B97B
:100590000120F04908700020EF49087012E0EC4893
:1005A00000785A280ED10420EA490870EB480078F8
:1005B000012807DBE9480078112803DCE7480078C8
:1005C000E5490870E5480078112802DD1120E2496C
:1005D000087009B000BD0BE0642019F0A5FCD248FA
:1005E0001BF0EEFFD0481CF062F80020DC494861A7
:1005F000F2E708B519F08DFF00901EE0D9480068B9
:10060000401CD84908600A21684619F032FCD648D7
:1006100001F021FBD44802F0D6FDD24800680A213F
:10062000B0FBF1F201FB120020B9D04802F09AFEB3
:1006300005F08BFC0020CA490861DFE79DE000203F
:10064000C749C860BB480078002872D002F099FC06
:10065000C82019F069FC02F0B3FCC82019F064FC52
:1006600002F08FFCC82019F05FFC02F0A9FCC82042
:1006700019F05AFC02F085FCC82019F055FC02F074
:100680009FFC4FF4FA7019F04FFC0020B449C86089
:1006900002F077FC4FF4C87019F046FC02F090FCB1
:1006A000C82019F041FC02F06CFC4FF4C87019F03E
:1006B0003BFC02F085FCC82019F036FC02F061FC1E
:1006C0004FF4C87019F030FC02F07AFC4FF4FA7065
:1006D00019F02AFC0020A249C86002F052FCC82090
:1006E00019F022FC02F06CFCC82019F01DFC02F08D
:1006F00048FCC82019F018FC02F062FCC82019F070
:1007000013FC00209649C86002F03BFCC82019F099
:100710000BFC02F055FC002407E000209049C86063
:100720004FF4C87019F000FC641C052C25D2F4E7C6
:10073000FFE781480078012806D102F022FC4FF43F
:10074000FA7019F0F1FB18E07948007801280CD113
:1007500002F017FC4FF4FA7019F0E6FB02F030FCDF
:100760004FF4FA7019F0E0FB07E002F029FC642076
:1007700019F0DAFB7E4803F013FD60E708B519F0C5
:10078000C8FE009019E0002075498860674800782D
:1007900003280EDA0A21684619F06BFB75481BF036
:1007A00048FD6C480078012807D15E4800F04DFFF5
:1007B00003E04FF47A7019F0B7FBE4E711E0002092
:1007C0006749486059480078032806DA142019F070
:1007D000ABFB694816F0A3FB03E04FF47A7019F005
:1007E000A3FBECE708B519F094FE009011E000209F
:1007F0005B4908604D480078032806DA0121684605
:1008000019F037FB11F08BFE03E04FF47A7019F00A
:100810008BFBECE71CB504460121080304F0DCFD6A
:100820001BF03BF817F042FF54490860544804217C
:1008300000230A02CDE9001052A1AFF2570019F0CF
:10084000F5F85448052100234FF48062CDE90010EB
:1008500051A1AFF2970019F0E9F8534802210023A3
:10086000CA01CDE9001051A1AFF2EF0019F0DEF896
:100870005248032100238022CDE9001050A1AFF29D
:10088000432019F0D3F85148062100234FF4807219
:10089000CDE900104EA1AFF2A52019F0C7F84F48DE
:1008A000072100234FF48072CDE900104CA1AFF274
:1008B000D92019F0BBF81BF013F81A4800F0F4FA2D
:1008C000642019F031FB174800F088FC1CF0BBF9DC
:1008D000642019F029FB1CF044FA44A1224802F0DC
:1008E00064FC322019F020FB0E4800F083FA32201D
:1008F00019F01AFB45F2555005F01EFB032005F0D8
:100900001EFB40F6FF7005F01DFB002005F014FBF8
:1009100005F020FB00203F4908603F4800687DE06B
:1009200000000240AC0000206E430320C400002001
:100930003100002032000020300000202C00002078
:100940001800002028000020EF1800200E1A0020B8
:1009500053000020330000205100002050000020F0
:1009600008030020A800002066040020CA00002020
:10097000142B00205C430320FC0100203C000020DD
:10098000980000206C6974746C655F76676C5F74A6
:1009900061736B009C000020646973706C61795F07
:1009A0007461736B00000000900000204B65796259
:1009B0006F6172645F7461736B00000094000020CB
:1009C0006C6564305F7461736B000000A0000020F0
:1009D000556172745F7461736B000000A4000020A5
:1009E00052463433335F7461736B00005379732064
:1009F0007374617274696E672C63726561746520CB
:100A000036207461736B73202E2E2E2E2E2E0D0A1F
:100A100000000000B48240428C00002019F054F81D
:100A20001CBD1CB500BF00BF00BF00BF2A481BF0A3
:100A300034F900240BE04FF48061284804F08EFA6A
:100A400018B9274800F0E2FD00E003E0641C2548E7
:100A50008442F0D300BF224800F0F7FD4FF0006061
:100A60002149086007230222C821102002F0C1F9A1
:100A7000642004F083F84FF4407004F017F94FF449
:100A8000E1311A4802F02CFBFFF73AFDFFF754FD65
:100A90001CF067F901F0C9FD0F481BF0FEF814487F
:100AA00003F023FB4FF4FA61124802F04DFC08F00A
:100AB000E1FA15F0CCFE05F08CFA0F480121002375
:100AC0000A02CDE900100DA1AFF2B72018F0AEFF79
:100AD00019F0D5FC00201CBD5C430320000402403B
:100AE000AC000020A086010008ED00E066040020B4
:100AF000142B0020CA0000208C0000207374617247
:100B0000745F7461736B000070477047012080F35D
:100B1000108800BF7047002080F3108800BF704726
:100B200010B5034600200FE0002207E000BF00BF21
:100B300000BF00BF00BF00BF541CA2B241F2A864B6
:100B4000A242F3DB441CE0B28842EDDB10BD7FB56E
:100B5000064600BF00BF0020FA490860FA48006856
:100B6000401CF9490860084600680A2802D2F74884
:100B70001BF04CFCF6480068401CF549086008462C
:100B80004068401C486008468068401C88600846F1
:100B9000C068401CC86008464069401C486108465F
:100BA0000069401C0861EB48007800B17FBD00255A
:100BB0000020E9498860E6480068052800D9312509
:100BC000E3484068052800D93225E14880680528B7
:100BD00000D93325DE48C068052800D93425DC4813
:100BE0004069052800D93525D9480069052800D96C
:100BF000362525B1D9480078401CD8490870D74817
:100C00000078012801D1D6490870D4480078052819
:100C10002DDDD448D0F8AC00401CD249C1F8AC005E
:100C2000D14968461CF026FE8DF80750002409E0E3
:100C30001DF80400CD49888032213046FFF770FF4F
:100C4000601CC4B20A2CF3DBFFF760FF00BFBFF3E8
:100C50004F8FC748006800F4E060C6490843001D94
:100C6000C3490860BFF34F8F00BF00BFFEE700BF5E
:100C70009CE710B5C048FFF76AFF10BD704770478A
:100C800070B5A0B006460D46012D27D10022802167
:100C9000684617F0E3F800240CE04FF6FF7000EA16
:100CA00044116B462022B54802F037FD0A2019F0A6
:100CB0003BF9641C202CF0D3B14968461CF0DAFDE6
:100CC0006B4610220021AD4802F027FD0A2019F0E2
:100CD0002BF9ACA1B24802F068FA03E0B1A1B04828
:100CE00002F063FAAE4802F06EFA012019F01CF926
:100CF000012D11D100209849087048707820488053
:100D00004FF4615088804FF41670C8800B4608225B
:100D100076219A4802F001FD20B070BD70B590B008
:100D2000064600BF00BF0020A5490860864908604C
:100D300008AB10220021914802F0AFFC6B46102254
:100D400011468E4802F0A9FC0A2019F0EDF80025A2
:100D500000240FE008A8005D8949095D884205D09C
:100D60001DF804009749095D884201D1681CC5B28D
:100D7000601CC4B2102CEDDB0F2D19DA01213046B6
:100D8000FFF77EFF7E4B102200217C4802F0C5FC5D
:100D90000A2019F0C9F88B4B10221146774802F04F
:100DA000BCFC0A2019F0C0F887A17D4802F0FDF9CB
:100DB00000BF00BF00BF00BF674B082276216F480D
:100DC00002F06BFC10B070BD704710B503460020F8
:100DD0000DE0002207E000BF00BF00BF00BF00BF62
:100DE00000BF541CE2B2022AF5DB441CA0B28842C8
:100DF000EFDB10BD10B58AB0044600BF00BF00BFD6
:100E000000BF00221821774817F028F8002220217F
:100E100001A817F023F81022734972481CF0BEFD98
:100E2000002070490874487470A15D4802F0BDF953
:100E30006C495B4802F0B9F960A1594802F0B5F974
:100E40006D480168564802F0B0F96C480168544892
:100E500002F0ABF96AA1524802F0A7F969480168AB
:100E60004F4802F0A2F966A14D4802F09EF9002217
:100E7000202101A816F0F2FF04226348016809A8A6
:100E80001CF000FE01A9099817F0BEF801A944481A
:100E900002F08BF949A1424802F087F90AB010BD6F
:100EA000704700BF00BF704730B589B0054600BF2E
:100EB00000BF5648046804F07C44A40E082C30D0CF
:100EC00006DC062C3AD2DFE804F0E51015212627CF
:100ED000112C34D004DC092C24D0102C2ED1CDE0E0
:100EE000202C2DD0212CF9D1CFE049A101A81CF054
:100EF000C1FCD4E04CA101A81CF0BCFC1948D0F8FE
:100F0000B000401C1749C1F8B000C8E04BA101A8CF
:100F10001CF0B0FCC3E000BF4EA101A81CF0AAFC6D
:100F2000BDE000BF4FA101A81CF0A4FC0D48D0F803
:100F3000B400401C0B49C1F8B400B0E0AAE09EE048
:100F4000A2E00000200000202C0000205C430320D1
:100F500008030020C400002020030020B00000206F
:100F6000440000202C0300209CEF010800100140E9
:100F70000CED00E00000FA05AC000020F0180020A5
:100F8000BAEF0108526573746F726520466163742D
:100F90006F727920446565706C790D0A000000005D
:100FA00066040020526573746F7265204661637435
:100FB0006F727920536C696768746C790D0A000050
:100FC00024000020A8EF010873797374656D206612
:100FD000697273742072756E20666C61670D0A0009
:100FE00000000000F0020020A0200008446576699F
:100FF00063652049443A000080000020740000200E
:1010000020000000780000207000002074380240AA
:101010000D0A52657365742050696E2052657365C0
:10102000740D0A00000000000D0A506F77657220F1
:101030004F6E2052657365740D0A00000D0A506FE3
:101040007765724F6E20526573657450696E0D0A34
:10105000000000000D0A536F6674205265736574BA
:101060000D0A00000D0A49205761746368646F67B8
:101070002052657365740D0A0000000000BFF3A1E3
:1010800001A81CF0F7FB0AE000BFF6A101A81CF0C4
:10109000F1FB04E0F9A101A81CF0ECFB00BF00BFCC
:1010A000FE48006840F08070FC49086001A9FC48D7
:1010B00002F07BF800BF00BF09B030BD704700BF31
:1010C00000BF70472DE9F04107460C46F54800780F
:1010D000002839D0F448016820461CF0CBFBF3A16E
:1010E00020461CF00AFC20461CF0E8FBC5B2611942
:1010F000EF4A1268106816F026FDECA120461CF09D
:10110000FCFB20461CF0DAFBC5B26119E94A126803
:10111000106816F018FDE5A120461CF0EEFB2046F5
:101120001CF0CCFBC5B2E4480268E4480168E4481E
:1011300003F033FC06466119304616F004FDC8A1E1
:1011400020461CF0DAFB46E0D748016820461CF038
:1011500091FBD6A120461CF0D0FB20461CF0AEFB34
:10116000C5B26119D24A1268106816F012FFCFA1F9
:1011700020461CF0C2FB20461CF0A0FBC5B2611942
:10118000CC4A1268106816F004FFC8A120461CF073
:10119000B4FBCA48016820461CF0AFFBC3A120463F
:1011A0001CF0ABFBC448016820461CF0A6FBBFA1A5
:1011B00020461CF0A2FB20461CF080FBC5B2BE48B6
:1011C0000268BE480168BE4803F0E7FB06466119A5
:1011D000304616F0B8FCBDE8F081704710B58CB011
:1011E0000446684604F027F8B6A1AD4801F0DDFFDB
:1011F000202104A81CF0ADFC04A9009816F004FFFF
:10120000AFF2482104A81CF078FBB4A1A44801F077
:10121000CCFF04A9A24801F0C8FF202104A81CF0BB
:1012200098FC04A9019816F0EFFEAFF2702104A813
:101230001CF063FBACA19A4801F0B7FF04A99848E1
:1012400001F0B3FF202104A81CF083FC04A902983C
:1012500016F0DAFEAFF29C2104A81CF04EFBA4A10C
:101260008F4801F0A2FF04A98D4801F09EFF2021C4
:1012700004A81CF06EFC04A9039816F0C5FEAFF29A
:10128000C42104A81CF039FB9BA1854801F08DFF07
:1012900004A9834801F089FF0CB010BD10B5C2B09D
:1012A00004466A464FF4FF51954802F04BFC9DF806
:1012B00000009DF80110884208D19DF80100FF2828
:1012C00004D09DF800008F49087002E008208D4985
:1012D00008709DF802009DF80310884208D19DF81F
:1012E0000200FF2804D09DF802008749087002E040
:1012F0000220854908709DF804009DF80510884279
:1013000008D19DF80500FF2804D09DF804007F490E
:10131000087002E000207D4908709DF808009DF8E3
:101320000910884208D19DF80900FF2804D09DF8D3
:1013300008007749087002E00020754908709DF8A0
:101340000C009DF80D10884208D19DF80D00FF2873
:1013500004D09DF80C006F49087002E000206D4930
:1013600008709DF810009DF81110884208D19DF872
:101370001000FF2804D09DF810006749087002E0B3
:1013800000206549087065A1454801F00EFF6B46D5
:101390004FF480720121424801F03AFEAFF2E4318D
:1013A0003F4801F002FF6A460121554802F0CAFB9E
:1013B00061A13B4801F0F9FE6B464FF480720121B8
:1013C000374801F025FEAFF20C41354801F0EDFE43
:1013D00042B010BDF0B5C3B0074600250026052277
:1013E0004FF4FF71464802F0B5FC322018F09CFD26
:1013F0000024584802782146641C01A842545548EC
:1014000002782146641C01A842543F4802782146D4
:10141000641C01A842543C4802782146641C01A87F
:1014200042543A4802782146641C01A84254374885
:1014300002782146641C01A84254344802782146AF
:10144000641C01A842543148027885E00D0A5720F7
:101450005761746368646F672052657365740D0A21
:10146000000000000D0A4C6F7720506F77657220E6
:1014700052657365740D0A00000000000D0A446F88
:101480006E2774206B6E6F7720726561736F6E20AC
:1014900052657365740D0A00000000007438024044
:1014A00066040020C4000020640000202C0000001E
:1014B000680000206C0000207800002074000020EC
:1014C000542B00200A53797374656D206672657120
:1014D00075656E63793A0D0A000000005359534355
:1014E0004C4B3A000000000048434C4B3A000000CF
:1014F00050434C4B313A000050434C4B323A0000C1
:101500000E1A00205000002052000020530000203E
:101510005400002055000020560000200A4C6F6146
:101520006420706172656D657465722054657374B2
:1015300020446174613A00000A466C61736820704F
:101540006167652031205465737420446174613A89
:1015500000000000510000202146641C01A84254F4
:101560005B4802782146641C01A84254584802781E
:101570002146641C01A84254554802782146641C47
:1015800001A84254524802782146641C01A84254E2
:10159000504802782146641C01A842544D48027804
:1015A0002146641C01A842544A4802782146641C22
:1015B00001A84254474802782046611C8CB201A918
:1015C0000A54454802782046611C8CB201A90A548D
:1015D000414802782046611C8CB201A90A543E4859
:1015E00002782046611C8CB201A90A543A4802785C
:1015F0002046611C8CB201A90A54032301AA4FF4AE
:10160000FF51364802F0F7FB43B0F0BD1CB504466D
:101610000121084603F0E0FE4FF40041304803F09A
:10162000B7FC4FF40140009000208DF80400012029
:101630008DF8060003208DF8050000208DF80700C6
:101640006946274803F028FC1CBD1CB5044601214F
:10165000084603F0C1FE0121022003F0BDFE4FF455
:101660000040009001208DF8040000208DF8060055
:1016700003208DF8050001208DF807006946184801
:1016800003F00AFC6946174803F006FC4FF480702B
:10169000009000208DF804008DF8060003208DF8DE
:1016A000050001208DF8070069460D4803F0F4FBA2
:1016B0004FF400410A4803F06DFC4FF40041094823
:1016C00003F068FC1CBD00B50748FFF7D7FA00BD62
:1016D0005400002055000020560000200E1A002063
:1016E0000000024000040240AC00002070B5054636
:1016F0000E4600BF41F26D00284490F80D0400280A
:10170000F8D1552484F07A04744000BF5520FA497A
:101710008880012018F008FC7A20F7498880012091
:1017200018F002FCF4488680012018F0FDFB002030
:10173000F1498880012018F0F7FBEF4884800120F0
:1017400018F0F2FB002041F26D012944A1F80E04CB
:1017500070BD70472DE9F84380460C460027A089EC
:10176000B0F5006F52DCE089B0F5806F4EDC02E02E
:10177000012018F0D9FBE14880780028F8D102E078
:10178000012018F0D1FBDD4800880028F8D10120A5
:10179000DA4988706689608900B1761E002510E0FC
:1017A000102000EB0523D548C01C1A1805EB860154
:1017B000D34802F0C7F9C821D14802F099FA681C51
:1017C000C5B2042DECDB4FF48060E081102221468D
:1017D000CA48C01C1CF0E2F8C8490B314FF48160C4
:1017E00016F09CFC009004226946C448C01D1CF001
:1017F000D5F84FF48260C1490880002088700846FF
:1018000001F0E1FC142018F08FFB00E001273846BE
:10181000BDE8F8832DE9F04180460D46A889B0F572
:10182000006F3CDCE889B0F5806F38DC687A3138CD
:10183000022834DAB3480078022803D0B14800788F
:1018400003282CD1687A312801D1002601E04FF419
:1018500000666C8904B1641EA400264406F00F00E3
:1018600018B93109A64802F092F8002413E04FF4A9
:10187000FA71A34802F03CFA102000EB042308F6AA
:1018800003001A1831199E4802F09DF9C8219C489E
:1018900002F02EFA641C042CE9D3002700E0012793
:1018A0003846BDE8F0812DE9F041C6B007464FF05B
:1018B0000008002600224FF4887102A816F0CEFA24
:1018C00007F60304E18901F1080007F60B0116F0A1
:1018D00025FC01906068019988427DD1207A3138D9
:1018E00005287AD2DFE800F00304348B960000BFAD
:1018F00015F062FF8348007830B9207A312803D18F
:1019000001208049087016E07E480078012806D141
:1019100002207C49087000207B4908700BE0794860
:101920000078022805D177490870002076490870B0
:1019300001E04FF00108B8F1010F08D006A9734883
:10194000FFF7C0FB4FF47A70714908602C2667E0FE
:1019500021463846FFF75EFF0546002D4CD16089D1
:10196000A18988423FD16B48D0F8A400401C694946
:10197000C1F8A4006548FFF730FC1022214602A8F8
:101980001CF00CF8022264A106A81CF009F912262A
:10199000A6F1080004A916F0C1FB0190042201A9D8
:1019A00003A81CF06FF802AB32460021384601F064
:1019B0002FFB524801F007FC0A2018F0B5FA00BFCF
:1019C000BFF34F8F5548006800F4E0605449084366
:1019D000001D5249086001E023E01EE0BFF34F8F75
:1019E00000BF00BFFEE70320464908704FF47A703D
:1019F00047490860102601E04FF0010810E0214639
:101A00003846FFF7A7FE05460DB9002601E04FF066
:101A1000010805E04FF0010802E04FF0010800BFA7
:101A200001E04FF00108B8F1010F06D102223DA1FB
:101A300006A81CF0B5F8122607E0102E05D10222E8
:101A400035A106A81CF0ACF81226AEB11022214632
:101A500002A81BF0A3FFA6F1080004A916F05EFB84
:101A60000190042201A903A81CF00CF802AB324635
:101A70000021384601F0CCFA207A31280ED12148D5
:101A8000007801280AD1384601F09DFB0A2018F0A1
:101A90004BFA4FF4E131384601F022FB46B0BDE885
:101AA000F0812DE9F043C5B0054600BF00BF00BF7F
:101AB00000BF4FF00009002740F6050010F8058030
:101AC000B8F1280F03D0B8F12A0F6ED148E000BF5B
:101AD00000BF05F6090440F60900465D532E30D1DB
:101AE000A078522822D1E288A1880DF10A030E487D
:101AF00001F0D3FDE78830E00010014066040020CB
:101B00000E1A0020C4000020B1000020AC0000200C
:101B1000C00000202C0300204F4B00000CED00E023
:101B20000000FA0545520000F0180020A078572860
:101B300013D1E288A18805F611036A4801F0EDFD92
:101B40000BE0492E05D1A078522801D1E78804E0A6
:101B500003E0452E01D04FF00109B81D87B241E0E6
:101B600005F6090440F60900465D462E32D1A078FC
:101B700052281BD1E078442808D1A1880DF10A022F
:101B8000594801F0DFFF4FF4807725E0E0785328D3
:101B900022D1554801F0B5FE8DF80A000DF10B0178
:101BA000514801F059FE052716E018E0A0785728A3
:101BB00007D1A18804F108024B4802F004F800277D
:101BC0000AE0A078452807D1A188474801F02EFFF8
:101BD000002701E04FF00109B81D87B202E04FF085
:101BE000010900BF00BFB9F1000F0AD0B8F1800FA2
:101BF00001DAFA2600E0FB2631462846FFF776FD9B
:101C000020E055208DF804007A208DF805008DF82D
:101C10000680B81FC11700EB1161090A8DF8071083
:101C2000C11700EB11610912A0EB0121C9B28DF8B7
:101C3000081000208DF8090001AB3A460021284623
:101C400001F0E6F90021284601F032FA00BF00BF9A
:101C500045B0BDE8F0832DE9F041044604F60300E9
:101C6000D0F86608401C04F60301C1F86608032892
:101C700001D0BDE8F08104F60300B0F8640800B9B3
:101C8000F7E704F603052846B0F86468002794F8DF
:101C90000308AA2808D140F60400005D752803D186
:101CA0002046FFF7FEFE15E094F80308472811D1FF
:101CB00040F60400005D49280CD140F60500005DA7
:101CC000412807D140F60600005D502802D1204689
:101CD000FFF7E9FD0021204601F0EAF900BFC8E75F
:101CE00070477047F01800200E1A00201CB5FE48FF
:101CF0000068AA2800D11CBD3C20009001208DF86E
:101D0000040000208DF8060003208DF80500012056
:101D10008DF807006946F54803F0BEF84FF480409F
:101D2000009001208DF8040000208DF806000320AB
:101D30008DF8050001208DF807006946EC4803F096
:101D4000ABF84FF4C250009001208DF80400002041
:101D50008DF8060003208DF8050001208DF807009E
:101D60006946E44803F098F80120E3490860E34934
:101D7000C1F88802E049091F0860AA20DA49086012
:101D800000BFB8E71CB5D8480068552800D11CBD75
:101D90003C20009000208DF8040003208DF8050001
:101DA00001208DF807006946D04803F075F84FF41C
:101DB0008040009000208DF8040003208DF805007D
:101DC00001208DF807006946C94803F065F84FF413
:101DD000C250009000208DF8040003208DF805000B
:101DE00001208DF807006946C24803F055F801202C
:101DF000C1490860C149C1F88802BF49091F08608C
:101E00005520B949086000BFC1E708B500909DF8AA
:101E1000001001F00101BA4A11609DF80010C1F3F1
:101E20004001B84AC2F898129DF80010C1F3800131
:101E3000B14A183211609DF80010C1F3C001B14AD7
:101E4000C2F8B0129DF80010C1F30011AE4AC2F8FA
:101E500088129DF80010C1F34011C2F88C129DF851
:101E60000010C1F38011C2F890129DF80010C9094A
:101E7000C2F8941208BD10B5002420219B4803F03D
:101E80006DF8012801D144F080041021974803F037
:101E900065F8012801D144F040040821934803F07B
:101EA0005DF8012801D144F0200404218F4803F09B
:101EB00055F8012801D144F010044FF480518D48A9
:101EC00003F04CF8012801D144F008044FF40061FC
:101ED000884803F043F8012801D144F0040440216C
:101EE000844803F03BF8012801D144F002044FF488
:101EF00080417F4803F032F8012801D144F0010409
:101F0000204610BD10B50446FFF7F0FE00207A49C8
:101F10000839086001207B49C1F894020020764905
:101F2000091F08602046FFF770FF00207349C1F8C1
:101F3000880200BF0120754908607249C1F890020B
:101F400010BD10B50446FFF7D1FE01206A490839DB
:101F500008606C49C1F8940200206749091F0860B5
:101F60002046FFF752FF00206449C1F8880200BFF5
:101F70000120664908606349C1F8900210BD10B5A0
:101F8000044600205C49091F08602012FFF73DFF4E
:101F900000205A49C1F8880200BF01205B4908604F
:101FA000E0B2FFF732FF00205449C1F8880200BFB9
:101FB0000120564908605349C1F8900210BD10B580
:101FC000FFF7E0FE01204C49083908604B49C1F891
:101FD000880200204849091F086000BF00204949C5
:101FE000C1F8940200BFFFF746FF044601204249B2
:101FF00008604449C1F89002204610BD2DE9F04127
:1020000004460D4616461F462A20FFF77BFF201286
:10201000FFF797FFE0B2FFF794FF3012FFF791FF51
:10202000F0B2FFF78EFF2B20FFF76CFF2812FFF7AF
:1020300088FFE8B2FFF785FF3812FFF782FFF8B29A
:10204000FFF77FFF2C20FFF75DFFBDE8F08170B543
:102050000646EF2340F23F1200210846FFF7CEFF6D
:10206000FFF744FE01202449083908602549C1F8DA
:10207000940200240BE0002504E03046FFF77FFFC8
:10208000681C85B2B5F5A07FF7DB601C84B2F02C2C
:10209000F1DB70BD1CB54FF42040009001208DF89D
:1020A000040000208DF8060002208DF805000120B4
:1020B0008DF8070069460E4802F0EEFE4FF480608E
:1020C000009001208DF8040000208DF80600022009
:1020D0008DF8050001208DF807006946054802F0DB
:1020E000DBFE0120064913E0B8000020000002409A
:1020F0000004024000080240940241420080414234
:10210000B882404200004142000040428882414281
:10211000091D0860FE49C1F8B4021CBD1CB50121AF
:102120000F2003F059F93C20009001208DF80400A5
:1021300000208DF8060003208DF8050001208DF8A1
:1021400007006946F34802F0A7FE4FF48040009074
:1021500001208DF8040000208DF8060003208DF882
:10216000050001208DF807006946EB4802F094FE57
:1021700041F67800009001208DF8040000208DF8D1
:10218000060003208DF8050001208DF80700694640
:10219000E24802F081FE0420009001208DF8040046
:1021A00000208DF8060003208DF8050001208DF831
:1021B00007006946DA4802F06FFE1CBD10B5FFF754
:1021C00069FF0020D74908604FF4967016F0B7F900
:1021D0000120D549C1F8A802322016F0B0F900203C
:1021E000D2490860C82016F0AAF90120CE49C1F8EA
:1021F000A8024FF4FA7016F0A2F910BD10B5FFF75F
:102200008DFFFFF7DBFFC820FFF77CFEFF20FFF705
:1022100098FE9320FFF795FE4220FFF792FE3620AE
:10222000FFF770FEC820FFF78CFE3A20FFF76AFE2A
:102230005520FFF786FEC020FFF764FE1320FFF74E
:1022400080FE0E20FFF77DFEC120FFF75BFE02201F
:10225000FFF777FEC520FFF755FED320FFF771FE8D
:10226000B120FFF74FFE0020FFF76BFE1B20FFF7AA
:1022700068FEB420FFF746FE0220FFF762FEE02072
:10228000FFF740FE0020FFF75CFE0320FFF759FE3A
:102290000820FFF756FE0620FFF753FE1320FFF736
:1022A00050FE0920FFF74DFE3920FFF74AFE392086
:1022B000FFF747FE4820FFF744FE0220FFF741FEEC
:1022C0000A20FFF73EFE0820FFF73BFE1720FFF72E
:1022D00038FE1720FFF735FE0F20FFF732FEE12012
:1022E000FFF710FE0020FFF72CFE2820FFF729FE45
:1022F0002920FFF726FE0120FFF723FE0D20FFF720
:1023000020FE0320FFF71DFE3F20FFF71AFE3320BB
:10231000FFF717FE5220FFF714FE0420FFF711FE0F
:102320000F20FFF70EFE0E20FFF70BFE3720FFF702
:1023300008FE3820FFF705FE0F20FFF702FE1120F0
:10234000FFF7E0FD782016F0FAF82920FFF7DAFD14
:1023500010BD01B5BDF80010C8B2FFF7D3FD08BD30
:1023600001B5BDF80010C8B2FFF7EBFD08BD08B518
:10237000FFF725FE0090BDF8000008BD70B50546CA
:102380000C46E8B2FFF7BEFD2012FFF7DAFDE0B21F
:10239000FFF7D7FD70BD10B504462046FFF7D9FF03
:1023A000052002F008FCFFF7E2FF10BD10B52C205D
:1023B000FFF7A8FD10BD30B5014601F01F04C1F3C1
:1023C0004513CA0AE50205EB43151544A8B230BD12
:1023D00000BF011EA0F10102D0B2FAD1704770B562
:1023E00004460D4652494889FFF7B3FF2012FFF714
:1023F000B7FFE0B2FFF7B4FF4D498889FFF7A9FFA7
:102400002812FFF7ADFFE8B2FFF7AAFF70BD2DE974
:10241000F04104460D4600260027B0464448008897
:10242000A04203DD42484088A84202DC0020BDE80B
:10243000F08129462046FFF7D2FF2E20FFF789FFC3
:10244000FFF795FF06460220FFF7C2FFFFF78FFF59
:1024500006460220FFF7BCFFFFF789FF8046F7B270
:102460004FF6FF7000EA07273046FFF7A4FFDEE7CC
:1024700010B52920FFF76DFF10BD10B52820FFF71C
:1024800068FF10BD10B504463620FFF73BFD20461F
:10249000FFF757FD10BD70B504460D46294620468E
:1024A000FFF79DFFFFF782FFFFF720FC01201F4988
:1024B0001C3908601C49C1F894021E480088FFF7C7
:1024C0005EFD70BD70B504460D4616461849488934
:1024D000FFF73FFF2012FFF743FFE0B2FFF740FF97
:1024E00013498889FFF735FF2812FFF739FFE8B253
:1024F000FFF736FF0E49087AFFF704FDFFF7F6FBFA
:1025000001200A491C3908600749C1F8940213E008
:1025100000804042000002400004024000080240E7
:10252000000C0240BC82404200004142A8024142ED
:1025300058040020B40000203046FFF720FD70BD95
:1025400070B52DED048B0446BE20FFF702FF052079
:10255000FFF706FF20461CF0A3FA41EC190B9FED94
:10256000F70B53EC102B1CF0AFFA41EC180B1CF0DE
:1025700053FA85B22846FFF7F3FE0120FFF7F0FE7D
:10258000FF20FFF7EDFE0020FFF7EAFE0020FFF737
:10259000E7FEBDEC048B70BD18B90021E94A9171CA
:1025A00002E00121E74A91714FF4A071E54A1180E0
:1025B000F02151802A2151812B2191812C211181DF
:1025C00070472DE9F04704460D4616461F46A019F0
:1025D000401E1FFA80F8E819401E1FFA80F9D949F9
:1025E0004889FFF7B6FE2012FFF7BAFEE0B2FFF708
:1025F000B7FE4FEA2820FFF7B3FE08F0FF00FFF711
:10260000AFFED0498889FFF7A4FE2812FFF7A8FE85
:10261000E8B2FFF7A5FE4FEA2920FFF7A1FE09F077
:10262000FF00FFF79DFEBDE8F08710B549F241308D
:10263000C4498880FFF7E2FD49F24130C1498880F2
:102640000120FFF7A9FF10BD10B504462046FFF793
:10265000FEFC10BD2DE9F05F05460E461746984674
:10266000DDF828A04FF0000B781B401C1FFA80FB00
:1026700034461BE021462846FFF7B1FEFFF796FEE1
:10268000FFF734FB0120B0490860B049C1F894025B
:102690004FF0000906E05046FFF771FC09F1010018
:1026A0001FFA80F9D945F6DB601C84B24445E1DDB0
:1026B000BDE8F09F2DE9F84F07460D469046994634
:1026C000DDF828B0A8EB0700401C1FFA80FAA9EB40
:1026D0000500401C80B2009000241CE0281981B243
:1026E0003846FFF77CFEFFF761FEFFF7FFFA012097
:1026F000954908609549C1F89402002607E004FB5B
:102700000A613BF81100FFF73AFC701C86B256458F
:10271000F5DB601C84B200988442DFDBBDE8F88FF3
:102720002DE9FF4F85B081468A4600200490039032
:102730000798A0EB09050898A0EB0A06CDF80890C9
:10274000CDF804A0002D01DD012705E00DB900271B
:1027500002E04FF0FF376D42002E02DD4FF001081E
:1027600006E016B94FF0000802E04FF0FF3876425D
:10277000B54201DD2C4600E034464FF0000B21E06D
:10278000019A91B2029A90B2FFF785FE049828440C
:1027900004900398304403900498A04205DD049807
:1027A000001B04900298384402900398A04205DD73
:1027B0000398001B03900198404401900BF1010025
:1027C0001FFA80FB601C8345DADD09B0BDE8F08F9D
:1027D0002DE9F04104460D4616461F462B4632466B
:1027E00029462046FFF79CFF3B46224629462046C5
:1027F000FFF796FF3B46324639462046FFF790FFEB
:102800003B46324629463046FFF78AFFBDE8F08155
:102810002DE9F04706460F46904600244546032022
:10282000A0EB48093CE07A1B91B2321990B2FFF755
:1028300032FE3A1B91B2721990B2FFF72CFE3A1990
:1028400091B2721990B2FFF726FE7A1991B232193D
:1028500090B2FFF720FE7A1991B2321B90B2FFF7C7
:102860001AFE3A1991B2721B90B2FFF714FE7A1B4E
:1028700091B2321B90B2FFF70EFE3A1B91B2721B5F
:1028800090B2FFF708FE641CB9F1000F03DAA00054
:10289000801D814404E0601B80000A3081446D1E6D
:1028A000AC42C0DDBDE8F0872DE9F84F80460E460A
:1028B00017461C46B3462046E31704EB5373DB1060
:1028C00021464FEAE47C04EB5C7C4FEAEC0CA4EB81
:1028D000CC0CBCF1000F02D04FF0010C01E04FF026
:1028E000000C6344224604EBD27C4FEA6C0C03FBE1
:1028F0000CF3DBB20093A7F12000C7B2002566E01D
:102900000C2C07D107EB4700114901EB800010F8B0
:10291000059023E0102C05D10E4800EB071010F8AD
:1029200005901BE0182C07D107EBC7000A4901EB03
:10293000800010F8059011E0BDE8F88F66666666C5
:1029400066660440580400208C0241420000414267
:10295000CBEF01083FF401082FFA01084FF0000AFD
:102960002FE009F0800030B18F48028831464046A0
:10297000FFF7A8FD07E00A9828B98C48028831467D
:102980004046FFF79FFD4FEA49604FEA1069701C0F
:1029900086B287484088B04200DCCDE7A6EB0B004A
:1029A000A0420AD15E4608F101001FFA80F8804873
:1029B0000088404500DCBFE706E00AF1010000F0B6
:1029C000FF0ABAF1080FCCDB00BF681CC5B2009843
:1029D000854295DB00BFAFE710B50246012000E05D
:1029E00050430B1EA1F10104E1B2F9D110BD2DE954
:1029F000FF4F81B0074691461E460E9D4FF0000ADC
:102A0000002439E0301B401EC1B20A20FFF7E4FF6A
:102A1000B9FBF0F00A21B0FBF1F201FB1208BAF1A8
:102A2000000F16D1701EA04213DDB8F1000F0ED1B9
:102A30000020AB4605EBDB71491001FB04710090EF
:102A400088B22B4620220299FFF72EFF12E04FF0AA
:102A5000010A0020AB4605EBDB71491001FB047154
:102A6000009088B208F13001CAB22B460299FFF7F4
:102A70001BFF00BF601CC4B2B442C3DB05B0BDE89D
:102A8000F08F2DE9FF4F83B0064692461F46DDE9E1
:102A900010480020029000254DE0781B401EC1B276
:102AA0000A20FFF799FFBAFBF0F00A21B0FBF1F220
:102AB00001FB1209029850BB781EA84227DDB9F12C
:102AC000000F22D108F0800078B108F00100A34681
:102AD00004EBDB71491001FB0561009088B22346CD
:102AE00030220499FFF7E0FE0EE008F00100A34653
:102AF00004EBDB71491001FB0561009088B22346AD
:102B000020220499FFF7D0FE13E00120029008F084
:102B10000100A34604EBDB71491001FB0561009045
:102B200088B209F13001CAB223460499FFF7BCFE0E
:102B300000BF681CC5B2BD42AFDB07B0BDE8F08F77
:102B40002DE9F84F04460D4690469946DDE90A679F
:102B500004F0FF0A08EB04001FFA80F809EB0500F7
:102B60001FFA80F916E0444502DB5446A81985B2E5
:102B70004D4500DB14E0002000903A7833462946AA
:102B80002046FFF791FE304606EBD07104EB610161
:102B90008CB27F1C38787E2802DC38782028E2DA74
:102BA00000BFBDE8F88F0000B4000020B600002090
:102BB000580400207FB505460C460121480402F068
:102BC00065FC0295ADF804400020ADF80600ADF8B4
:102BD0000C0001A9264803F088FB01221146244875
:102BE00004F024F80121224803F008FC19208DF894
:102BF000000002208DF8010001208DF802008DF800
:102C00000300684602F057F87FBD10B50021194A4D
:102C100011605160632140F2E730FFF7CBFF10BD38
:102C200010B50121124804F018F801281AD11148F2
:102C300002684068521C40F100000E490A6048607A
:102C400001200EF073FB0C480068401C0A49086024
:102C500008460068B0F57A7F04D3FEF70AF8002032
:102C6000054908600121024804F008F810BD000081
:102C70000044014018000020BC0000201CB50020CA
:102C80000190009002F0CCF99948006840F480303F
:102C90009749086000BF9648006800F40030009033
:102CA0000198401C0190009818B90198B0F5A04F08
:102CB000F1D18F48006800F4003010B1012000907D
:102CC00001E0002000900098012846D1884840305B
:102CD000006840F0805086494031086085480068AF
:102CE00040F44040834908608148083000688049CA
:102CF000083108600846006840F400400860084653
:102D0000006840F4A05008607B48091F0860081F55
:102D1000006840F08070091F086000BF74480068B8
:102D200000F000700028F9D040F205707349086087
:102D30006F480830006820F003006D4908310860D2
:102D40000846006840F00200086000BF684808308C
:102D5000006800F00C000828F8D11CBD2DE9F843EC
:102D600004460D4616461F464FF0000802F058F97B
:102D7000012002F07EF902F0A1F98046B8F1010FBE
:102D800035D15B484030006840F0805058494031B0
:102D900008605848006840F44040564908600020E8
:102DA00002F02AFA4FF4A05002F030FA4FF48050AB
:102DB00002F036FA33462A4621464FF48000009747
:102DC00002F0BFF9012002F0CCF900BF392002F077
:102DD00057F90028FAD040F20570484908600220EF
:102DE00002F0FAF900BF02F001FA0828FBD1BDE8B1
:102DF000F8832DE9FC4104460D4616461F46002087
:102E0000019002F00DF9012002F07EF938480068C7
:102E100000F0020001900198022834D1344840307B
:102E2000006840F080503249403108603148006805
:102E300040F440402F490860002002F0DDF94FF4D3
:102E4000A05002F0E3F94FF4805002F0E9F9334664
:102E50002A4621460020009702F073F9012002F073
:102E600080F900BF392002F00BF90028FAD040F2B7
:102E7000057022490860022002F0AEF900BF02F09E
:102E8000B5F90828FBD1BDE8FC811CB50121084635
:102E900002F0A2FA4FF48070009002208DF8040036
:102EA00000208DF8060001208DF8070003208DF822
:102EB00005006946124801F0EFFF1CBD1CB5012159
:102EC000042002F089FA4FF40070009002208DF87F
:102ED000040000208DF8060001208DF80700032073
:102EE0008DF805006946074801F0D6FF1CBD0000BB
:102EF000003802400070004019544007003C024076
:102F0000000002400008024070471CB50121022069
:102F100002F062FA4FF48050009001208DF8040016
:102F200000208DF8060003208DF8050001208DF8A3
:102F300007006946324801F0AFFF4FF48051304836
:102F400002F028F81CBD1CB50121022002F044FA51
:102F50004FF480512A4802F01BF84FF48050009043
:102F600000208DF8040001208DF8060003208DF864
:102F7000050000208DF807006946214801F08CFF0C
:102F80001CBD1CB50121022002F026FA4FF4C070CE
:102F9000009001208DF8040000208DF80600032029
:102FA0008DF8050001208DF807006946154801F0ED
:102FB00073FF0020144908601449C1F8A0021CBD29
:102FC0001CB50121022002F007FA01200E49086019
:102FD0000E49C1F8A0024FF4C070009000208DF897
:102FE000040001208DF8060003208DF80500002064
:102FF0008DF807006946034801F04EFF1CBD000034
:1030000000040240000802409C024142000041428C
:103010002DE9F04104460F4615461E4600BF00BF8D
:1030200000BF02E0012016F07FFFA0780028F9D150
:103030000120A0702088C0F50060A8420DDB228826
:10304000E11C50182A4631461AF0A8FC2088284472
:1030500020800020A070BDE8F0810020A070012039
:10306000F9E701B56B46012211468B48FFF7D0FF07
:1030700008BD00BF00BF002141F26D02024482F88A
:103080000D1441F26D02024482F80C1441F26D02FB
:103090000244A2F80E14704710B57F481AF02EFFB4
:1030A00010BD704700BF00BF0021817001807047D4
:1030B00000BF00BF642300F60302C2F86638002395
:1030C000A2F8643859B1002105E0002300F603029C
:1030D00053544A1C91B240F664029142F5DB7047AA
:1030E00030B587B005460C460121084602F074F958
:1030F0000121102002F0CAF907220921674801F0D6
:1031000056FF07220A21654801F051FF4FF4C060C5
:10311000059002208DF818008DF8190000208DF818
:103120001A0001208DF81B0005A95C4801F0B4FECF
:1031300001940020ADF80800ADF80A00ADF80C00CD
:10314000ADF810000C20ADF80E0001A9544802F0B3
:10315000FEFA0121524802F082FB012240F2255181
:103160004F4802F032FC012240F226614C4802F046
:103170002CFC25208DF8000003208DF801008DF82F
:10318000020001208DF80300684601F094FD00BFA5
:1031900000BF20212846FFF78BFF2846FFF769FF75
:1031A0002846FFF77FFF07B030BD70B505460C46D7
:1031B00020461AF083FB86B2234632460121284678
:1031C000FFF726FF70BD70B5044600BF00BF208822
:1031D00008B9002070BD02E0012016F0A5FEA0781D
:1031E0000028F9D10120A07002E0012016F09CFE19
:1031F00041F26D00204490F80D040028F5D120889C
:10320000B0F5806F01DC258801E04FF480652A4627
:10321000E11C41F26D0020441AF0C0FB2088421BE3
:10322000E01C41191AF0BAFB2088401B208041F2B3
:103230006D002044A0F80E5441F26D00211804F5F1
:103240008050C0F87D1441F26D002044B0F80E04A7
:10325000401E41F26D012144A1F80E0404F5805096
:10326000D0F87D24D0F87D04401C04F58051C1F8CD
:103270007D0410780A4988800020A070012041F266
:103280006D01214481F80D040020A3E700B5024838
:10329000FFF707FF00BD00006604002000000240A9
:1032A0000010014000210170704770B58AB00646D9
:1032B0000C4615460121022002F0D7F80121042016
:1032C00002F08AF84FF40070089002208DF8240074
:1032D00003208DF8250000208DF8260001208DF8B0
:1032E000270008A9344801F0D7FD022209213248FD
:1032F00001F05DFEA8B2ADF814000020ADF8160094
:103300000694ADF81C0005A92C4802F0EEFF6020E1
:10331000ADF800000120ADF802000020ADF80C006F
:10332000600802906946254803F060F908212348A7
:1033300003F01CFA0121214803F042F801211F4843
:1033400003F05CF80AB070BD70B504460D4600206D
:1033500020701B48B0FBF5F6711E63222046FFF774
:10336000A4FF70BD10B50446207801280DD1134884
:103370002030008840F4805010492031088014200B
:1033800016F0D2FD002020700AE02078022807D035
:103390000A482030008820F48050084920310880F5
:1033A00010BD01210170704702210170704700B506
:1033B0000448FFF777FF00BD00080240000400400A
:1033C00040420F00CA000020704770B505460C4609
:1033D00000BF02216E4803F03DFF0028F9D02146CE
:1033E0006B4803F0EEFE00BF0121694803F032FF95
:1033F0000028F9D0664803F0E1FEC0B270BD70B598
:1034000005460C46624800884FF6C771084060497F
:103410000880084600882043088001215C4803F0AA
:103420004FFE70BD10B588B004460121022001F0A6
:10343000D3FF0121080302F029F8C02006900120E3
:103440008DF81C0000208DF81E0003208DF81D0053
:1034500001208DF81F0006A94E4801F01DFD4021F6
:103460004C4801F095FD80214A4801F091FD38203B
:10347000069002208DF81C0000208DF81E0003200D
:103480008DF81D0001208DF81F0006A9414801F0AC
:1034900003FD052203213F4801F089FD0522042197
:1034A0003C4801F084FD052211463A4801F07FFDB9
:1034B0000121080302F03FF800214FF4805002F090
:1034C0003AF80020ADF804004FF48270ADF8060021
:1034D0000020ADF808000220ADF80A000120ADF888
:1034E0000C004002ADF80E003820ADF810000020AE
:1034F000ADF812000720ADF8140001A9244803F02C
:10350000E5FC10212448FFF77AFF0121204803F051
:10351000D7FDFF212046FFF758FF08B010BD70B55A
:1035200005460C4600BF0221194803F093FE00280F
:10353000F9D02146164803F044FE00BF012114488B
:1035400003F088FE0028F9D0114803F037FEC0B21E
:1035500070BD10B5044600BF02210D4803F07AFE8D
:103560000028F9D0FF210A4803F02BFE00BF0121FB
:10357000074803F06FFE0028F9D0054803F01EFE4F
:10358000C0B210BD00B50448FFF71EFF00BD00002B
:103590000030014000040240EF18002000210DE03F
:1035A000002207E000BF00BF00BF00BF00BF00BF98
:1035B000531CDAB2022AF5DB4B1C99B28142EFDBD5
:1035C000704770471CB504460121022001F004FF3A
:1035D00044F20800009001208DF8040000208DF8CE
:1035E000060001208DF8070002208DF805006946CD
:1035F000944801F051FC1020009000208DF8040048
:103600008DF8070069468F4801F046FC1CBD70B577
:10361000054602E0012016F087FC8B48007801285F
:10362000F8D00120884908704021864801F0B2FC9A
:103630008021844801F0ACFC00BF00BF0521834815
:10364000FFF76DFF8148FFF784FF044640217D4866
:1036500001F09EFC00BF00BF00207B49087020469F
:1036600070BD70B505460C464021764801F092FCCD
:103670008021744801F08CFC00BF00BF0121734819
:10368000FFF74DFF21467148FFF749FF40216D4884
:1036900001F07EFC00BF00BF70BD2DE9F8438046FD
:1036A0000E4617461C4602E0012016F03DFC664817
:1036B00000780128F8D00120634908700096402165
:1036C000604801F067FC80215E4801F061FC00BFAA
:1036D00000BF03215D48FFF722FF9DF801105B4802
:1036E000FFF71DFF9DF800105848FFF718FF002551
:1036F00006E05648FFF72DFF2070641C681C85B259
:10370000BD42F6DB40214F4801F042FC00BF00BF44
:1037100000204D490870BDE8F8832DE9F843804644
:103720000E4617461C4602E0012016F0FDFB4648F7
:1037300000780128F8D00120434908700096402104
:10374000404801F027FC80213E4801F021FC00BFE9
:1037500000BF06213D48FFF7E2FE4021394801F055
:1037600017FC00BF00BF0120FFF718FF40213548BC
:1037700001F010FC8021334801F00AFC00BF00BFBB
:1037800002213248FFF7CBFE9DF801102F48FFF7CA
:10379000C6FE9DF800102D48FFF7C1FE002506E08B
:1037A00021782A48FFF7BBFE641C681C85B2BD4225
:1037B000F6DB4021234801F0EBFB00BF00BF0120F6
:1037C000FFF7ECFE40211F4801F0E4FB80211D487B
:1037D00001F0DEFB00BF00BF04211C48FFF79FFE85
:1037E0004021184801F0D4FB00BF00BF022016F0B2
:1037F0009BFB002014490870BDE8F88338B50546E6
:103800000C4600BF00BF6B46022221461048FFF75E
:1038100044FF00BF00BFBDF8000038BDF8B5064644
:103820000D46144600946B46022229460848FFF7CD
:1038300074FF00BF00BFF8BD00B50548FFF7C1FE2B
:1038400000BD000000040240CB000020EF18002063
:10385000F01800207047704770B505460C4680216F
:10386000FC4801F097FB4021FA4801F091FB00BFB2
:1038700000BF9F21F848FFF752FEF748FFF769FEA7
:103880002070641CF448FFF764FE2070641CF2484A
:10389000FFF75FFE2070641C8021EE4801F078FB8A
:1038A00000BF00BF70BD30B589B004460D4601A908
:1038B0002046FFF7D1FF9DF806008DF808009DF81F
:1038C00005008DF809009DF804008DF80A0000201D
:1038D0008DF80B00E14902980861E1A1E548FFF786
:1038E00064FCDE480069059005AB04220121E14833
:1038F000FFF78EFBE0A1DF48FFF757FC002009B07F
:1039000030BD70B5054602E0012016F00DFBDB4826
:1039100000780128F8D00120D84908708021CD48CE
:1039200001F038FB4021CB4801F032FB00BF00BF63
:103930000521C948FFF7F3FDC748FFF70AFE044613
:103940008021C44801F024FB00BF00BF0020CB4908
:103950000870204670BD70B505460C468021BD48F4
:1039600001F018FB4021BB4801F012FB00BF00BF73
:103970000121B948FFF7D3FD2146B748FFF7CFFD36
:103980008021B44801F004FB00BF00BF70BD38B512
:1039900005460C4602E0012016F0C6FAB74800784A
:1039A0000128F8D00120B54908708021A94801F00C
:1039B000F1FA4021A74801F0EBFA00BF00BF062151
:1039C000A548FFF7ACFD8021A24801F0E1FA00BF55
:1039D00000BF0121AA48FDF7A3F880219D4801F00E
:1039E000D9FA40219B4801F0D3FA00BF00BF200361
:1039F000009020219848FFF792FD9DF8021096480C
:103A0000FFF78DFD9DF801109348FFF788FD9DF8A5
:103A100000109148FFF783FD80218E4801F0B8FA2D
:103A200000BF00BF00209549087038BD38B5054675
:103A30000C4602E0012016F077FA90480078012841
:103A4000F8D001208D4908708021824801F0A2FA47
:103A50004021804801F09CFA00BF00BF06217E484B
:103A6000FFF75DFD80217B4801F092FA00BF00BFA7
:103A700001218348FDF754F88021764801F08AFA45
:103A80004021744801F084FA00BF00BF2004009078
:103A9000D8217148FFF743FD9DF802106E48FFF7EB
:103AA0003EFD9DF801106C48FFF739FD9DF80010B0
:103AB0006948FFF734FD8021664801F069FA00BFCC
:103AC00000BF00206D49087038BD10B5044602E003
:103AD000012016F029FA694800780128F8D0012061
:103AE0006649087080215B4801F054FA402159482A
:103AF00001F04EFA00BF00BF06215748FFF70FFD47
:103B00008021544801F044FA00BF00BF01215C4805
:103B1000FDF706F880214F4801F03CFA40214D485E
:103B200001F036FA00BF00BFC7214B48FFF7F7FC92
:103B30008021484801F02CFA00BF00BF00204F4907
:103B4000087010BDF8B507460E46144602E0012085
:103B500016F0EAF9494800780128F8D001204749D1
:103B60000870009680213B4801F014FA4021394842
:103B700001F00EFA00BF00BF03213748FFF7CFFC6A
:103B80009DF801103448FFF7CAFC9DF80010324838
:103B9000FFF7C5FC00213048FFF7C1FC002506E017
:103BA0002D48FFF7D6FC04F8010B681C85B2FF2DE9
:103BB000F6D98021274801F0EBF900BF00BF0020B3
:103BC0002E490870F8BDF8B507460E46144602E0C7
:103BD000012016F0A9F9294800780128F8D0012021
:103BE0002649087080211B4801F0D4F9402119486A
:103BF00001F0CEF900BF00BF06211748FFF78FFC88
:103C00008021144801F0C4F900BF00BF01211C4805
:103C1000FCF786FF009680210E4801F0BBF9402199
:103C20000C4801F0B5F900BF00BF02210A48FFF7B8
:103C300076FC9DF801100848FFF771FC9DF8001014
:103C40000548FFF76CFC00210348FFF768FC0025DE
:103C500024E0000000040240EF180020F4180020C7
:103C6000466C617368205465737420446174613AD2
:103C700000000000660400200D0A0000CB000020B8
:103C8000AC0000202178C148FFF749FC641C217872
:103C9000BE48FFF744FC641C681C85B2802DF1D33C
:103CA0008021BB4801F074F900BF00BF0020B94972
:103CB0000870F8BD10B50446B921B448FFF72FFCD1
:103CC00010BD10B504468021B14801F063F94021D0
:103CD000AF4801F05DF900BF00BFAB21AB48FFF773
:103CE0001EFC8021AA4801F053F900BF00BF10BD9F
:103CF00070B506460C4600250DE0A748FFF701FE0B
:103D000000F0010018B1012016F00EF901E00020CA
:103D100070BD681C85B2A542EFDB0120F8E72DE9F4
:103D2000F04107460D46164600240EE04FF4FA71A6
:103D30003846FFF7DDFF29193846FFF777FEC8211F
:103D40003846FFF7D5FF601C84B2B442EEDB00209A
:103D5000BDE8F0812DE9F05F04468946154602E092
:103D6000012016F0E1F820780028F9D10120207018
:103D70000DB10A2D00DD03254FF0000835E0642168
:103D80002046FFF7B5FF49462046FFF700FE6421B5
:103D90002046FFF7ADFF4FF0000A4FEA091B00264F
:103DA00017E00BEB0601621C2046FFF7CBFE002755
:103DB00007E0601CC05DFF2802D04FF0010A02E05E
:103DC0007F1CFF2FF5D900BFBAF1010F00D102E02F
:103DD000761C102EE5D300BFBAF1000F03D10020EE
:103DE0002070BDE8F09F08F10108A845C7D3002066
:103DF00020700120F5E72DE9FF5F04460E461F46BF
:103E000002E0012016F090F820780028F9D1012076
:103E100020700FB10A2F00DD032731462046029A99
:103E2000FFF7D1FE0A212046FFF762FF621C3146F0
:103E30002046FFF787FE4FF48072611C029819F04C
:103E4000EDFC00287ED055A15948FFF7AEF94FEAA6
:103E50001618A6EB081000F1010B4FEA081955A13E
:103E60005348FFF7A2F900224FF48051584813F04D
:103E7000F5FF002508E0564800EB052209EB050197
:103E80002046FFF75FFE6D1C5D45F4D34FF0000A3E
:103E900064E050A14648FFF788F9002020703109FE
:103EA0000A223D48FFF756FF002853D10120207019
:103EB0004CA13F48FFF779F9002520E0444800EB8A
:103EC000052209EB05012046FFF77DFE0A21204669
:103ED000FFF70EFF09EB0501621C2046FFF732FEDB
:103EE0003B4901EB05204FF48072611C19F096FCF0
:103EF00020B146A12E48FFF758F902E06D1C5D4540
:103F0000DCD300BF4AA12A48FFF74FF931462046CB
:103F1000029AFFF758FE0A212046FFF7E9FE621CCD
:103F200031462046FFF70EFE4FF48072611C029866
:103F300019F074FC50B944A11D48FFF736F9002070
:103F4000207000E00DE004B0BDE8F09F44A11848E7
:103F5000FFF72BF9012020700AF1010ABA4598D326
:103F600007E00020207039A11148FFF71EF900205A
:103F7000E7E70020207040A10D48FFF716F9012067
:103F8000DFE700B50448FFF765FC00BDEF1800202F
:103F900000040240CB0000200E1A0020666C617302
:103FA0006820C3BBB1A3B4E6D5FDC8B70D0A0000B5
:103FB00066040020B0D1B5B1C7B0C9C8C7F8CAFD02
:103FC000BEDDD4DDB4E6D4DAC4DAB4E60D0A00000E
:103FD000131B0020B2C1B3FDB5B1C7B0C9C8C7F843
:103FE0000D0A0000CAB9D3C3D2D1B1A3B4E6B5C497
:103FF000C4DAB4E6CAFDBEDDD6D8D0C2D0B4B5B1FD
:10400000C7B0C9C8C7F80D0A00000000BBD8D0B4BB
:10401000D4F8BEADB1A3B4E6D4DAB5B1C7B0C9C85F
:10402000C7F8CAFDBEDDD3D0CEF30D0A00000000F4
:10403000D0B4B5B1C7B0D2B3D2AAB1A3B4E6B5C4B7
:10404000CAFDBEDD0D0A0000D6D8D0C2B1A3B4E6C9
:10405000464C415348CAFDBEDDD5FDC8B70D0A0028
:10406000D6D8D0C2B1A3B4E6464C415348CAFDBE2F
:10407000DDB4EDCEF30D0A00666C617368207772D3
:10408000697465206572726F720D0A0070472DE9C0
:10409000F04180460D46A04801F045FE074602214A
:1040A0009D4801F02EFF002D02DD681E84B200E065
:1040B00003244FF6FF7000EA043404F47044C7F39D
:1040C0000B0727439548465D122E02D1012001F0CF
:1040D00070FD0723012231468F4801F08CFD8E4888
:1040E00001F0E5FD3846BDE8F08110B58CB004461E
:1040F0000121042001F070F90121080201F0C6F944
:1041000007200A9003208DF82C0000208DF82F0046
:104110000AA9834800F0C0FE0121080201F00BFA51
:1041200000214FF4807001F006FA002006900990FB
:1041300008904FF48030079006A801F005FD00209C
:1041400000908DF804008DF8050002900490012085
:104150008DF814006946704801F0C7FC6E4880680D
:1041600020F410606C498860012001F022FD0121DB
:10417000694801F000FD012014F0E1F9002120461A
:10418000FFF785FF012014F0DAF900212046FFF740
:104190007EFF012084F83E00002020870CB010BD77
:1041A0002DE9F047044600BF00BF54F83A0F401C09
:1041B000206021793A3C2046FFF769FF8046474658
:1041C0003F13C8F30B0807EB870004EB4000218F77
:1041D00020F811804FF0000A00260AE007EB870064
:1041E00004EB400030F81A0006440AF1010000F028
:1041F000FF0ABAF1050FF1DB0520B6FBF0F081B242
:1042000004F1280020F8171030F8176041F6797093
:10421000464342F21070B6FBF0F604F1300020F88D
:104220001760B5B237B1012F2ED0022F2DD0032F3A
:1042300045D135E040F2FA466E434FF47A70B6FB52
:10424000F0F085B2B5F57A6F03DB042035490880BC
:1042500019E040F6D860854203DB0320314908802D
:1042600011E0B5F5616F03DB02202E4908800AE0FA
:1042700040F64850854203DB01202A49088002E0CD
:104280000020284908801BE01AE0A08D14F06EF988
:104290002549088008460088C01F00B208800FE04A
:1042A000A94609EB89004FEA4009A9F58059A9F50B
:1042B0005B69192099FBF0F909F1190900E000BFC9
:1042C00000BF00BF00BF00BF00BF94F83E00401C0D
:1042D000C0B284F83E0003280ADB002084F83E00C8
:1042E000208F401C2087208F052801DB002020879D
:1042F000BDE8F0870246002006E002F1300333F803
:10430000103021F81030401C0428F6D3704700B557
:104310000648FFF7BBFE00BD00200140CC00002096
:10432000000802403800002036000020142B002036
:1043300000BF00BF704770477047F0B505460020CA
:1043400092F903400A2694FBF6F430341C54401CC6
:1043500092F9034094FBF6F706FB174430341C54E3
:10436000401C19B13A241C54441CE0B292F9044098
:104370000A2694FBF6F430341C54441CE0B292F943
:10438000044094FBF6F706FB174430341C54441CDD
:10439000E0B219B13A241C54441CE0B292F9054031
:1043A0000A2694FBF6F430341C54441CE0B292F913
:1043B000054094FBF6F706FB174430341C54441CAC
:1043C000E0B2F0BD70B50346002093F907400A251E
:1043D00094FBF5F430341454401C93F9074094FBDB
:1043E000F5F605FB164430341454401C19B13A2438
:1043F0001454441CE0B293F908400A2594FBF5F4E8
:1044000030341454441CE0B293F9084094FBF5F6A0
:1044100005FB164430341454441CE0B219B13A245C
:104420001454441CE0B293F909400A2594FBF5F4B6
:1044300030341454441CE0B293F9094094FBF5F66F
:1044400005FB164430341454441CE0B270BD10B562
:104450000246002091F90030002B03DB91F9003077
:10446000632B00DD012091F90130012B03DB91F971
:1044700001300C2B00DD022091F90230012B03DB0F
:1044800091F902301F2B00DD032091F90330002B3E
:1044900003DB91F90330172B00DD042091F9043080
:1044A000002B03DB91F904303B2B00DD052091F953
:1044B0000530002B03DB91F905303B2B00DD062096
:1044C000B1F90630B3F5FA6F05DBB1F9063040F605
:1044D0003404A34200DD072010BD70472DE9F04FE2
:1044E0008046FE48814202D90120BDE8F08F0025B8
:1044F00000230DE0FA4EFB48405D08B1FA4806443F
:10450000B14200D206E0581C03B2891B681CC5B238
:10451000642DEFDB00BF58B2107003F5FA6000B2F3
:10452000D080F04810F803C00025012411E0EF48C6
:104530004657ED484643BCF1000F02D0022C00D193
:104540000644B14200D206E0601CC4B2891B681C5C
:10455000C5B20C2DEBDB00BF60B25070E248B1FB7E
:10456000F0F040B290709078401C40B29070DE48FD
:10457000B1FBF0F900FB19114FF46160B1FBF0F0F1
:1045800040B2D0704FF46160B1FBF0F900FB19113B
:104590003C20B1FBF0F040B210713C20B1FBF0F9CF
:1045A00000FB191040B25071B2F906305478977878
:1045B000012C01D0022C04D104F10C00C4B2581E0D
:1045C00003B204F1010909EB49094FF0050A99FB0F
:1045D000FAF94FF0020A0AFB047AD14499441846CA
:1045E0004FEAE37A03EB9A7A09EBAA094FF0640ADF
:1045F00093FBFAFAA9EB0A094FF4C87A93FBFAFA8B
:10460000D14409F101094FF0070A99FBFAFB0AFBB3
:104610001B994FFA89F982F80A90002065E770B576
:1046200004460E4600BF00BF251D2A4631462046DF
:10463000FFF754FF29462046FFF74FFF00BF00BF9A
:1046400070BD02790A7042794A7082798A70C279A3
:10465000CA70027A0A71427A4A714289CA80828992
:104660000A81827B8A727047704770B504460D4696
:10467000207913F01AF940B22870607913F015F917
:1046800040B26870A07913F010F940B2A870E079D8
:1046900013F00BF940B2E870207A13F006F940B23B
:1046A0002871607A13F001F940B26871A07B13F0B1
:1046B000FCF840B2A87270BD2DE9F04F83460C465D
:1046C00000BF00BFB4F90600B0F5FA6F07DA94F93D
:1046D0000000E080E08800F5FA6000B2E08021464A
:1046E0005846FFF7B4FE054615B10020BDE8F08F2F
:1046F000B4F90680A8F5FA600FFA80F800250027C3
:1047000008E0774807447748405D08B17648074499
:10471000681CC5B24545F4DB724810F808A094F94E
:104720000100401E724931F9106094F902000644FC
:10473000761EBAF1000F04D094F90100022800DDC2
:10474000761C94F903004FF4616110FB01F094F9B9
:104750000410C1EB011100EB810094F9051000EB8E
:104760000109B94440F2A320704309EBC01948463F
:10477000BCE730B50446251D29462046FFF79CFFBF
:1047800030BD2DE9F04704460E46914631460220E1
:1047900013F0CBFA8046B8F1000F01D1182000E0E9
:1047A00040464FF4616100FB01F5B11C022013F09B
:1047B000BCFA8046C8EB081005EB8005311D0220CD
:1047C00013F0B3FA80464544E07908B9182001E0B7
:1047D00094F907004FF46161484394F90810C1EB64
:1047E000011100EB810194F909000F18E81B002862
:1047F00002DC781B484502D20120BDE8F08700208A
:10480000FBE7C2790A70027A4A70427A8A7070476E
:104810002DE9F04180460F4616461D460424F188D6
:1048200088B2294613F01EFA1FB12D202855601CAE
:10483000C4B296F901000A2190FBF1F030302855FE
:10484000601CC4B296F9010090FBF1F201FB12006A
:1048500030302855601CC4B21FB12D202855601C73
:10486000C4B296F902000A2190FBF1F030302855CD
:10487000601CC4B296F9020090FBF1F201FB120039
:1048800030302855601CC4B21FB120202855601C50
:10489000C4B22B19324639464046FFF74EFDBDE8FB
:1048A000F08114490968491C124A1160704770B5BB
:1048B00006460C464FF4FA65207813F00DF80544CF
:1048C000E580207813F008F840B22070607813F08B
:1048D00003F840B26070E0780EE00000801319BC6D
:1048E0008033E10198070208805101008C0702081B
:1048F000FC0702084800002012F0EEFF40B2E07012
:10490000A07812F0E9FF40B2A070207912F0E4FF25
:1049100040B22071607912F0DFFF40B26071214631
:104920003046FFF7C9FE70BD7FB505460E461446FA
:1049300010222146684618F0ECFF6A4631462846A8
:10494000FFF7CCFD9DF8000012F0AFFF40B22070E1
:104950009DF8010012F0A9FF40B260709DF80200BE
:1049600012F0A3FF40B2A0709DF8030012F09DFF6B
:1049700040B2E0709DF8040012F097FF40B2207141
:104980009DF8050012F091FF40B260719DF80A0099
:1049900012F08BFF40B2A0727FBD2DE9FF47804629
:1049A0000C461546E01D13F013FB00B2ADF80600EF
:1049B000BDF90600642190FBF1F201FB120040B248
:1049C0008DF800005CA1204619F004FB18B101200D
:1049D0008DF801006EE058A1204619F0FBFA18B1DD
:1049E00001208DF8010065E054A1204619F0F2FA8B
:1049F00018B102208DF801005CE051A1204619F0A9
:104A0000E9FA18B103208DF8010053E04DA12046CA
:104A100019F0E0FA18B104208DF801004AE04AA12B
:104A2000204619F0D7FA18B105208DF8010041E0B1
:104A300046A1204619F0CEFA18B106208DF80100E3
:104A400038E043A1204619F0C5FA18B107208DF8C7
:104A500001002FE03FA1204619F0BCFA18B1082050
:104A60008DF8010026E03CA1204619F0B3FA18B1F8
:104A700009208DF801001DE038A1204619F0AAFA9E
:104A800018B10A208DF8010014E035A1204619F074
:104A9000A1FA18B10C208DF801000BE031A12046DD
:104AA00019F098FA18B10C208DF8010002E00C20E2
:104AB0008DF8010026796779A7F1300040B28DF8B2
:104AC0000200312E06D19DF802000A3040B28DF866
:104AD000020010E0322E06D19DF80200143040B2E0
:104AE0008DF8020007E0332E05D19DF802001E303C
:104AF00040B28DF80200284613F06AFA40B28DF8F1
:104B00000300E81C13F064FA40B28DF80400A81DFD
:104B100013F05EFA40B28DF8050069464046FFF793
:104B2000CBFD8146484604B0BDE8F08700B50E488D
:104B3000FFF701FC00BD00004A616E00466562009F
:104B40004D617200417072004D6179004A756E00CE
:104B50004A756C0041756700536570004F637400BF
:104B60004E6F760044656300542B002010B515F09D
:104B70003AFF012801D016F0CBFE10BD70B50446F7
:104B8000042000F0E5F83248047025464FF47A70AE
:104B9000454301202F4908804FF0E020006940F094
:104BA00002004FF0E021086108464561006940F0CD
:104BB0000100086170BD70B5034600224FF0E02689
:104BC0007569234E367803FB06F44FF0E026B16991
:104BD00010E04FF0E026B06988420BD0884202D244
:104BE0000E1A324402E02E1A0E4432440146A2420A
:104BF00000D300E0EDE700BF70BD70B5044615F0CE
:104C0000F2FE012810D013480088844206D31148D0
:104C10000088B4FBF0F5284615F086F90D480088A9
:104C2000B4FBF0F100FB11444FF47A7104FB01F086
:104C3000FFF7C1FF70BD30B50446002504E04FF416
:104C40007A70FFF7B8FF6D1CA542F8D330BD0000A5
:104C5000D0000020D200002000BF704770B504468D
:104C60000D46E0B2FEF7FDF9204670BD09488047C9
:104C700009480047FEE7FEE7FEE7FEE7FEE7FEE73E
:104C8000FEE7FEE7FEE7FEE704480549054A064B56
:104C900070470000DF03000889010008F04303208B
:104CA000F04D0320F0450320F04503203249014335
:104CB000324A1160704770B5002100230F22C4787A
:104CC0001CB32E4C246804F4E064C4F5E064C4F31F
:104CD0000721C1F10404E3B20A4144789C40E1B2E7
:104CE0008478144021430C07210E254C057861552A
:104CF000047804F01F050124AC4005786D11AD0067
:104D000005F1E025C5F8004109E0047804F01F052D
:104D10000124AC401B4D0678761145F8264070BD45
:104D2000194A0A400243154B1B1F1A60704739B1DC
:104D3000124A121D12680243104B1B1D1A6006E036
:104D40000E4A121D126882430C4B1B1D1A607047DD
:104D5000042808D14FF0E021096941F004014FF027
:104D6000E022116107E04FF0E021096921F0040120
:104D70004FF0E022116170470000FA050CED00E0F1
:104D800000E400E080E100E080FFFF1F10B5044672
:104D90009848844208D10121084600F088FB002190
:104DA000012000F084FB76E09348844208D1012181
:104DB000022000F07CFB0021022000F078FB6AE07A
:104DC0008E48844208D10121042000F070FB0021AC
:104DD000042000F06CFB5EE08948844208D1012188
:104DE000082000F064FB0021082000F060FB52E086
:104DF0008448844208D10121102000F058FB002192
:104E0000102000F054FB46E07F48844208D1012185
:104E1000202000F04CFB0021202000F048FB3AE06D
:104E20007A48844208D10121402000F040FB002153
:104E3000402000F03CFB2EE07548844208D101215F
:104E4000802000F034FB0021802000F030FB22E0C5
:104E50007048844208D10121801500F028FB002110
:104E6000A01500F024FB16E06B48844208D1012114
:104E7000401500F01CFB0021601500F018FB0AE053
:104E80006648844207D10121001500F010FB002183
:104E9000201500F00CFB10BDF0B50A4600210023E0
:104EA000002400BF3DE0012505FA01F3156805EA7D
:104EB00003049C4234D105684F000326BE40B5432D
:104EC000056015794E00B5400668354305601579D3
:104ED000012D02D01579022D16D185684F000326C9
:104EE000BE40B543856055794E00B5408668354370
:104EF0008560456801268E40B543456045689679D2
:104F00008E40B6B235434560C5684F000326BE40AB
:104F1000B543C560D5794E00B540C6683543C56018
:104F2000491C1029BFD3F0BD4FF6FF71016000216D
:104F3000017141718171C171704708B54FF48032C0
:104F40000092009A0A430092009AC261C161009ADD
:104F5000C261C2690092C269009208BD0246002087
:104F600013690B400BB1012000E00020704701469F
:104F7000086980B270470246002053690B400BB1AC
:104F8000012000E0002070470146486980B2704768
:104F900001837047418370470AB1018300E0418378
:104FA00070474161704742694A4042617047F0B5BD
:104FB000002300244D07ED0E02FA05F3CE1000F198
:104FC000200555F826504E07F70E0F26BE40B54374
:104FD000CF1000F1200646F82750CE1000F1200532
:104FE00055F8265045EA0304CE1000F1200545F897
:104FF0002640F0BD000002400004024000080240CC
:10500000000C024000100240001402400018024050
:10501000001C024000200240002402400028024000
:10502000FA48006840F00100F84908600020F7499C
:1050300008310860F5480068F5490840F349086000
:10504000F448091D0860F448F04984310860F148CB
:105050001038091D0860ED48006820F48020EB49F5
:1050600008600020E9490C310860E8498C3108608B
:1050700070470021E54A921C117011460870704774
:1050800010B501460022002300204A11012A02D156
:10509000DE4C236808E0022A03D1DC4C703423681C
:1050A00002E0DA4C7434236801F01F0201249440BA
:1050B0001C400CB1012000E0002010BD38B50020DC
:1050C00000900024002500BF3120FFF7D9FF0546DE
:1050D0000098401C00900098B0F5A04F01D0002D22
:1050E000F2D03120FFF7CCFF08B1012400E000240A
:1050F000204638BD01460020C44A106820F0F80060
:1051000040EAC10010607047C44908607047002140
:10511000BE4A703211701170012802D004280AD1E1
:1051200004E00121B94A7032117005E00521B74A47
:105130007032117000E000BF00BF7047B8490860CE
:10514000704770B5049C41EA82150126C6EB5306F0
:1051500045EA0645054345EA0465AC4E361D356013
:1051600070BDAE490866704710B5830143EA01730C
:105170001343A64C8434236010BDA8498866704749
:1051800010B5830143EA016343EA02739F4C8834FC
:10519000236010BDA14908677047A049C8647047E3
:1051A00002460020994B0833186820F0EC6042EA70
:1051B00001031843954B08331860704702460020DE
:1051C000924B0833186820F0784042EA01031843F4
:1051D0008E4B083318607047014600208B4A083216
:1051E000106820F0030008431060704787480830BB
:1051F000006800F00C00704701460020834A083226
:10520000106820F0F000084310607047014600204D
:105210007E4A0832106820F4E0500843106070475E
:1052200001460020794A0832106820F4604040EAC4
:10523000C10010607047F0B5002100220024022553
:1052400000260223714F08373F6807F00C0121B197
:10525000042905D0082937D105E0724F076036E0F0
:10526000714F076033E0694F3F1D3F68C7F38056B9
:10527000664F3F1D3F6807F03F036EB16A4FB7FBB3
:10528000F3F7DFF888C10CF1040CDCF800C0CCF3B4
:10529000881C07FB0CF40CE0624FB7FBF3F7DFF858
:1052A0006CC10CF1040CDCF800C0CCF3881C07FBCB
:1052B0000CF4564F3F1D3F68C7F301477F1C7D002C
:1052C000B4FBF5F7076002E0564F076000BF00BF70
:1052D0004E4F08373F6807F0F0010909534F7A5CD9
:1052E0000768D7404760494F08373F6807F4E051E7
:1052F000890A4E4F7A5C4768D7408760434F08372A
:105300003F6807F46041490B484F7A5C4768D740D3
:10531000C760F0BD002100F44072B2F5407F0AD1B1
:105320003A4A0832116821F4F811414A0240114307
:10533000364A08321160354A70321268C0F30B03E6
:105340001A43324B70331A6070473549443908604C
:1053500070473349403908607047364908607047E4
:1053600001460020294A8C32106820F01F004A1E96
:105370001043264A8C321060704701460020234AB1
:105380008C32106820F4F8504A1E40EA02201F4A6E
:105390008C3210607047014600201C4A8C32106825
:1053A00020F4401008431060704701460020174A5F
:1053B0008C32106820F440000843106070470146AA
:1053C0000020124A8C32106820F4403008431060EC
:1053D000704719490860704739B10C4A3032126879
:1053E00002430A4B30331A6006E0084A3032126832
:1053F0008243064B30331A607047F9B1034A3432A6
:1054000012680243014B34331A601CE0003802403A
:10541000FFFFF6EA10300024003000200000474271
:10542000800E47420024F40000127A00D8000020C9
:10543000FFFCFF0F5C014742E01147428F4A1268B0
:1054400082438E4B1A60704739B18C4A121D126824
:1054500002438A4B1B1D1A6006E0884A121D12681F
:105460008243864B1B1D1A60704739B1834A0C3248
:1054700012680243814B0C331A6006E07F4A0C32FB
:10548000126882437D4B0C331A60704739B17B4AF6
:10549000103212680243794B10331A6006E0774AE3
:1054A000103212688243754B10331A60704739B15D
:1054B000724A243A12680243704B243B1A6006E099
:1054C0006E4A243A126882436C4B243B1A60704740
:1054D00039B16A4A203A12680243684B203B1A608D
:1054E00006E0664A203A12688243644B203B1A6009
:1054F000704739B1614A1C3A126802435F4B1C3B4A
:105500001A6006E05D4A1C3A126882435B4B1C3B02
:105510001A60704739B1594A143A12680243574B1E
:10552000143B1A6006E0554A143A12688243534B02
:10553000143B1A60704739B1504A103A126802435E
:105540004E4B103B1A6006E04C4A103A12688243F8
:105550004A4B103B1A60704739B1484A1C321268F6
:105560000243464B1C331A6006E0444A1C32126860
:105570008243424B1C331A60704739B13F4A203294
:10558000126802433D4B20331A6006E03B4A20324A
:1055900012688243394B20331A60704739B1374A59
:1055A000243212680243354B24331A6006E0334A32
:1055B000243212688243314B24331A60704739B168
:1055C0002E4A2C32126802432C4B2C331A6006E010
:1055D0002A4A2C3212688243284B2C331A607047B7
:1055E00039B1264A303212680243244B30331A60F4
:1055F00006E0224A303212688243204B30331A6070
:105600007047012808D11D493C31096841F0080163
:105610001A4A3C32116007E018493C31096821F010
:105620000801164A3C321160704739B1134A273AD3
:1056300012780243114B273B1A7006E00F4A273AB3
:10564000127882430D4B273B1A7070470B4840304D
:10565000006840F080700949403108607047014699
:105660000020064A283A12680A400AB1012000E0E8
:1056700000207047014926390870704734380240CD
:1056800010B50446FA48844208D101211020FFF7E2
:1056900052FF00211020FFF74EFF57E0F5488442EB
:1056A00009D101214804FFF735FF00214FF40030F4
:1056B000FFF730FF4AE0F048844209D10121880415
:1056C000FFF728FF00214FF48020FFF723FF3DE084
:1056D000EA48844209D10121C804FFF71BFF0021D9
:1056E0004FF40020FFF716FF30E0E548844209D16F
:1056F00001210805FFF70EFF00214FF48010FFF78E
:1057000009FF23E0DF48844208D101212020FFF770
:1057100012FF00212020FFF70EFF17E0DA48844235
:1057200009D101218807FFF7F5FE00214FF08040E5
:10573000FFF7F0FE0AE0D548844207D10121400579
:10574000FFF7E8FE00216005FFF7E4FE10BD2DE93C
:10575000FF4705460E460024A14600BFA046B0897B
:1057600000B100BF2C8A24F44054F08804432C82FA
:10577000AC8941F20C608443B08831890843718957
:1057800008430443AC81AC8A24F44074B0890443D8
:10579000AC826846FFF74FFDB548854202D0B94854
:1057A000854202D1DDF80C9001E0DDF80890A8896F
:1057B00000F4004040B109EBC90000EB091031686A
:1057C0004900B0FBF1F707E009EBC90000EB091055
:1057D00031688900B0FBF1F76420B7FBF0F00401F9
:1057E0002009642101FB1078A88900F4004040B131
:1057F000322000EBC800B0FBF1F000F007000443DA
:1058000008E0322000EB08106421B0FBF1F000F05A
:105810000F0004432C81BDE8FF874FF4165101604F
:1058200000218180C18001810C2141810021818181
:10583000704710B502460020108A20F470600B8873
:105840004C8823438C882343CC88234318431082FD
:1058500010BD0021018041808180C180704721B14D
:10586000828942F40052828104E082894DF6FF73FE
:105870001A4082817047028B02F47F420283028BBE
:105880000A430283704721B1828942F40042828137
:1058900003E08289C2F30E028281704721B1828ABD
:1058A00042F40062828204E0828A4FF2FF731A405F
:1058B00082827047C1F3080282807047014688885F
:1058C000C0F308007047028A4FF6F0731A40028254
:1058D000028A0A430282704721B1828942F00202A1
:1058E000828104E082894FF6FD731A4082817047FD
:1058F00082894FF2FF731A40828182890A43828132
:105900007047028A4FF6DF731A400282028A0A4306
:105910000282704721B1028A42F48042028204E08E
:10592000028A4BF6FF731A4002827047818941F068
:1059300001018181704721B1828A42F0080282828E
:1059400004E0828A4FF6F7731A4082827047028B16
:10595000D2B20283028B42EA01220283704721B154
:10596000828A42F02002828204E0828A4FF6DF734C
:105970001A408282704721B1828A42F010028282EC
:1059800004E0828A4FF6EF731A4082827047828A5F
:105990004FF6FB731A408282828A0A4382827047E2
:1059A00021B1828A42F00202828204E0828A4FF6AA
:1059B000FD731A40828270471AB1838A0B43838237
:1059C00002E0838A8B4383827047F0B5034600244C
:1059D00000260025002040F66A17B94200D100BF1A
:1059E0001846C1F3421401F01F06012707FA06F515
:1059F000012C01D10C3004E0022C01D1103000E068
:105A000014301AB107682F43076002E00768AF43FC
:105A10000760F0BD02460020B1F5007F00D100BF55
:105A200013880B400BB1012000E00020704701F407
:105A30000072B2F5007F00D100BFCA4302807047F8
:105A400070B50246002400230025002040F66A16A7
:105A5000B14200D100BFC1F3421501F01F0301267E
:105A600006FA03F3012D13D19689334017E00000A5
:105A7000001001400044004000480040004C00403D
:105A8000005000400014014000780040007C0040BD
:105A9000022D02D1168A334001E0968A33400C125F
:105AA000012606FA04F41688344013B10CB1012023
:105AB00000E0002070BD10B50022002340F66A14FB
:105AC000A14200D100BF0A1201249440A3B2DC43DA
:105AD000048010BD10B501210802FFF72CFD002144
:105AE0004FF48070FFF727FD10BD30B5024600204F
:105AF00000235068F84C20400D790C6844EA0524D6
:105B0000204350609068F54C2040D1E903542C4369
:105B10008D682C434D7944EA450420439060D06A57
:105B200020F470000C7D641EE4B2234340EA03506D
:105B3000D06230BD00210160017141718160C1609E
:105B400001610121017570470021E54A1168E54AAC
:105B50001140D0E900231A4383681A43C3681A43EB
:105B60001143E14AC2F8041370470021016041600B
:105B70008160C160704721B1826842F00102826099
:105B800003E0826822F00102826070470A46002129
:105B90004168D64B194011434160704741628262AF
:105BA00070470A460021416821F01F0111434160FE
:105BB000704738B1CA49096841F40001CA4AC2F8BD
:105BC000041306E0C649096821F40001C64AC2F878
:105BD0000413704738B1C249096841F48001C24AD0
:105BE000C2F8041306E0BE49096821F48001BE4AE8
:105BF000C2F804137047F0B504460D46002000219A
:105C0000092D11DDE068A5F10A0606EB4607072617
:105C100006FA07F18843A5F10A0606EB460603FAE1
:105C200006F10843E0600CE0206905EB4507072614
:105C300006FA07F1884305EB450603FA06F1084327
:105C40002061072A0FDA606B561E06EB86071F26B7
:105C500006FA07F18843561E06EB860605FA06F19A
:105C60000843606322E00D2A0FDA206BD61F06EB93
:105C700086071F2606FA07F18843D61F06EB86061D
:105C800005FA06F10843206310E0E06AA2F10D0670
:105C900006EB86071F2606FA07F18843A2F10D06D8
:105CA00006EB860605FA06F10843E062F0BD81685E
:105CB00041F0804181607047014600208A6802F00F
:105CC00080420AB1012000E00020704721B18268C3
:105CD00042F48062826003E0826822F48062826023
:105CE000704721B1826842F00202826003E082685C
:105CF00022F002028260704710B50A46002100239C
:105D0000416821F46041531E41EA4331416010BDB6
:105D100021B1426842F40062426003E0426822F42A
:105D20000062426070470146C86C80B270476C48A0
:105D3000001D0068704721B1826842F48072826061
:105D400003E0826822F480728260704721B1826829
:105D500042F40072826003E0826822F40072826082
:105D6000704738B15E49096841F400515E4AC2F893
:105D7000041306E05A49096821F400515A4AC2F84E
:105D800004137047F0B50446154600200022002693
:105D9000092911DDE068A1F10A0707EB470C072785
:105DA00007FA0CF29043A1F10A0707EB470703FA41
:105DB00007F21043E0600CE0206901EB410C07277B
:105DC00007FA0CF2904301EB410703FA07F2104384
:105DD0002061A06BC0F30156EF1C06F1010CA7EB8C
:105DE0000C0707EB870C1F2707FA0CF29043EF1CF8
:105DF00006F1010CA7EB0C0707EB870701FA07F286
:105E00001043A063F0BD10B50A4600210023816B4A
:105E100021F44011531E41EA0351816310BD08B5BE
:105E2000002300930090009B0B440093009B1A609A
:105E300008BD0A460021816821F470211143816068
:105E400070470A460021816821F4401111438160A6
:105E50007047816841F480018160704701460020ED
:105E60008A6802F480020AB1012000E00020704735
:105E700021B1426842F48062426003E0426822F449
:105E800080624260704721B1426842F480524260B1
:105E900003E0426822F480524260704708B502462F
:105EA00000200090009201F12800009B184400900F
:105EB0000098006880B208BD10B50B460021D9B229
:105EC000012404FA01F11AB144680C43446002E071
:105ED00044688C43446010BDFFFEFFFCFDF7FFC02B
:105EE00004230140E030FCFF00200140FFFD3FFFA4
:105EF0000246002013680B400BB1012000E0002097
:105F00007047CA430260704770B502460020002304
:105F100000240B12556801268E4005EA0604156818
:105F20001D4015B10CB1012000E0002070BD002221
:105F30000A12D343036070470E49086070470D4949
:105F4000486070470B49886070474AF6AA200949A3
:105F5000086070474CF6CC4006490860704701461F
:105F60000020044AD2680A400AB1012000E0002063
:105F7000704700000030004070B504460D462946C9
:105F800020466268904770BD2DE9F04104460D46F9
:105F900016461F463B46324629462046D4F800C0E6
:105FA000E047BDE8F0812DE9FC4106460C46154668
:105FB0002B46224669463046FFF7E6FF07461FB1EB
:105FC000BDF80000BDE8FC810020FBE70246002090
:105FD000704700B587B068460BF02CF902208DF8A9
:105FE00000000348019068460BF036F907B000BD89
:105FF000CD5F0008704770477047704770470000DA
:106000000000000000000000000000000000000090
:106010000000000000000000000000000000000080
:1060200057313800000000000000000000000000B0
:106030000001000000020000640000004D617920B2
:10604000313320323032350032303A31323A333463
:106050000000000053544D33324634313252450073
:106060004E4F4E4500000000000000000000000000
:106070004E4F4E45000000000000000000000000F0
:106080003132302E32342E3234322E36333A3830EA
:10609000313500000000000000000000000000009A
:1060A0007777772E67756F7965652E636F6D000062
:1060B00000000000000000000000000000000000E0
:1060C0003133393232323830353836000000000092
:1060D0003133393232323832353836000000000080
:1060E0004E4F4E4500000000000000000000000080
:1060F00000000000000000000000000000000000A0
:10610000000000000000000000000000000000008F
:10611000000000000000000000000000000000007F
:10612000000000000000000000000000000000006F
:10613000000000000000000000000000000000005F
:106140004D6F64656C3A2057313820202C4D4355F3
:106150003A2053544D33324634313252452C486143
:1061600072645665723A312E302C536F66745665E0
:10617000723A312E302E300D0A000000E007000088
:10618000485F302E312E3020535F312E302E3000BC
:1061900010B50446FE48844208D101210846FFF7A5
:1061A000CAF900210120FFF7C6F99DE0B4F1804F44
:1061B00008D101210846FFF7ADF900210120FFF7C2
:1061C000A9F991E0F348844208D101210220FFF7A8
:1061D000A1F900210220FFF79DF985E0EE488442F5
:1061E00008D101210420FFF795F900210420FFF7D1
:1061F00091F979E0E948844208D101210820FFF7AC
:1062000089F900210820FFF785F96DE0E448844210
:1062100008D101211020FFF77DF900211020FFF7A0
:1062200079F961E0DF48844208D101212020FFF79D
:1062300071F900212020FFF76DF955E0DA4884421A
:1062400008D101210220FFF776F900210220FFF793
:1062500072F949E0D548844209D101210804FFF7C9
:106260006AF900214FF48030FFF765F93CE0D0482F
:10627000844209D101214804FFF75DF900214FF460
:106280000030FFF758F92FE0CA48844209D10121B4
:106290008804FFF750F900214FF48020FFF74BF9F5
:1062A00022E0C548844208D101214020FFF732F99D
:1062B00000214020FFF72EF916E0C048844208D1A3
:1062C00001218020FFF726F900218020FFF722F925
:1062D0000AE0BB48844207D101218015FFF71AF973
:1062E0000021A015FFF716F910BD00220288A84B67
:1062F00098420ED0AC4B98420BD0B0F1804F08D0F2
:10630000A44B984205D0A44B984202D0A34B98428C
:1063100004D14FF68F731A404B881A43A04B984212
:1063200007D0A04B984204D04FF6FF431A400B8988
:106330001A4302804B68C3620B880385944B9842D2
:1063400002D0994B984201D18B7A03860123838234
:1063500070474FF0FF314160002101800181418091
:10636000817270470185828270470A460021018848
:106370004FF68F7319401143018070474162704797
:10638000C16270470146486A70470146088D7047F0
:1063900021B1028842F00202028004E002884FF636
:1063A000FD731A400280704721B1028842F0040256
:1063B000028004E002884FF6FB731A4002807047A7
:1063C00021B1028842F08002028004E002884FF688
:1063D0007F731A400280704702884FF6F7731A40A5
:1063E000028002880A430280704702884FF6FF430A
:1063F0001A40028002880A430280704721B1028855
:1064000042F00102028004E002884FF6FE731A4057
:106410000280704770B5002400220023058C4FF6DF
:10642000FE7635400584028C8388048B4FF68F7589
:106430002C40B51E2C400D882C43751E2A408D899A
:106440002A434D882A43524DA84202D0564DA842B5
:1064500013D14FF6F7752A40CD892A434FF6FB75C5
:106460002A408D882A434FF6FF652B404FF6FF5593
:106470002B400D8A2B434D8A2B43838004838D68E8
:106480004563028470BD70B5002400220023058C92
:106490004FF6EF7635400584028C8388048B48F6EE
:1064A000FF752C404FF6FF452C400D884FF6FF76C8
:1064B00006EA05252C434FF6DF752A408D8906EA4A
:1064C00005152A434D8806EA05152A43304DA84292
:1064D00002D0354DA8421DD14FF67F752A40CD8997
:1064E0004FF6FF7606EA05152A434FF6BF752A4098
:1064F0008D8806EA05152A434FF6FF352B404FF2EB
:10650000FF752B400D8A06EA85052B434D8A06EA66
:1065100085052B43838004838D688563028470BD69
:1065200070B5002400220023058C4FF6FF6635402D
:106530000584028C8388848B4FF68F752C404FF630
:10654000FC752C400D882C434FF6FF552A408D8951
:106550004FF6FF7606EA05252A434D8806EA05250B
:106560002A430B4DA84202D00F4DA84238D14FF21A
:10657000FF752A40CD894FF6FF7606EA05252A43A6
:106580004FF6FF352A408D8806EA05252A4319E093
:10659000000001400004004000080040000C0040E2
:1065A0000010004000140040000401400040014081
:1065B000004401400048014000180040001C004019
:1065C000002000404EF6FF752B404DF6FF752B4026
:1065D0000D8A06EA05152B434D8A06EA05152B435D
:1065E000838084838D68C563028470BD70B500228A
:1065F00000230024058C4EF6FF7635400584038C7D
:106600008488828B48F6FF752A404FF6FF452A4062
:106610000D884FF6FF7606EA05252A434DF6FF75ED
:106620002B408D8906EA05352B434D8806EA053552
:106630002B43FE4DA84202D0FD4DA84208D14BF697
:10664000FF752C400D8A4FF6FF7606EA85152C4320
:10665000848082838D680564038470BD002101807D
:106660004180818081608181C18101824182704746
:1066700070B50346002000241846183001258D40CF
:10668000ACB21D8CA5431D8409B108290AD100EBC9
:10669000610005684FF68F76354005600568154343
:1066A00005600FE00D1FC5F34E052844056848F648
:1066B000FF763540056005684FF6FF7606EA02264C
:1066C0003543056070BD4163704781637047C163A6
:1066D0007047016470470A460021018B4FF68F73A3
:1066E00019401143018370470A460021018B48F687
:1066F000FF7319404FF6FF7303EA02231943018326
:1067000070470A460021818B4FF68F731940114361
:10671000818370470A460021818B48F6FF73194038
:106720004FF6FF7303EA02231943818370470A4639
:106730000021018B4FF6F773194011430183704715
:106740000A460021018B4FF2FF7319404FF6FF7389
:1067500003EA02231943018370470A460021818B13
:106760004FF6F77319401143818370470A460021A1
:10677000818B4FF2FF7319404FF6FF7303EA022338
:106780001943818370470A460021018B4FF6FB7342
:1067900019401143018370470A460021018B4FF6CF
:1067A000FF3319404FF6FF7303EA022319430183B5
:1067B00070470A460021818B4FF6FB731940114345
:1067C000818370470A460021818B4FF6FF331940C1
:1067D0004FF6FF7303EA02231943818370470A4689
:1067E0000021018B4FF67F731940114301837047DD
:1067F0000A460021018BC1F30E014FF6FF7303EA35
:1068000002231943018370470A460021818B4FF60A
:106810007F7319401143818370470A460021818BA1
:10682000C1F30E014FF6FF7303EA0223194381837C
:1068300070470A460021018C4FF6FD731940114341
:10684000018470470A460021018C4FF6F773194006
:106850001143018470470A460021018C4FF6DF7313
:1068600019404FF6FF7303EA02131943018470477E
:106870000A460021018C4FF67F7319404FF6FF73D3
:1068800003EA02131943018470470A460021018C70
:106890004FF6FF5319404FF6FF7303EA02231943E3
:1068A000018470470A460021018C4FF2FF731940A2
:1068B0004FF6FF7303EA02231943018470470A4627
:1068C0000021018C4DF6FF7319404FF6FF7303EA68
:1068D000023319430184704730B5002301248C40F2
:1068E000A3B2048C9C430484048C02FA01F5ADB27B
:1068F0002C43048430BD30B5002304248C40A3B263
:10690000048C9C430484048C02FA01F5ADB22C4340
:10691000048430BD828B4FF2FF331A408283828B16
:106920004FF6FF7303EA01231A4382837047F0B5E1
:106930000C461546002100220026078C4EF6FF7CEF
:1069400007EA0C070784818B028C4FF6FF7707EA72
:10695000043640F6FF4739404FF6FF7707EA052730
:1069600039434FF6FF7707EA0337394345F6FF7798
:106970003A4046F480573A4381830284F0BD828BCB
:106980004FF6F3731A408283828B0A4382837047E7
:10699000F0B50C461546002100220026078C4FF664
:1069A000FF6C07EA0C070784818B028C4FF6FF7798
:1069B00007EA04264FF60C7739404FF6FF7707EACF
:1069C00003172F4339434FF2FF573A4046F480777D
:1069D0003A4381830284F0BD028B4FF2FF331A40A9
:1069E0000283028B4FF6FF7303EA01231A430283EB
:1069F0007047F0B50C461546002100220026078C92
:106A00004FF6EF7C07EA0C070784018B028C4FF6E8
:106A1000FF7707EA041640F6FF4739404FF6FF7745
:106A200007EA033739434FF6FF7703E000000140E0
:106A30000004014007EA052739434FF65F773A40E3
:106A400046F010073A4301830284F0BD028B4FF6F3
:106A5000F3731A400283028B0A4302837047F0B536
:106A60000C46154600210022068C4FF6FE773E406C
:106A70000684018B028C4FF60C7631407E1C06EAB0
:106A800003162E4331434FF6F576324044F00106AB
:106A9000324301830284F0BD70B505460C46208860
:106AA00050B92389A28861882846FFF7D8FFE1887A
:106AB0002846FFF7CBFF25E0208804280AD1238948
:106AC000A28861882846FFF794FFE1882846FFF7EF
:106AD00083FF17E0208808280AD12389A2886188CB
:106AE0002846FFF755FFE1882846FFF748FF09E0F1
:106AF0002389A28861882846FFF719FFE188284684
:106B0000FFF708FF70BD00210180418001218180D5
:106B10000021C180018170472DE9F04105460C46F6
:106B200000260127608808B9022600E00026A08818
:106B3000012801D1022700E001272088A0B923897C
:106B4000A28861882846FFF78AFFE1882846FFF778
:106B50007DFF23893A4631462846FFF74AFFE18800
:106B60002846FFF739FF13E02389A2886188284669
:106B7000FFF73FFFE1882846FFF72EFF23893A46BB
:106B800031462846FFF76BFFE1882846FFF75EFF96
:106B9000BDE8F0810146486B70470146886B70473D
:106BA0000146C86B70470146086C70470A884B88DD
:106BB0001A438B881A43CB881A430B891A434B8993
:106BC0001A438B891A43A0F84420704700210180A2
:106BD00041808180C180018141818181704731B1D3
:106BE000B0F8442042F40042A0F8442005E0B0F898
:106BF0004420C2F30E02A0F84420704721B18288DD
:106C000042F00402828004E082884FF6FB731A404F
:106C10008280704721B1828842F00102828004E0C4
:106C200082884FF6FE731A40828070471AB18389BA
:106C30000B43838102E083898B4383817047818288
:106C4000704702460020138A0B400BB1012000E080
:106C500000207047CA430282704730B502460020C8
:106C600000230024158A05EA0103958905EA010439
:106C700013B10CB1012000E0002030BDCA430282F4
:106C8000704741EA0203A0F8483070471AB183897F
:106C90000B43838102E083898B438381704721B159
:106CA000828842F00802828004E082884FF6F773FF
:106CB0001A408280704701894FF6F87211400181B5
:106CC00070470A46002101894FF68F73194011431E
:106CD0000181704730B504460D4629462046FFF72E
:106CE000F0FF208940F00700208130BD2DE9F04100
:106CF00004460D4616461F46602D06D13B4601222E
:106D000031462046FFF775FE05E03B46012231463D
:106D10002046FFF7A4FE29462046FFF7D2FF208930
:106D200040F007002081BDE8F08130B50C4600211D
:106D30000189C9B24FF6FF7505EA032515432543BE
:106D40002943018130BD2DE9F04105460E46174625
:106D50009846002443463A4631462846FFF7E5FF69
:106D60002C894FF6F870044044F007044FF68F70FA
:106D7000044044F070042C81BDE8F081F0B5044675
:106D80000D4616461F463B46324629462046FFF72B
:106D9000CCFF208940F480402081F0BD82884FF6EE
:106DA0008F731A40828082880A43828070470289EA
:106DB0004FF6F8731A40028102890A430281704734
:106DC00002894FF67F731A40028102890A430281C9
:106DD0007047F0B50C4615461E46002100220023E0
:106DE0000189028B038C4FF6F877394021434FF627
:106DF000FC473A4040F201173A434FF6DD773B40FB
:106E00004FF6FF7707EA06172F433B4301810283C2
:106E10000384F0BD21B1828842F08002828004E0C8
:106E200082884FF67F731A4082807047A0F8501016
:106E30007047000010B50446FB48844208D1012188
:106E40008014FEF778FB0021A014FEF774FB3CE0F1
:106E5000F648844208D101210014FEF75BFB0021B3
:106E60002014FEF757FB30E0F148844208D101219D
:106E7000C013FEF74FFB0021E013FEF74BFB24E0AD
:106E8000EC48844208D101214014FEF754FB002154
:106E90006014FEF750FB18E0E748844209D1012155
:106EA0000805FEF748FB00214FF48010FEF743FB76
:106EB0000BE0E248844208D101214805FEF73BFB84
:106EC00000214FF40010FEF736FB10BD10B5002274
:106ED000028802F441520B884C8823438C88234358
:106EE000CC8823430C8923434C8923438C89234337
:106EF000CC8923431A430280838B4FF2FF742340D3
:106F000083830B8A038210BD2DE9F04F00250223F5
:106F100000244FF0010900220026002794469046E5
:106F2000B0F81CA04FF2400B0AEA0B0AA0F81CA014
:106F30004FF0020AA0F820A0858BD1F808A0BAF182
:106F4000020F01D100BF82E0B1F804A0BAF1000F36
:106F500002D14FF0010901E04FF00209DFF8E0A291
:106F6000DAF800A00AF4000ABAF1000F09D0DFF83D
:106F7000D0A2DAF800A02AF4000ADFF8C4B2CBF8F5
:106F800000A0DFF8BCA20AF17C0ADAF800A0CAF37C
:106F9000881CDFF8ACA20AF17C0ADAF800A0CAF378
:106FA0000278DFF89CA2AAF1040ADAF800A00AF03D
:106FB0003F07DFF88CA2AAF1040ADAF800A00AF46D
:106FC000800ABAF5800F08D1DFF878A2BAFBF7FA89
:106FD0000AFB0CFABAFBF8F607E0DFF86CA2BAFB82
:106FE000F7FA0AFB0CFABAFBF8F6B1F806A0BAF504
:106FF000007F0ED14FEA162A0AEB8A0A4FEA4A0AA4
:10700000D1F808B0BAFBFBFA0AF1050A1FFA8AF2B6
:107010000FE04FEA491AB6FBFAFA0AEB8A0A4FEA7E
:107020004A0AD1F808B0BAFBFBFA0AF1050A1FFABE
:107030008AF24FF00A0AB2FBFAF202F00104A2EB64
:10704000040ACAF34F034FF6FF7A0AEA0424022B1C
:1070500001DBFF2B01DD02230024B1F806A04AEA80
:10706000040A4AEA030AA0F820A0B1F804A0B1F883
:107070000CB04AEA0B0AB1F802B04AEA0B0AB1F8BE
:1070800000B04AEA0B0A4AF4006A4AEA0505858319
:10709000BDE8F08F0021018041808180C1800181A5
:1070A00041818181C18107210182704700210180D6
:1070B00041808180C18002218160002181817047EF
:1070C00021B1028842F04002028004E002884FF6BB
:1070D000BF731A400280704721B1828B42F48062F4
:1070E000828304E0828B4FF6FF331A40828370471D
:1070F00002884FF2FF731A40028002880A4302801E
:107100007047B1F5804F04D1028842F4804202807A
:1071100004E002884BF6FF731A40028070474FF676
:10712000FF62914204D0028842F48072028004E03F
:1071300002884FF6FF631A400280704721B18288AF
:1071400042F00402828004E082884FF6FB731A400A
:107150008280704721B1828842F01002828004E070
:1071600082884FF6EF731A408280704730B5002254
:107170000023848B4FF240052C4084830224048436
:10718000828B0C88B4F5007F01D00C8814B94FF4C1
:10719000807308E00C88B4F5407F03D00C88B4F508
:1071A000807F00D100238C888D892C434D882C430F
:1071B0001C4344F400642243828330BD0146888925
:1071C00070478181704721B1028842F400520280E9
:1071D00004E002884DF6FF731A4002807047018870
:1071E00041F480510180704702460020012901D0FE
:1071F000108B00E0908A70470146088A70471AB1E8
:1072000083880B43838002E083888B4383807047AD
:1072100030B5002400230C110125A540ABB2AAB162
:1072200085881D43858014E000300140003800400F
:10723000003C004000340140005001400054014037
:107240000838024000127A000024F40085889D432B
:10725000858030BD0246002013890B400BB1012010
:1072600000E000207047CA4302817047F0B5024633
:10727000002000240023002501F00F070126BE4056
:10728000B4B20B1101269E40B3B2968806EA0305FC
:107290001689264016B10DB1012000E00020F0BD96
:1072A00010B5002201F00F040123A3409AB2D3438A
:1072B000038110BD10B5044614B909F0DDFE044683
:1072C0000CB9002010BD206BFCE770B504462046C9
:1072D00001F00CFF05462C63204601F033FF70BD22
:1072E00010B5044614B909F0C7FE04460CB90020D5
:1072F00010BD606BFCE710B5044614B909F0BCFE84
:1073000004460CB9002010BDA06BFCE770B5054623
:107310000E46304601F0D4FE00B170BD304601F09B
:10732000E5FE0446AC4200D1F7E70123324605F101
:10733000240104F124000AF03FFE00BFEDE710B580
:10734000044614B909F098FE04460CB9002010BD9B
:10735000206AFCE770B5044614B909F08DFE0446B6
:107360000CB9002070BD24B1D4F8600109F0F2FF1F
:10737000F8E74FF0FF36002009F00EFF054610E059
:10738000D5F8600109F0E6FFB04201D9304603E0CC
:10739000D5F8600109F0DEFF0646284609F0FCFE3C
:1073A0000546002DECD13046DCE710B5044614B993
:1073B00009F062FE044604B910BD09F0C0FFC4F82C
:1073C000600100BFF8E7000007B581B0BDF8080014
:1073D000C00AC2F1FF014843BDF80410C90A01FB0D
:1073E0000200010ABDF8000061F3CF200090BDF853
:1073F0000800C0F34510C2F1FF014843BDF8041076
:10740000C1F3451101FB0200010ABDF8000061F360
:107410004A100090BDF8080000F01F00C2F1FF0103
:107420004843BDF8041001F01F0101FB0200010AEE
:10743000BDF8000061F304000090BDF8001008469C
:1074400004B000BD10B55C21FA480AF084FC10BD00
:1074500030B587B005460C46FF21E173F648006859
:107460000690A01CBDF818106181207A08B9A08987
:1074700008B10321A181F048001D006805906088D3
:10748000B22200900599FFF79FFF0190BDF804001C
:107490006080E948083000680490A088B22200901B
:1074A0000499FFF791FF0190A01CBDF80410A18082
:1074B000E1480C3000680390208A992200900399DB
:1074C000FFF782FF0190A01CBDF804102182DA486A
:1074D000103000680290B2220299206AFFF774FF10
:1074E0000190BDF8040020843220005D10280ADAE3
:1074F000D148143000680190BDF804002086662150
:107500003220015500BF07B030BD30B587B0054609
:107510000C46FF21E173C848183800680690A01C8B
:10752000BDF818106181207A08B9A08908B103213B
:10753000A181C1481438006805906088B22200908B
:107540000599FFF741FF0190BDF804006080BA483B
:10755000103800680490A088B22200900499FFF7C8
:1075600033FF0190A01CBDF80410A180B2480C3874
:1075700000680390208A992200900399FFF724FF66
:107580000190A01CBDF804102182AB4808380068A7
:107590000290B2220299206AFFF716FF0190BDF80F
:1075A000040020843220005D10280ADAA248001F5F
:1075B00000680190BDF80400208666213220015544
:1075C00000BF07B030BD9D4A02619D4A426169B16A
:1075D000D1F8A82112B1D1F8A82102614FF4D672D6
:1075E00052581AB14FF4D67252584261704770B572
:1075F00090480AF0E9FB04460CB900BFFEE70CB95D
:10760000002070BD042120460AF0A5FB002039347B
:1076100044F82D0CE07F20F00100E077002044F8D2
:10762000210CE07F20F00400001DE077E07F20F0D7
:107630000200E077E07F20F008000830E077E07F8C
:1076400020F010001030E077393C0DF073FF054654
:1076500029462046FFF7B7FF2046D2E770B504461B
:10766000E06848B1E168086800221021C3699847C2
:10767000E168086801F066FD20460AF0CFFB054688
:1076800007E000202968C862294620460AF027FC46
:107690000546002DF5D120460AF076FC21466548C6
:1076A0000AF02DFC20460AF00CFE70BD70B50546B0
:1076B0002C46002609E094F83000C0F3401000B1D9
:1076C0002646204601F0FCFC0446002CF3D116B1FE
:1076D000304602F067FA70BD2DE9F84F044688463F
:1076E000914694F8580000F0010008B1BDE8F88F09
:1076F000E56800264FF0010A4FF0010B00BF8DB97D
:1077000094F85800C0F3001000B956B9BBF1000F4F
:1077100000D1EBE72046C04705464FF0000AD346AC
:1077200000E0E3E716B92E4606B9DFE7BAF1000F2D
:1077300006D029462046C8470546B54200D1D5E7C0
:107740004FF0010A05B9DAE7286801F0BCFC00B97E
:1077500000E0D4E700BFE068A84200D1C6E7E068D7
:10776000A8B1E168086800221021C3699847E16860
:10777000002208680D2102F0B1F80090009801285D
:1077800000D0B3E7E168086801F0DCFC00BFE56009
:10779000E168086800220F21C3699847E168002268
:1077A00008680C2102F09AF80746012F00D09DE7E7
:1077B000E1680868FFF77AFFE168086801F0C2FC39
:1077C000A06910B12046A169884700BF8EE710B5B7
:1077D00004461C4A1C492046FFF77EFF10BD10B529
:1077E00004461A4A1A492046FFF776FF10BD70B5C5
:1077F000044614F8580FC0F30015207820F010004C
:107800001030207014F85809C0F3C00018B9204691
:10781000FFF7E5FF07E094F85800C0F3C00010B18F
:107820002046FFF7D4FF94F8580065F3041084F85D
:10783000580070BDC02E0020300802080B750008EB
:1078400051740008091E0108F51E0108DF1E010819
:107850001D1E01082DE9F04107460C460FB9BDE891
:10786000F08138460AF0DAFA064608E03068A042AD
:1078700000D1F4E7314638460AF031FB0646002EC7
:10788000F4D1E06A30B1204603F011F810B1E06A9B
:10789000FFF7ADFFE76238460AF0FEFA05460DB97C
:1078A00000BFFEE705B9DAE72C6038460AF0B6FA01
:1078B000A84202D13846FFF79AFF00BFCFE770B564
:1078C0000546EC6A04B970BDE06800B9FBE7E06802
:1078D0000068A84215D120460AF0A0FAE168884263
:1078E0000CD120460AF006FBE168884206D1E16827
:1078F000086800221021C369984702E02046FFF77C
:1079000076FFE0680068A84201D10020E0602046D0
:107910000AF084FA064611E03068A84209D13146DF
:1079200020460AF0ECFA30460AF0CBFC0020E86270
:1079300006E0314620460AF0D2FA0646002EEBD188
:1079400000BF00BFBFE770B50446E06858B1E1680A
:10795000086800221021C3699847E168086801F0AF
:10796000F1FB0020E06020460AF058FA054607E0E7
:1079700000202968C862294620460AF0B0FA054668
:10798000002DF5D120460AF0FFFA70BD014609B975
:1079900000207047C86808B90020FAE7C868006886
:1079A000F7E72DE9F04104460E46374694F85800B3
:1079B000C0F34000B84201D1BDE8F08194F858000E
:1079C00067F3410084F858002046FFF7DFFF0546C3
:1079D00085B100220F212846EB699847E168002213
:1079E00008680C2101F07AFF8046B8F1010F00D041
:1079F000E2E700BF284601F0A5FB00BFDCE72DE968
:107A0000F04106460EB9BDE8F081F46A04B9FAE720
:107A100094F8580000F0010000B1F4E7002120467E
:107A2000FFF7BFFF20460AF0F9F9054640E0286855
:107A3000B04238D1E068A0B1E168086800221021A6
:107A4000C3699847E168002208680D2101F046FFEC
:107A50000746012F00D0D6E7E168086801F072FB05
:107A600000BFE560E068E8B1E168086800220F2126
:107A7000C3699847A06910B12046A1698847E168A9
:107A8000002208680C2101F029FF0746012F00D0D1
:107A9000B9E7E168086801F055FBE1680868FFF79D
:107AA00005FE00BF06E0294620460AF018FA054602
:107AB000002DBCD100BF00BFA5E731B990F8582018
:107AC00022F0010280F8582006E090F8582022F0B9
:107AD0000102521C80F85820704773B506463046A4
:107AE000FFF754FF05460DB901207CBD01AA112105
:107AF0002846EB6998470446012C01D02046F4E75C
:107B000001AA0B21284601F0E9FE0446012C01D010
:107B10002046EAE72046E8E770B504460D462561B1
:107B2000E06818B1E168086801F00CFB70BD70B541
:107B300004460D466561E06818B1E168086801F027
:107B400001FB70BD8161704790F8582061F382029B
:107B500080F85820704790F8582061F3C30280F8ED
:107B60005820704790F8582061F3041280F858208C
:107B7000704770B504460D46294604F11C0003F019
:107B8000F9FA94F85800C0F3400038B1606960B168
:107B900004F11C0120466269904706E0206920B18B
:107BA00004F11C0120462269904704F11C0070BDBD
:107BB000014609B9002070470869FCE7014609B988
:107BC000002070474869FCE7014609B9002070476A
:107BD0008869FCE7014609B90020704791F8580010
:107BE000C0F34000F9E7014609B90020704791F859
:107BF0005800C0F38000F9E7014609B9002070473A
:107C000091F85800C0F30010F9E770B505460DF083
:107C100091FC064625B131462846FFF7D4FC70BDDD
:107C200008480AF0FBF8044608E031462046FFF712
:107C3000CAFC214603480AF052F90446002CF4D14C
:107C400000BFECE7C02E002070B504463CB194F8AC
:107C50004C0020F00200801C84F84C0012E0002050
:107C600009F035FB05460AE095F84C0020F00200CB
:107C7000801C85F84C00284609F029FB0546002D9C
:107C8000F2D100BF70BD10B50020FFF7DDFF10BDC1
:107C900090F84C10C1F3400129B300224263826383
:107CA000C26390F8401021F0010280F8402090F863
:107CB000401021F0020280F8402090F84C1021F092
:107CC000010280F84C200022426482648285C285D1
:107CD0000286428690F84C1021F0020280F84C2077
:107CE0000021FE4A11607047014691F83000C0F350
:107CF000400010B10020F94A106091F83000C0F344
:107D0000400070472DE9FF41044694F82400C0F379
:107D1000400008B9BDE8FF81E56903E0284601F0AD
:107D2000CFF90546284602F075FD08B1002DF5D1C2
:107D300005B9EFE7284602F067FDD8B994F82400AA
:107D400020F0020184F82410E548EB690E21026856
:107D50002846984700220921284601F0BFFD204609
:107D6000FFF7C2FF00B1D5E700220921284601F044
:107D7000B5FDCFE7284602F041FD0646A08AD84966
:107D80000968497DC1F1640110FB01F0642190FB99
:107D9000F1F001B2A182E08AD1490968497DC1F1BF
:107DA000640110FB01F0642190FBF1F001B2E1826B
:107DB000A08A10B9E08A00285DD002A9284601F007
:107DC00050FA284601F0B3FAA18A08440FFA80F865
:107DD000284601F0A0FA0146E08A084407B2032EC3
:107DE00005D13A464146284601F044FA0EE006F035
:107DF000010020B14146284601F012FF06E006F0DE
:107E0000020018B13946284601F017FF6946284696
:107E100001F027FABDF90800BDF90010884201D031
:107E2000A08A38BBBDF90A00BDF90210884201D012
:107E3000E08AF8B994F8240020F0020184F82410B4
:107E40000021A181E181A182E182A548EB690E2197
:107E50000268284698472046FFF746FF00B159E7D9
:107E600000220921284601F039FD2046FFF73CFF9A
:107E700000B14FE71AE094F8240020F0020184F8E2
:107E800024109748EB690E2102682846984720463F
:107E9000FFF72AFF00B13DE700220921284601F043
:107EA0001DFD2046FFF720FF00B133E700BF31E79B
:107EB0002DE9F041044694F83000C0F3C00058B1F9
:107EC0000021A161E1610020A062E06294F830002D
:107ED00020F0080084F830008049A0690860084656
:107EE0000068002874D010217C48006801F0F4FA82
:107EF00000283AD079480068C36979480A210268A5
:107F00007648006898472046FFF7EEFE08B1BDE8C6
:107F1000F08194F82400C0F34000D0B994F8300008
:107F200000F0010050B9002203216C48006801F004
:107F3000D5FC2046FFF7D8FE00B1E8E70022062175
:107F40006648006801F0CAFC2046FFF7CDFE00B18C
:107F5000DDE7002207216148006801F0BFFC2046F0
:107F6000FFF7C2FE00283FD0D1E75C480068C36934
:107F70005B480A2102685948006898472046FFF785
:107F8000B3FE00B1C3E794F8300000F0010078B907
:107F900094F82400C0F3400050B9002203214F4858
:107FA000006801F09BFC2046FFF79EFE00B1AEE7A3
:107FB00094F82400C0F3400058B900220621474835
:107FC000006801F08BFC2046FFF78EFE08B19EE7AB
:107FD0008EE0002207214148006801F07FFC204626
:107FE000FFF782FE00B192E72046FFF77DFE00B169
:107FF0008DE74FF000083948006801F0B8F90546F0
:1080000020213648006801F067FA10BB3348076842
:1080100010E0384601F054F8074607B90CE020217B
:10802000384601F059FA08B1002705E0384601F05A
:108030009EF90546002DECD000BF4DB147B1284652
:10804000FFF7D1FD20B14FF001083846FFF7D7FC0C
:1080500000BF2249206A0968884219D0B8F1000F90
:1080600016D100220D21206A01F038FC2046FFF7CE
:108070003BFE00B14BE700220C21A06901F02EFC71
:108080002046FFF731FE00B141E714480168216244
:108090002046FFF729FE00B139E71048066803E0E3
:1080A000304601F00DF80646304602F0B3FB08B149
:1080B000002EF5D1B6B1304602F0A6FB90B194F88F
:1080C0002400C0F3400068B100220A21304601F0CC
:1080D00005FC2046FFF708FE20B118E7EC00002061
:1080E000E80000200021A1610020A062E06200BF42
:1080F000E06960B194F83000C0F3400038B9204620
:10810000FFF700FE2046FFF7EFFD00B1FFE600BFDE
:10811000FDE62DE9F04F87B00446A569002703E08E
:10812000284600F0CDFF0546284602F073FB08B153
:10813000002DF5D115B907B0BDE8F08F284602F043
:1081400057FB00B9F7E7284602F058FB0646218A9C
:10815000A089084401B22182618AE089084401B201
:10816000618294F8240000F0010058BB06F0010081
:1081700070B1B4F91000002802DDB4F9100002E07B
:10818000B4F910004042F8490968097D884211DAC3
:1081900006F00200B0B1B4F91200002802DDB4F913
:1081A000120002E0B4F912004042EF490968097D6B
:1081B000884207DB94F8240020F00100401C84F87A
:1081C0002400012794F8240000F0010000287DD04D
:1081D000A08910B9E0890028F9D0E3490968C86886
:1081E00008F0E9FF8246B5F910B0B5F91200069023
:1081F000284600F065FF039001F034FD0590284605
:1082000000F05EFF039001F025FD0490284601F088
:108210008EF88046284601F07EF88146032E12D162
:108220003FB1208A40440FFA80F8608A48440FFA30
:1082300080F9E089484402B2A089404401B228464E
:1082400001F018F81CE006F0010058B11FB1208AB7
:1082500040440FFA80F8A089404401B2284601F05A
:10826000DFFC0DE006F0020050B11FB1608A484407
:108270000FFA80F9E089484401B2284601F0DDFC9C
:10828000B5F9100058452DD1B5F912100698814264
:1082900028D1284600F014FF019001F0E3FC039080
:1082A000284600F00DFF019001F0D4FC02900599E2
:1082B0000398884215D104990298884211D1AA499D
:1082C0000968C86808F077FF019000E028E0019A8B
:1082D000A2EB0A0291B2A44A1268D06808F071FFBA
:1082E00000BF1CE094F8240020F00200801C84F8F9
:1082F0002400A7B19C48EB690D21026828469847E5
:108300002046FFF7F1FC00B115E7002208212846BE
:1083100001F0E4FA2046FFF7E7FC00B10BE700BFED
:1083200000BF08E72DE9F04107460C460025391D3E
:1083300004F1100009F061FB00282BD0201D09F08A
:108340006DFD80460BE041463846FFF7EBFF0546E2
:1083500005B107E04146201D09F0C1FD8046B8F196
:10836000000FF0D100BFA5B9204602F035FA80B168
:10837000264608E0304600F0A6FE00B105E0304693
:1083800000F09EFE0646002EF4D100BF06B9254639
:1083900000BF00BF2846BDE8F0812DE9F04104464A
:1083A0007249A069086094F83000C0F3C00008B1B9
:1083B000BDE8F0816C480068C66800276B4800681B
:1083C00028BB3046FEF797FF054629462046FFF7B3
:1083D000A9FF664908600846006848B93046FEF7BC
:1083E0007FFF054629462046FFF79CFF5F4908604E
:1083F0005E48006848B93046FEF75CFF05462946EE
:108400002046FFF78FFF5949086001272FE094F8B5
:108410002400C0F3400050BB10215448006801F014
:108420005BF820BB3046FEF766FF0546294620462E
:10843000FFF778FF4D4908600846006848B93046A4
:10844000FEF74EFF054629462046FFF76BFF4749DA
:1084500008604648006848B93046FEF72BFF0546DD
:1084600029462046FFF75EFF4049086001273FB1DB
:10847000E06928B10021A182E1822046FFF742FC99
:108480003A49A0690968884273D0A1882181E188AE
:108490006181A069B0B1A5693348EB69092102681F
:1084A000284698472046FFF71FFC00B180E70022CE
:1084B0000221284601F012FA2046FFF715FC00B110
:1084C00076E700BF29480168A1610168E1610068A1
:1084D00000284ED008F033FFA06294F8300020F05E
:1084E000010084F8300094F8240020F0010184F8A1
:1084F000241094F8240020F0020184F824100021B4
:1085000021826182A181E18118480568884609E0DD
:1085100095F83000C0F3401000B1A846284600F09E
:10852000CFFD0546002DF3D1B8F1000F02D0404633
:1085300001F038FB0D480068C3690B480721026849
:108540000A48006898472046FFF7CEFB00B12FE7A6
:10855000002211460548006801F0C0F92046FFF7E7
:10856000C3FB28B124E704E0E8000020EC00002071
:1085700000BFA1882089081A01B2A181E188608921
:10858000081A01B2E181B4F9140000EB8000C010B8
:10859000A082B4F9160000EB8000C110E182B4F9AA
:1085A0001400002804DAA08A401C01B2A18207E06E
:1085B000B4F91400002803DDA08A401E01B2A18294
:1085C000B4F91600002804DAE08A401C01B2E18206
:1085D00007E0B4F91600002803DDE08A401E01B26E
:1085E000E182A18AB4F90C00800001EBE00001B245
:1085F000A182E18AB4F90E00800001EBE00001B233
:10860000E182F9480068002875D0F7480068C3691E
:10861000F64808210268F448006898472046FFF7AA
:1086200063FB00B1C4E600220121EF48006801F0BD
:1086300055F92046FFF758FB00B1B9E62046FFF791
:1086400068FD2046FFF750FB00B1B1E694F8240026
:10865000C0F3400078BB94F8300000F0010050BB3C
:10866000A06A08F077FEE1490968C98A884222D9E0
:10867000DD480068C369DD480B210268DA480068FC
:1086800098472046FFF730FB00B191E60022042115
:10869000D548006801F022F92046FFF725FB00B11C
:1086A00086E694F8300020F00100401C84F8300089
:1086B00008F045FEE06294F82400C0F34000D0B911
:1086C00094F8300000F00100A8B1E06A08F042FE22
:1086D000C6490968098B88421CD9C3480068C36928
:1086E000C2480C210268C048006898472046FFF73E
:1086F000FBFA08B15CE60DE000220521BA480068EB
:1087000001F0ECF82046FFF7EFFA00B150E608F070
:1087100016FEE06200BF4BE670B504460D46A06D44
:10872000A96830F821102184A06DA96800EB8100B0
:1087300041886184B4F92410B4F9200081420DD13C
:10874000B4F92610B4F92200814207D1A87B012890
:1087500004D104F11C00FFF720FE03E004F11C002B
:10876000FFF7A6FB218CA184618CE18470BD2DE90B
:10877000F84304460D46A87B012806D194F84C0026
:10878000C0F3C00008B1BDE8F88394F84C00C0F312
:10879000C00080B194F84C0020F0080184F84C101F
:1087A0000021616494F84C0020F0010184F84C1021
:1087B00000212020015594F82080A97B202001551C
:1087C00069686162676D07B9DDE73846FFF7DEF873
:1087D000854908600846006800B9D4E7A87B0028EE
:1087E00043D13846FFF7F6F900B3B5F90C0000287D
:1087F0000CDA002604E014213846FFF76EF9761CE7
:10880000B5F90C004042B042F5DC0EE0B5F90C00C1
:1088100000280ADD002604E013213846FFF75DF941
:10882000761CB5F90C00B042F6DC1EE0B5F90C0080
:1088300000280BDA002603E03846FEF7C8FF761C56
:10884000B5F90C004042B042F6DC0DE0B5F90C0081
:10885000002809DD002603E03846FEF7C0FF761C3D
:10886000B5F90C00B042F7DC00BF3846FFF78EF8D0
:108870005D4908600846006800B984E7A87B0128C4
:1088800031D1B8F1000F2ED1002000905648006879
:108890006A461221C36954480068984708F04FFDA2
:1088A00060643846FFF796F910B99DF80000C8B922
:1088B0004D48006800220721C3694B48006898476B
:1088C00004F11C00FFF710FA00B15CE7002211462A
:1088D0004548006801F002F804F11C00FFF704FAB3
:1088E00000B150E7FDE0A87B01284BD1B8F1010FA2
:1088F00048D194F84C0000F001000028F2D1606CDF
:1089000008F028FDE18A8842ECD900200090364822
:1089100000686A461221C3693348006898479DF889
:10892000000068B1384609F0C7FB18BB3846FFF7AE
:1089300051F980F0010631463846FFF732F819E068
:108940002948006800220B21C3692748006898471E
:1089500004F11C00FFF7C8F900B114E7002204215C
:108960002148006800F0BAFF04F11C00FFF7BCF9D1
:1089700000B108E794F84C0020F00100401C84F896
:108980004C00AEE0A87B0028ACD1B8F1010FA9D112
:108990000090154800686A461221C36912480068B1
:1089A00098479DF80000F0B90F48006800220A219E
:1089B000C3690D480068984704F11C00FFF794F95B
:1089C00000B1E0E694F84C0000F0010028B9002264
:1089D00003210548006800F081FF04F11C00FFF747
:1089E00083F928B1CFE61BE0EC000020E80000206E
:1089F00000220621FB48006800F070FF04F11C0013
:108A0000FFF772F900B1BEE600220721F5480068C1
:108A100000F064FF04F11C00FFF766F9A0B3B2E6B2
:108A200097F85800C0F3400078B394F84C0000F079
:108A3000010018B1384609F03FFB28B3E948006847
:108A400000220A21C369E7480068984704F11C0026
:108A5000FFF74AF900B196E600220321E1480068D9
:108A600000F03CFF04F11C00FFF73EF900B18AE67C
:108A700000220621DB48006800F030FF04F11C00F2
:108A8000FFF732F910B17EE622E010E00022072164
:108A9000D448006800F022FF04F11C00FFF724F91D
:108AA00000B170E60A213846FFF717F810E09DF88C
:108AB000000068B197F85800C0F3400040B994F83E
:108AC0004C0000F0010018B901213846FEF769FF9B
:108AD0000021616494F84C0020F0010184F84C10EE
:108AE00000BF0020BF49086000BF4CE62DE9F041FF
:108AF00004460D46A87B012806D194F84C00C0F32B
:108B0000C00008B1BDE8F08194F84C00C0F3C0008B
:108B100080B194F84C0020F0080184F84C1000213A
:108B2000616494F84C0020F0010184F84C1000219D
:108B300020200155676D07B9E4E73846FEF726FFA8
:108B4000A84908600846006800B9DBE7D4F824802B
:108B5000696861622020065DA97B0155A87B012818
:108B600061D1002E5FD108F0EAFB606468680A28D2
:108B70001ED10A213846FEF7B0FF9A48006800224D
:108B80000721C36997480068984704F11C00FFF764
:108B9000ABF800B1B6E7002211469248006800F039
:108BA0009DFE04F11C00FFF79FF800283AD0A9E7CA
:108BB00068681B2810D11B213846FEF78EFF002263
:108BC00012218848006800F089FE04F11C00FFF7BC
:108BD0008BF80028EAD095E7686809280DD10021B4
:108BE0003846FEF7DEFE3846FEF7F9FD04F11C00BC
:108BF000FFF77AF80028D9D084E768680B280DD1F0
:108C000000213846FEF7CDFE3846FEF7E0FD04F1C0
:108C10001C00FFF769F80028C8D073E73846696878
:108C2000FEF75BFFD9E0A87B012872D1012EFCD1B1
:108C300094F84C0000F0010068BB606C08F08AFBFF
:108C4000E18A884227D994F84C0020F00100401CAA
:108C500084F84C0068680A28E4D108F070FBA0642E
:108C60006048006800220B21C3695E48006898478D
:108C700004F11C00FFF738F800B143E7002204219B
:108C80005848006800F02AFE04F11C00FFF72CF899
:108C90000028C7D036E794F84C0000F00100002807
:108CA000C0D0A06C08F056FB218B8842BAD908F0DE
:108CB00046FBA06468680A281AD14A480068002266
:108CC0000C21C36947480068984704F11C00FFF76E
:108CD0000BF800B116E7002205214248006800F0B9
:108CE000FDFD04F11C00FEF7FFFF002875D009E729
:108CF000686809280ED100213846FEF752FE384632
:108D0000FEF76DFD04F11C00FEF7EEFF002864D0B5
:108D1000F8E619E068680B280CD100213846FEF708
:108D200040FE3846FEF753FD04F11C00FEF7DCFF61
:108D300090B3E7E638466968FEF7CFFE04F11C0001
:108D4000FEF7D2FF40B3DDE6A87B28BB012E44D15D
:108D5000C5F8048068680A2837D1224800680022D4
:108D60000A21C3691F480068984704F11C00FEF7F8
:108D7000BBFF00B1C6E694F84C0000F0010060B9FA
:108D8000002203211748006800F0A8FD04F11C0030
:108D9000FEF7AAFF08B1B5E61FE000220621114840
:108DA000006800F09BFD04F11C00FEF79DFF00B180
:108DB000A8E6002207210B48006800F08FFD04F1AF
:108DC0001C00FEF791FF00B19CE60021616494F85D
:108DD0004C0020F0010184F84C100020014908608B
:108DE00000BF8FE6EC00002070B504460D46206DF4
:108DF00090B1B4F92400B5F90010884205D1B4F956
:108E00002600B5F90210884206D0B5F90220B5F95E
:108E10000010206D00F02EFA298821846988618471
:108E2000207F012804D104F11C00FFF7B6FA03E00B
:108E300004F11C00FFF73CF8218CA184618CE184D3
:108E400070BD7FB504468949E0680860084600683F
:108E5000C06800B97FBD85480068FEF719FF8348E8
:108E6000006890F84C00C0F3800000B1F2E700BF4A
:108E700069467E48006808F036FA05467B48006877
:108E8000FEF706FF00207A4908609DF80E0077493A
:108E90000968087775480068007F012807D108F045
:108EA0004EFA72490968C968C1F860010EE06F485E
:108EB00000680078042809D1BDF80C0030B108F032
:108EC0003EFA6A490968C968C1F8600167480068E4
:108ED0000078012805D1694664480068FFF784FFDF
:108EE0001FE0624800680078022805D169465F48A3
:108EF0000068FFF7FBFD14E05C4800680078042878
:108F000005D1694659480068FFF731FC09E0574828
:108F100000680078032804D1694654480068FFF7C8
:108F2000FBFB52480068FEF7B3FE002DA0D10020E5
:108F30004E4908604E49086000BF8BE74B48006807
:108F40007047014609B9002070470878FCE710B562
:108F5000044694F84C0020F0010184F84C1008F00D
:108F6000EEF9A06408F0EBF9606410BD00B9704739
:108F7000CA4390F84C3062F3820380F84C3000BF53
:108F8000F5E770B504460D462078012800D070BD85
:108F90002565E068FEF7AFF906463146206D00F022
:108FA000CDFDB4F92220B4F92010206D00F062F953
:108FB00000BFECE70278022A02D00278042A00D12E
:108FC000416570470278032A00D1816570470278B5
:108FD000012A07D00278032A04D04FF0FF320A801A
:108FE0004A8003E0028C0A80428C4A807047014626
:108FF0000878022801D000207047486AFCE7014643
:1090000009B9002070470878012804D0087803289F
:1090100001D00020F6E791F84000C0F34000F1E7EE
:1090200018B900220A804A8070470278012A06D0C7
:109030000278032A03D000220A804A8003E0028DCE
:109040000A80428D4A8000BFEEE790F84C1021F074
:109050000801083180F84C107047014609B900201A
:109060007047086AFCE7024800687047E800002083
:10907000EC00002010B5FE48007800B110BD09F0EA
:109080008DF809F00EFA08F02EFAFEF7DBF902F07F
:109090007AF801F021FC4FF4B271F64808F05BFE5B
:1090A0005C21F54808F057FEFEF7EDFD07F0E2FC05
:1090B000012007F0A5F90120ED49087000BFDDE7A8
:1090C000014608687047014691F83000C0F300106F
:1090D000704710B50246134600BF1C462046FFF7F6
:1090E000EFFF0346002BF8D1204610BD2DE9F041DB
:1090F0000646306808B9354603E03046FFF7E9FF19
:109100000546DC4808F08AFE044617E004F1240016
:1091100008F084FE07460AE0AF4202D12046BDE8CF
:10912000F081394604F1240008F0D9FE0746002FEB
:10913000F2D12146CF4808F0D2FE0446002CE5D1FA
:109140000020ECE72DE9FC4706463046FFF7BBFF61
:1091500008B1BDE8FC873046FFF7BBFF0446204658
:10916000FFF7C4FF81464846FEF7A4F8A04209D0A5
:109170004846FEF7B5F8A04204D04846FEF7BBF8D3
:10918000A04244D13046FFF79BFF07464FF001084D
:10919000B6F9345006F11001684601F095FBBDF8B0
:1091A0000000401B00B2ADF80000BDF80200401BFB
:1091B00000B2ADF80200BDF80400284400B2ADF8DA
:1091C0000400BDF80600284400B2ADF8060013E024
:1091D00007F110026946684608F09CFB8046B8F12A
:1091E000000F00D10AE03846FFF76DFF00B1B0E78D
:1091F0003846FFF765FF0746002FE9D100BFB8F1F9
:10920000000F03D06946484601F0D5FE00BF00BFFD
:109210009FE72DE9F04107460D461646381D08F038
:10922000FDFD044619E0208A284400B22082608AAD
:10923000304401B26182A08A284401B2A182E08A4E
:10924000304401B2E182324629462046FFF7E1FF71
:109250002146381D08F043FE0446002CE3D1BDE84A
:10926000F08170B505460C4605F11001204601F06D
:109270002BFB70BDFEB504460E4617462568288AAE
:10928000304406B2688A384407B2208A301A00B2E5
:10929000ADF80800608A381A00B2ADF80A00BDF8CF
:1092A000080018B9BDF80A0000B9FEBD2046FFF756
:1092B00049FF69462046FFF7D4FF208ABDF8081011
:1092C000084400B22082608ABDF80A10084401B246
:1092D0006182A08ABDF80810084401B2A182E08A28
:1092E000BDF80A10084401B2E182BDF90A20BDF9B7
:1092F00008102046FFF78DFF6A4602212046E369E9
:109300009847224601212846EB6998472046FFF7F7
:1093100019FF00BFC9E710B502461046FFF7D0FE9F
:109320000446518A608A081A03B2184610BD10B567
:1093300002461046FFF7C4FE0446108A218A401AEE
:1093400003B2184610BD00B503461A460BE092F86A
:109350003000C0F3801010B192F8330000BD104609
:10936000FFF7AEFE0246002AF1D1FF20F6E70146E4
:10937000C86A70472DE9F0410546AE6AFEB92C680F
:1093800019E0A06AB0B1A06A007800F0010080B9CD
:109390002046FFF7ECFF07463846FEF7F7FAA042F3
:1093A00005D13846A16AFEF7E4FB064600E0A66A4E
:1093B00003E000BF2468002CE3D100BF00BFE86ACF
:1093C00048B1E86AFEF7E2FAA84204D13146E86AF9
:1093D000FEF7CFFB064606B9284E3046BDE8F081C1
:1093E0002DE9FC41064688461746022F52D106F168
:1093F0001001404608F03BFB10B90020BDE8FC819D
:109400003046FFF7B7FF0546287AFB2801DA00202F
:10941000F4E7B5F9064047F61840844201D1002030
:10942000ECE769463046FFF71CFFBDF8000020441A
:1094300000B2ADF80000BDF80400001B00B2ADF8AA
:1094400004006946404608F012FB08B90020D5E741
:1094500069463046FFF705FFBDF80200204400B220
:10946000ADF80200BDF80600001B00B208E00000E5
:10947000F0000020842E0020902E00205C2C002084
:10948000ADF806006946404608F0F1FA08B9002038
:10949000B4E710E07FB93046FFF76CFF0446304672
:1094A000FFF751FF05462B462246414606F11000C4
:1094B00006F08AFE00BF0120A0E70162704710B5E8
:1094C00004460020A086002205212046E369984733
:1094D0002046FFF737FE10BD024692F832000840E2
:1094E00008B1012070470020FCE72DE9F041054656
:1094F0000C4616464FF001082846FFF73BFF07468B
:10950000012C07D101212846FFF7E6FFC8B14FF033
:10951000000816E0052C08D1B7F91200B5F934108F
:1095200088420EDD788AA8860BE0042C03D12846F9
:10953000FFF7C5FF05E0062C03D13046F9A1016015
:1095400000BF4046BDE8F081C16170472DE9F041A0
:1095500006460D460024002E79D107F08DFD804689
:10956000B8F1000F02D10020BDE8F08108F124001D
:1095700008F02AFC04460CB900BFFEE70CB9002035
:10958000F2E7002020604421201D08F0E4FB0020C9
:1095900020820021618207F086FD401E01B2A18277
:1095A000002007F06CFD401E01B2E1820020A08681
:1095B000002140200155A187E1870020A0634120C0
:1095C000005D20F00101412001550BF0B3FF07467B
:1095D00017B13868A06201E0D448A062D44920469F
:1095E000FFF7B2FFD3492046FFF767FF002044F89A
:1095F000180F6061207E20F001002076207E20F090
:1096000002002076207E20F004002076207E20F0CC
:1096100008002076207E20F010002076207E20F0AA
:10962000200020760020A076207E20F040002076CA
:10963000FF20E076207E20F080002076607E20F003
:10964000FC0060760020E060183C6DE0FFE7301D14
:1096500008F0BAFB04460CB900BFFEE70CB90020C5
:1096600082E726604421201D08F075FB308A2082A5
:10967000718A6182308A3C3001B2A182708A2830BE
:1096800001B2E1820020A086002140200155A1877F
:10969000E1870020A0634120005D20F0010141200E
:1096A00001550BF047FF074617B1B868A06201E00B
:1096B000A148A0629E492046FFF746FF9D492046EB
:1096C000FFF7FBFE002044F8180F6061207E20F0B9
:1096D0000100401C2076207E20F002002076607E73
:1096E00020F00300C01C6076207E20F0040020766D
:1096F000207E20F008002076207E20F010002076CA
:10970000207E20F0200020760020A076FF20E0764A
:10971000207E20F040002076207E20F08000207601
:109720000020E060183C00BF002D76D005F110014C
:1097300004F1100001F0C8F8A88EA0864020415D19
:109740000155A98FA187E98FE187A86BA06341200C
:10975000405D4121095D60F300014120015555F84C
:10976000180F44F8180F287E217E60F3000121763F
:10977000287E4108207E61F341002076687E617E6C
:1097800060F301016176287E8108207E61F382000A
:109790002076287EC108207E61F3C3002076287ED3
:1097A0000109207E61F304102076287E4109207E85
:1097B00061F345102076287EC109207E61F3C71031
:1097C0002076287E8109207E61F386102076A87E8F
:1097D000A076E87EE07628692061183C6869183D2B
:1097E00018B12146E86AFEF735F82846FFF768FC0D
:1097F00070B16EB12846FFF78EFD07462846FFF789
:1098000096FD80463A4641462046FFF733FD04E088
:10981000002211462046FFF72DFD3EB122460121D0
:109820003046F36998472046FFF78CFC20469BE6BC
:109830000146424A106805E002688A4201D10122CD
:10984000027180680028F7D170472DE9FE4F064667
:109850000C4690461F46009400208DF804000290AC
:109860003648006810B13548006802903349C1F8A5
:1098700000D03348D0F800900760FFF75FFB054643
:109880002DB1A86818B141462846AA68904716B17C
:1098900041462046B0472A48C0F800902748006853
:1098A0008068264908609DF8040010B10020BDE8DA
:1098B000FE8F8CB194F83000C00968B1206858B1AF
:1098C0003A464146206800F009F88246BAF1010F95
:1098D00001D00020EBE700BF0120E8E72DE9F041CF
:1098E00004460D46164614B90120BDE8F081334602
:1098F0002A462146A069FFF7A8FF07463846F4E745
:109900002DE9F0470446201D08F088FA0646204657
:10991000FFF72DFD8046B8F1000F02D02046FDF77D
:10992000CEFF18E06C765F6F626A00006C2B00203F
:10993000EB940008E1930008982C0020F40000202C
:10994000F80000203146201D08F0C9FA07463046CD
:10995000FFF7D6FF3E46002EF4D100221321204609
:10996000FFF7BCFF2046FFF763FF0021204607F00A
:10997000F5FD002007F0ABFC05461BE0686BA0423C
:1099800002D0A86BA04202D12846FEF75DF9E86B31
:10999000A04201D10021E963686D404506D1FFF77F
:1099A00062FBA04202D12846FEF74EF9284607F096
:1099B0008EFC0546002DE1D12046FFF781FB814654
:1099C000214609F1040008F09AFA002211462046C7
:1099D000E3699847606A10B1606A08F072FC20463B
:1099E00008F06FFCBDE8F0872DE9F04704462046FB
:1099F000FFF7A8FB2046FFF7BAFC8046B8F1000F3E
:109A000002D02046FDF75BFF0021204607F0A6FDAF
:109A1000201D08F003FA074608E03946201D08F02B
:109A20005EFA81463846FFF76BFF4F46002FF4D1B0
:109A3000002213212046FFF751FF2046FFF7F8FED2
:109A40002046FFF73DFB06464EB92046FFF74EFB8A
:109A5000824621460AF1240008F051FA03E021462B
:109A6000301D08F04CFA002007F031FC05461BE0E1
:109A7000686BA04202D0A86BA04202D12846FEF734
:109A8000E3F8E86BA04201D10021E963686D40452D
:109A900006D1FFF7E8FAA04202D12846FEF7D4F833
:109AA000284607F014FC0546002DE1D1002211469E
:109AB0002046E3699847606A10B1606A08F001FCCB
:109AC000204608F0FEFB26B1002201213046F36952
:109AD00098470020BDE8F08710B504462046FFF700
:109AE00083FF10BD10B504462146FC4807F0E6FF91
:109AF00010BD70B504460D46002625B9201D08F09E
:109B00008DF9064604E02946201D08F0E8F90646CE
:109B1000304670BD70B5064600213046FFF7E9FFBC
:109B2000044608E021463046FFF7E3FF054620469D
:109B3000FFF75AFF2C46002CF4D170BDF8B504464F
:109B40000D46206800B9F8BD05B9FCE72046FFF7CF
:109B5000F9FA2046FFF7EBFBADF800002046FFF7CF
:109B6000DAFBADF8020026682168081D01232246B1
:109B7000291D08F021FA2560BDF90220BDF9001069
:109B80002046FFF777FB002201213046F369984712
:109B9000224601212846EB6998472046FFF7D2FA72
:109BA00000BFD0E770B505462846FFF789FA04469E
:109BB000201D08F033F9A84200D170BD2046FFF700
:109BC000C1FA01232A46211D201D08F0F5F92A4675
:109BD00001212046E36998472046FFF7B3FA00BF0A
:109BE000EBE770B505462846FFF76AFA0446201DE4
:109BF00008F080F9A84200D170BD2046FFF7A2FA14
:109C000000232A46211D201D08F0D6F92A460121ED
:109C10002046E36998472046FFF794FA00BFEBE738
:109C200070B504460D462046FFF775FB06463246E2
:109C300029462046FFF71EFB70BD70B505460C4651
:109C40002846FFF774FB0646224631462846FFF7B2
:109C500011FB70BD014600BFC88A4A8A801A401CA9
:109C600000B27047014600BF888A0A8A801A401CE9
:109C700000B270472DE9F04F87B004460D461646F6
:109C80001F46DDF840B02046FFF751FB80462046D6
:109C9000FFF741FB81461DB92046FFF711FA054643
:109CA000152E2ED2DFE806F00B2E324653607C9143
:109CB000A5C1CAE2FCFAF9F8F7F6F5F4F300284674
:109CC000FFF7D0FF019000EBD07043102046FFF764
:109CD000C9FF029000EBD070A3EB60000FFA80F890
:109CE0002846FFF7B7FF019000EBD07043102046E5
:109CF000FFF7B0FF029000EBD070A3EB60000FFA0B
:109D000080F95AE14FF00008C14656E12846FFF7B6
:109D1000A9FF019000EBD07043102046FFF7A2FF8F
:109D2000029000EBD070A3EB60000FFA80F84FF0C8
:109D3000000942E12846FFF795FF03462046FFF75A
:109D400091FF181A0FFA80F84FF0000935E14FF033
:109D500000082846FFF77EFF03462046FFF77AFFFC
:109D6000181A0FFA80F928E12846FFF77BFF0190C7
:109D700000EBD07043102046FFF774FF029000EB19
:109D8000D070A3EB60000FFA80F82846FFF762FF5F
:109D900003462046FFF75EFF181A0FFA80F90CE120
:109DA0002846FFF75FFF03462046FFF75BFF181AC0
:109DB0000FFA80F82846FFF74DFF03462046FFF7CD
:109DC00049FF181A0FFA80F9F7E04FF0000828460B
:109DD000FFF740FF019000EBD07043102046FFF7E3
:109DE00039FF029000EBD070A3EB60000FFA80F90E
:109DF000E3E02846FFF736FF03462046FFF732FF31
:109E0000181A0FFA80F82846FFF724FF019000EB9C
:109E1000D07043102046FFF71DFF029000EBD0707A
:109E2000A3EB60000FFA80F9C7E04FF0000820466E
:109E3000FFF710FF40420FFA80F9BEE02846FFF717
:109E400011FF019000EBD07043102046FFF70AFF8E
:109E5000029000EBD070A3EB60000FFA80F8204670
:109E6000FFF7F8FE40420FFA80F9A6E02846FFF718
:109E7000F9FE03462046FFF7F5FE181A0FFA80F8A0
:109E80002046FFF7E7FE40420FFA80F995E085E0B3
:109E90006EE066E054E03BE031E021E007E0FFE700
:109EA0004FF000082846FFF7D5FE814685E028469A
:109EB000FFF7D8FE019000EBD07043102046FFF76B
:109EC000D1FE029000EBD070A3EB60000FFA80F897
:109ED0002846FFF7BFFE81466FE00000D99A0008D0
:109EE0002846FFF7BFFE03462046FFF7BBFE181AC1
:109EF0000FFA80F82846FFF7ADFE81465DE0204668
:109F0000FFF7B0FE40420FFA80F84FF0000954E02E
:109F10002046FFF7A7FE40420FFA80F82846FFF7D9
:109F200099FE019000EBD07043102046FFF792FE9F
:109F3000029000EBD070A3EB60000FFA80F93CE0D8
:109F40002046FFF78FFE40420FFA80F82846FFF7C1
:109F500081FE03462046FFF77DFE181A0FFA80F9AE
:109F60002BE02846FFF77EFE80464FF0000924E0F4
:109F70002846FFF777FE80462846FFF76BFE0190E4
:109F800000EBD07043102046FFF764FE029000EB18
:109F9000D070A3EB60000FFA80F90EE02846FFF7BF
:109FA00061FE80462846FFF755FE03462046FFF730
:109FB00051FE181A0FFA80F900BF00BF2046FFF7C4
:109FC0007FF88246B5F910000690B5F912000590A9
:109FD000BAF910000490BAF91200039006983844B8
:109FE00040440FFA80F80598584448440FFA80F925
:109FF0000498A8EB00000FFA80F80398A9EB000082
:10A000000FFA80F94A4641462046FFF733F94020CF
:10A010000655A787A4F83EB0A5634120005D20F057
:10A0200002014120015507B0BDE8F08F2DE9F04F46
:10A0300085B006460F46904699463046FFF777F9B9
:10A0400082463046FFF767F983463046FFF70AFE3F
:10A05000034600EBD37044103046FFF7FBFD034688
:10A0600000EBD37045101FB93046FFF729F80746BB
:10A07000B8F1150F20D2DFE808F00B2027353F4953
:10A080005A6775868D9BA5AFC0CDD4E2EFF9EC0081
:10A090003846FFF7E7FD034600EBD370C4EB6000E2
:10A0A0000FFA80FA3846FFF7D5FD034600EBD37070
:10A0B000C5EB60000FFA80FBF6E060420FFA80FA11
:10A0C00068420FFA80FBEFE03846FFF7CBFD03460E
:10A0D00000EBD370C4EB60000FFA80FA68420FFA0D
:10A0E00080FBE1E03846FFF7BDFD001B0FFA80FA68
:10A0F00068420FFA80FBD7E060420FFA80FA3846D8
:10A10000FFF7A8FD401B0FFA80FBCDE03846FFF7B4
:10A11000A9FD034600EBD370C4EB60000FFA80FA90
:10A120003846FFF797FD401B0FFA80FBBCE038462E
:10A13000FFF798FD001B0FFA80FA3846FFF78AFDFB
:10A14000401B0FFA80FBAFE060420FFA80FA3846FE
:10A15000FFF780FD034600EBD370C5EB60000FFAFC
:10A1600080FBA1E03846FFF77DFD001B0FFA80FA67
:10A170003846FFF76FFD034600EBD370C5EB600078
:10A180000FFA80FB90E060420FFA80FA68420FFA03
:10A1900080FB89E03846FFF765FD034600EBD3708E
:10A1A000C4EB60000FFA80FA68420FFA80FB7BE094
:10A1B0003846FFF757FD001B0FFA80FA68420FFA86
:10A1C00080FB71E060420FFA80FA3846FFF742FDEB
:10A1D000401B0FFA80FB67E03846FFF743FD03465C
:10A1E00000EBD370C4EB60000FFA80FA3846FFF73B
:10A1F00031FD401B0FFA80FB56E03846FFF732FD79
:10A20000001B0FFA80FA3846FFF724FD401B0FFAB7
:10A2100080FB49E060420FFA80FA68420FFA80FB47
:10A2200042E060420FFA80FA3846FFF713FD03461A
:10A2300000EBD370C5EB60000FFA80FB34E06042A6
:10A240000FFA80FA3846FFF705FD401B0FFA80FB36
:10A250002AE01CE00AE0FFE73846FFF703FD001B99
:10A260000FFA80FA68420FFA80FB1DE03846FFF7CC
:10A27000F9FC001B0FFA80FA3846FFF7EBFC0346A7
:10A2800000EBD370C5EB60000FFA80FB0CE03846A2
:10A29000FFF7E8FC001B0FFA80FA3846FFF7DAFCFC
:10A2A000401B0FFA80FB00BF00BF3046FEF708FFDF
:10A2B0000490B7F910000390B7F9120002900498C7
:10A2C000B0F9100001900498B0F9120000900398C2
:10A2D000484450440FFA80FA0E99029808445844B2
:10A2E0000FFA80FB0198AAEB00000FFA80FA0098A1
:10A2F000ABEB00000FFA80FB5A4651463046FEF7A2
:10A30000B9FF86F84080A6F83C900E98F087B763B6
:10A310004120805D20F00200801C4121885505B05D
:10A32000BDE8F08F38B504464120005DC0F3400021
:10A3300058B1B4F93E000090B4F93C304020025DC1
:10A340002046A16BFFF772FE0AE0B4F93E000090D0
:10A35000B4F93C304020025D2046A16BFFF78AFC37
:10A3600038BD2DE9FC4104460F4690462046FFF7D4
:10A3700079FCB84206D12046FFF76CFC404501D17C
:10A38000BDE8FC812046FEF7DDFE69462046FEF76B
:10A3900068FF208A3844401E01B2A182608A40448E
:10A3A000401E01B2E1826A4602212046E3699847D5
:10A3B0002046FEF785FE064626B12246012130469C
:10A3C000F3699847201D07F029FD054609E00022A2
:10A3D00003212846EB6998472946201D07F07FFD99
:10A3E0000546002DF3D12046FEF7ACFE4120005D6E
:10A3F00000F0010010B12046FFF794FF00BFBFE757
:10A4000070B504460D462046FFF724FC064632464A
:10A4100029462046FFF7A5FF70BD70B505460C46DE
:10A420002846FFF71FFC0646224631462846FFF71E
:10A4300098FF70BD4122125C61F3000241231A545F
:10A44000704710B5029C10BD10B504462046FEF7BB
:10A4500079FE002204212046E36998472046FEF752
:10A4600071FE10BD70B5054600212846FFF741FB7F
:10A47000044615E0A06A30B92046FFF7F3FF2046F6
:10A48000FFF7E2FF07E0A06A007800F0010010B1DA
:10A490002046FFF7E7FF21462846FFF72AFB044640
:10A4A000002CE7D170BD70B504460D46A56220466C
:10A4B000FFF7D8FF2046FFF7C7FF70BD70B5054610
:10A4C0000E46301D07F0AAFC044612E0A06AA8421E
:10A4D00000D02DB92046FFF7C5FF2046FFF7B4FF97
:10A4E00021462846FFF7EAFF2146301D07F0F7FC1A
:10A4F0000446002CEAD170BD70B50646002006F077
:10A500004BFE04461DE004F1240007F087FC0546DD
:10A5100010E0A86AB04200D016B92846FFF794FFB1
:10A5200029463046FFF7CAFF294604F1240007F008
:10A53000D6FC0546002DECD1204606F02DFE044643
:10A5400000BF002CDFD170BD70B504460D4694F8F5
:10A550003000C0F3001010B92046FEF7F3FD14F8E8
:10A56000300F65F30410207014F83009C0F30010A8
:10A5700010B92046FEF7E6FD2046FEF7A1FD06468F
:10A58000224601213046F369984770BDCA43D24341
:10A5900090F8303062F3000380F830307047CA43DF
:10A5A000D24390F8303062F3451380F83030704772
:10A5B00030B504460D46012D02D12046FFF7E6FFD7
:10A5C000E843C04394F8301060F3410184F8301040
:10A5D00030BD30B504460D4614F8310F65F3010067
:10A5E000207014F8310900F0030018B10121204651
:10A5F000FFF7DEFF30BDCA43D24390F8303062F33C
:10A60000820380F830307047CA43D24390F830302C
:10A6100062F3C30380F830307047CA43D24390F8E6
:10A62000303062F3C71380F83030704790F8302034
:10A6300061F3861280F83020704770B504460D46ED
:10A6400084F833502046FEF77DFD70BD90F832202F
:10A650000A4380F832207047CA43D1B290F83220C2
:10A660000A4080F83220704781617047994800683D
:10A67000704770B504460D461646E06920B1324673
:10A6800029462046E369984770BD70B504460D46DB
:10A690002946606A07F04CFE6062606A70BD70B562
:10A6A00004460D46002625B9201D07F023FC06466A
:10A6B00004E02946201D07F0A7FB0646304670BD82
:10A6C00070B504460026201D07F0A8FB054606E0ED
:10A6D000701C86B22946201D07F001FC0546002D9E
:10A6E000F6D1304670BD70B506460025301D07F026
:10A6F00095FB04460BE0681C85B22046FFF7F3FF8C
:10A70000284485B22146301D07F0E9FB0446002CA1
:10A71000F1D1284670BD70B506460C463046FEF7AE
:10A7200029FE0546A87B00F0040020B12188A889F5
:10A73000084400B22080A87B00F0080020B1A18866
:10A74000A889081A00B2A080A87B00F0020020B1FE
:10A750006188A889084400B26080A87B00F00100ED
:10A7600020B1E188A889081A00B2E08070BD70B5F8
:10A7700005462846FEF7FEFD04462846FFF772FA16
:10A780000146608B091AA08B081A00B270BD70B523
:10A7900005462846FEF7EEFD04462846FFF75AFA1E
:10A7A000E18A411A208B081A00B270BD014641208F
:10A7B000405C00F0010070470146002070470146F0
:10A7C0000020704701460020704701460020704776
:10A7D0000146B1F934007047014691F8300000F0AD
:10A7E00001007047014691F83000C0F340107047F7
:10A7F000014691F83000C0F340007047014691F8DF
:10A80000310000F003007047014691F83000C0F3BA
:10A8100080007047014691F83000C0F3C0007047D7
:10A82000014691F83000C0097047014691F83000A8
:10A83000C0F380107047014691F83200704701461E
:10A84000C86970470146086A7047014688697047C1
:10A850000146486A7047F0B589B007460E46202188
:10A86000304613F076F9202101A813F072F901AAFD
:10A8700006213846FB699847002406E001A850F8F5
:10A88000240000B903E0601CC4B2082CF6DB00BF52
:10A89000002508E0601E401B01A951F8200046F881
:10A8A0002500681CC5B2A542F4DB09B0F0BD10B5A7
:10A8B0000446E06A30B1E06AFDF768F8A04201D1D1
:10A8C000012010BD0020FCE70A6802604A6842606F
:10A8D00070470000F80000207047FE48006870478D
:10A8E00070B5FC48006806F063FC0446F94800684F
:10A8F00006F079FC28B100BFA06900F00100002833
:10A90000FAD1A06920F00100401CA061FFF7E5FF2B
:10A910000546E86828B1A26804F110012846EB68F2
:10A920009847206850B1606840B12168A0688842AB
:10A9300002D16068A06001E02068A06070BD2DE9D0
:10A94000F0418AB00546884695F83000C0F3001003
:10A9500010B10AB0BDE8F081B5F9344004A9284629
:10A96000FEF77FFCBDF81000001B00B2ADF8100030
:10A97000BDF81200001B00B2ADF81200BDF81400C3
:10A98000204400B2ADF81400BDF81600204400B217
:10A99000ADF8160004AA414606A806F0BBFF06461D
:10A9A000002E4AD0002206A928462B6A984704A9FF
:10A9B0002846FEF756FC04AA414608A806F0AAFF5E
:10A9C0000646AEB3281D07F095FA07462DE0694606
:10A9D0003846FEF746FCB7F93440BDF80000001BCE
:10A9E00000B2ADF80000BDF80200001B00B2ADF8E7
:10A9F0000200BDF80400204400B2ADF80400BDF828
:10AA00000600204400B2ADF806006A4608A902A874
:10AA100006F080FF06461EB102A93846FFF78FFFF9
:10AA20003946281D07F0F0F90746002FCFD100BFA7
:10AA3000012206A928462B6A984700BF89E72DE91D
:10AA4000F0410546884625B9A2480068FCF732FC6B
:10AA5000054641462846FFF772FF2F462846FEF777
:10AA60002FFB04461BE03946201D07F0CDF90646B2
:10AA700008E041463046FFF762FF3146201D07F0EF
:10AA8000C3F90646002EF4D1012241462046236A2E
:10AA9000984727462046FEF713FB044600BF002CCC
:10AAA000E1D1BDE8F0812DE9F04106460C460025D4
:10AAB00004F11001304606F0DAFF00282FD094F898
:10AAC0003000C0F3001050BB201D07F0A7F9074667
:10AAD0000BE039463046FFF7E6FF054605B106E0D4
:10AAE0003946201D07F0FBF90746002FF1D100BFC2
:10AAF000A5B92046FEF73EFC804698F80800FF28DE
:10AB00000BD1022231462046236A984728B12046BD
:10AB1000FEF719FCFF2800D1254600BF00BF2846DC
:10AB2000BDE8F0812DE9FC4104466A48006806F062
:10AB30003FFB05466748006806F055FB28B900BF93
:10AB4000A86900F001000028FAD105F110022146A1
:10AB5000684606F0DFFE5F480068FCF7ABFB07467F
:10AB600039466846FFF79FFF064669463046FFF7BD
:10AB700066FF58480068FCF7B3FB07466946FFF7D5
:10AB80005EFF54480068FCF7B6FB07466946FFF7CE
:10AB900056FF5048006806F031FB08B9FFF7A0FEE9
:10ABA000BDE8FC812DE9FE4F05464A48006806F0E5
:10ABB00025FBD0B14748006806F0FAFA04460020A9
:10ABC00020824448006806F06EFA401E01B2A1825D
:10ABD000002161823F48006806F051FA401E01B230
:10ABE000E1822846FFF79EFF88E03A48006806F0B9
:10ABF000DFFA0446284600F055FA0290284600F095
:10AC000058FA82463348006806F039FAB5F906105A
:10AC1000884206DC2F48006806F031FA401E00B278
:10AC200001E0B5F906000746E1680298B1FBF0F6CD
:10AC3000564500DD564627480068006950B300209D
:10AC4000ADF80000ADF80400ADF80200701E0FFA78
:10AC500080F900BFADF806901E4800686946026999
:10AC60001C4800689047684600F023FAB04200DCB8
:10AC700006E0A9F101000FFA80F9B9F1000FE9D15E
:10AC800000BFB9F1000F01D1BDE8FE8FBDF906008C
:10AC9000461C00BF4FF0000BB5F9028018E0288871
:10ACA0002082A988A182A4F8128008EB0600401E29
:10ACB00001B2E182B4F91600B84200DDE782B4F9CE
:10ACC00016B02846FFF72EFF08EB06000FFA80F8B3
:10ACD00002E000000001002008EB0600401EB84220
:10ACE000DDDD5F4509D028882082A988A182A4F8EB
:10ACF0001280E7822846FFF715FF00BF00BFC3E7B9
:10AD000010B50020EE49086000241DE0ED48006801
:10AD100000F59E70005DB0B9EA4909683C3101EB6D
:10AD2000C400FFF73FFFE7480068806958B1E54974
:10AD300009683C3101EBC40006F0DBFDE04909681D
:10AD40000844DF490860641CDE480068B0F85C0114
:10AD5000C0F30900A042D9D810BD2DE9FC4100255F
:10AD60005CE0D848006800F59E70405D00B154E09A
:10AD7000002449E0D348006800F59E70005D08B9E2
:10AD8000A54200D13FE0CF4A12683C3202EBC40139
:10AD9000CC4A12683C3202EBC50006F04BFE00B90B
:10ADA00031E0C84800683C3000EBC402C548006888
:10ADB0003C3000EBC501684606F0EDFD684606F044
:10ADC00098FD0646BF4909683C3101EBC50006F015
:10ADD00090FD0746BB4909683C3101EBC40006F011
:10ADE00088FD384486420DD2B64909683C3101EBF2
:10ADF000C500694600F051F90121B248006800F52C
:10AE00009E70015500BF641CAE480068B0F85C013C
:10AE1000C0F30900A042ADD800BF6D1CA94800686E
:10AE2000B0F85C01C0F30900A8429AD8BDE8FC81E3
:10AE30002DE9FC5F804606F082FA0190A149D8F81E
:10AE40000C000860FFF789FFFFF75AFF9D48006874
:10AE5000B0F85C01C0F3090000287DD09948006873
:10AE600006F0CCF9002865D09648006806F0A0F9F5
:10AE70000546FFF735FD00BFA86900F00100002876
:10AE8000FAD1D5F808902968A868884201D1686885
:10AE900000E0286800908B48006806F004F9064638
:10AEA00000243EE08748006800F59E70005DB0BB5E
:10AEB000844800683C3030F93410824800683C30E7
:10AEC00000EBC400B0F9020006FB001047007D490A
:10AED00009683C3101EBC40000F0E4F84FEA400B94
:10AEE000784800683C3000EBC400B0F902A00CE0E8
:10AEF000009AD11909EB07005A4612F00AFD07EB38
:10AF000046070AF101000FFA80FA6E4800683C30EB
:10AF100000EBC400B0F906005045E9DA00BF601C40
:10AF200084B268480068B0F85C01C0F30900A04230
:10AF3000B8DC00BF4FF48071624800683C3012F00A
:10AF4000E6FD20215F48006800F59E7012F001FECA
:10AF500000205C49096800E012E0C1F85C01594832
:10AF60000068806960B1019806F0F4F9044655481C
:10AF70000068836952482146026852480068984731
:10AF800000F012FEBDE8FC9F70B504461CB1206ABB
:10AF9000FFF74EFF0EE0002006F0FEF8054606E043
:10AFA000286AFFF745FF284606F0F6F80546002D0B
:10AFB000F6D100BF70BD2DE9FF4104460F4614B91C
:10AFC00006F05AF804460CB9BDE8FF811FB900200D
:10AFD000C4F85C01F8E70020ADF80800ADF80A00FD
:10AFE000204606F060F8401E00B2ADF80C00204686
:10AFF00006F045F8401E00B2ADF80E0002AA394630
:10B00000684606F087FC0646F6B3206918B1694623
:10B0100020462269904700250AE004F13C0000EB3D
:10B02000C501684606F023FD00B1CDE7681C85B276
:10B03000B4F85C01C0F30900A842EEDCB4F85C018E
:10B04000C0F3090020280BDAB4F85C11C1F309023F
:10B0500004F13C0101EBC200694600F01EF80DE06E
:10B060000020C4F85C01B4F85C11C1F3090204F1DA
:10B070003C0101EBC20002A900F00FF8B4F85C013A
:10B08000C0F30900401C00E002E0C4F85C0100BF0E
:10B0900000BF99E70B49086070470A6802604A6878
:10B0A00042607047014688880A88801A401C00B2B6
:10B0B00070470146C8884A88801A401C00B2704711
:10B0C000FC0000200001002007B581B0BDF8080099
:10B0D000C00AC2F1FF014843BDF80410C90A01FBD0
:10B0E0000200010ABDF8000061F3CF200090BDF816
:10B0F0000800C0F34510C2F1FF014843BDF8041039
:10B10000C1F3451101FB0200010ABDF8000061F323
:10B110004A100090BDF8080000F01F00C2F1FF01C6
:10B120004843BDF8041001F01F0101FB0200010AB1
:10B13000BDF8000061F304000090BDF8001008465F
:10B1400004B000BD18B50346D408BDF8000064F390
:10B15000040000908C08BDF8000064F34A100090D1
:10B16000DC08BDF8000064F3CF200090BDF800407B
:10B17000204618BD70B504460D463C22294620469F
:10B1800012F04EFC70BD00B589B00020FE49087079
:10B19000FF21FD48017200200890FB48BDF82010F7
:10B1A000418000200790F848BDF81C1081800021E4
:10B1B000C18041838183C18201830321C183002037
:10B1C0000690F148BDF818104181FF21C17300219C
:10B1D00081810F218173ED4800680590EA48BDF830
:10B1E000141001820121017500214182FF2180F8A4
:10B1F0002C10302211461046FFF7A4FF0190E248C0
:10B20000BDF804100184D82296215520FFF79AFF3B
:10B210000190DD48BDF804104184DD494162002100
:10B22000018502214185FF2180F83310202211463B
:10B230001046FFF787FF0190D348BDF80410018640
:10B24000002180F83210FF2180F8381020221146AA
:10B250001046FFF777FF0190CB48BDF804108186B8
:10B260000221C186002180F839100146C948FFF744
:10B2700081FF0321C74841838183C1820183014645
:10B28000C548FFF777FFF02211461046FFF75AFF37
:10B290000190C148BDF804100184F0221146104607
:10B2A000FFF750FF0190BC48BDF804100186F02262
:10B2B00011461046FFF746FF0190B748BDF804104D
:10B2C0008186D82296215520FFF73CFF0190B24895
:10B2D000BDF804104180014649888180AD49AF48DE
:10B2E000FFF748FF202211461046FFF72BFF019081
:10B2F000AA48BDF804100184202211461046FFF729
:10B3000021FF0190A548BDF80410018620221146B6
:10B310001046FFF717FF0190A048BDF80410818682
:10B320009A48001D006804909C48BDF810104180A8
:10B3300096480830006803909848BDF80C1081804A
:10B340000421C180402211461046FFF7FBFE019008
:10B350009248BDF804104181012181814C21C173C3
:10B3600001468F48FFF706FFE02211461046FFF71F
:10B37000E9FE01908A48BDF804100184E0221146DC
:10B380001046FFF7DFFE01908548BDF804100186E6
:10B39000C02211461046FFF7D5FE01908048BDF847
:10B3A00004108186C7229A216B20FFF7CBFE019003
:10B3B0007B48BDF8041041808B2259212B20FFF7D8
:10B3C000C1FE01907648BDF80410818042222C21F4
:10B3D0001520FFF7B7FE01907148BDF804104181B8
:10B3E0006C497048FFF7C6FE01206E4908700021C5
:10B3F0006C488181017201466B48FFF7BBFE00215A
:10B40000694841838183C182018301466748FFF710
:10B41000B1FE00216548C1835E496548FFF7AAFE79
:10B42000D022A2217620FFF78DFE01906048BDF862
:10B43000041041805D223A211920FFF783FE01901C
:10B440005B48BDF8041081800421C1800F21418335
:10B4500081830A21C18201830621C1832822192107
:10B460000B20FFF76FFE01905148BDF80410418199
:10B4700001218181B221C17344480C3000680290DF
:10B480004B48BDF80810018200214182FF2211467D
:10B490001046FFF757FE01904548BDF8041001849F
:10B4A000FF2211461046FFF74DFE01904048BDF8BF
:10B4B0000410018601463F48FFF75CFE942262219A
:10B4C0003320FFF73FFE01903A48BDF80410418059
:10B4D0003C2226211020FFF735FE01903548BDF8AB
:10B4E00004108180C622B521A420FFF72BFE019015
:10B4F0003048BDF804100184C622B521A420FFF70E
:10B5000021FE01902B48BDF804100186C622B5210A
:10B51000A420FFF717FE01902648BDF8041081868D
:10B5200023492548FFF726FE222211210A20FFF792
:10B5300009FE01902048BDF804104180902262214C
:10B540003720FFF7FFFD01901B48BDF804108180F4
:10B550000D2207210120FFF7F5FD01901648BDF8E7
:10B5600004104181F422DD21C820FFF7EBFD01909A
:10B570001148BDF804100184F422DD21C820FFF732
:10B58000E1FD01900C4819E06C2B002048080208EE
:10B59000480100205C2C0020982C0020D42C002096
:10B5A000102D0020A82B0020E42B0020202C0020B0
:10B5B0004C2D0020882D0020C42D0020BDF8041043
:10B5C0000186F422DD21C820FFF7BCFD0190FE4872
:10B5D000BDF8041081860146FC48FFF7CBFD272209
:10B5E00014210220FFF7AEFD0190F848BDF80410C9
:10B5F000418070224C212B20FFF7A4FD0190F348DD
:10B60000BDF804108180C622B521A420FFF79AFD61
:10B610000190EE48BDF804100184C622B521A42093
:10B62000FFF790FD0190E948BDF804100186C6229D
:10B63000B521A420FFF786FD0190E448BDF8041071
:10B640008186E349E348FFF795FDD822114610466D
:10B65000FFF778FD0190DF48BDF804104180D82243
:10B6600011461046FFF76EFD0190DA48BDF8041050
:10B670008180902211461046FFF764FD0190D54865
:10B68000BDF804104181702211461046FFF75AFDA3
:10B690000190D048BDF80410018470221146104674
:10B6A000FFF750FD0190CB48BDF8041001867022D1
:10B6B00011461046FFF746FD0190C648BDF804103C
:10B6C000818609B000BD2DE9FE4304460E461546AD
:10B6D0001F46217A307A814208D0317A207A081ABE
:10B6E0007843217A01EB2020287201E0217A297227
:10B6F000B4F90610B6F9060081420BD0B6F906106F
:10B70000B4F90600081A7843E18801EB202001B261
:10B71000E98001E0E188E980B4F90C10B6F90C0089
:10B7200081420BD0B6F90C10B4F90C00091A794318
:10B7300080B200EB212001B2A98101E0A189A98199
:10B74000E17BF07B814207D0F17BE07B091A7943F2
:10B7500000EB2120E87301E0E17BE973B4F91210FA
:10B76000B6F9120081420BD0B6F91210B4F91200EA
:10B77000091A794380B200EB212001B2698201E00D
:10B78000618A6982B4F91A10B6F91A0081420BD0A5
:10B79000B6F91A10B4F91A00091A794380B200EB0D
:10B7A000212001B2698301E0618B6983B4F91C1027
:10B7B000B6F91C0081420BD0B6F91C10B4F91C007C
:10B7C000091A794380B200EB212001B2A98301E07C
:10B7D000A18BA983B4F91610B6F9160081420BD0DB
:10B7E000B6F91610B4F91600081A7843E18A01EB8D
:10B7F000202001B2E98201E0E18AE982B4F918105F
:10B80000B6F9180081420BD0B6F91810B4F9180037
:10B81000091A794380B200EB212001B2298301E0AB
:10B82000218B2983B4F91E10B6F91E0081420BD07A
:10B83000B6F91E10B4F91E00091A794380B200EB64
:10B84000212001B2E98301E0E18BE983B4F92A10F8
:10B85000B6F92A0081420BD0B6F92A10B4F92A00B1
:10B86000081A7843618D01EB202001B2698501E05F
:10B87000618D6985B4F92810B6F9280081420BD092
:10B88000B6F92810B4F92800081A7843218D01EB85
:10B89000202001B2298501E0218D29852C20015D20
:10B8A000805D81420CD02C20815D005D081A7843B8
:10B8B0002C21095D01EB2020C1B22C20415502E072
:10B8C0002C20015D4155B4F93610B6F9360081429D
:10B8D0000BD0B6F93610B4F93600081A7843E18E69
:10B8E00001EB202001B2E98601E0E18EE9863820F3
:10B8F000015D805D81420CD03820815D005D081AB9
:10B9000078433821095D01EB2020C1B23820415530
:10B9100002E03820015D41553220015D805D8142A9
:10B920000CD03220815D005D081A78433221095D18
:10B9300001EB2020C1B23220415502E03220015DEE
:10B9400041553320015D805D81420CD03320815D03
:10B95000005D081A78433321095D01EB2020C1B254
:10B960003320415502E03320015D4155B7F5807F1A
:10B9700001D1FF2000E0384600F0FF086088019008
:10B980007088424600900199FFF79EFB0290BDF837
:10B9900008006880A0880190B08842460090019914
:10B9A000FFF792FB0290A81CBDF80810A9806089DF
:10B9B00001907089424600900199FFF785FB029043
:10B9C000A81CBDF8081007E0C42D0020002E0020A0
:10B9D0004C2D00203C2E00206981208A0190308A65
:10B9E000424600900199FFF76FFB0290A81CBDF83A
:10B9F000081029824246216A306AFFF765FB0290EF
:10BA0000BDF808002884208E0190308E42460090B8
:10BA10000199FFF759FB0290BDF808002886A08E17
:10BA20000190B08E424600900199FFF74DFB0290C5
:10BA3000BDF80800A886802F10DAA17BA9732078B2
:10BA400000F001002870616A6962217D2975392042
:10BA5000005D00F00100392148550FE0B17BA9736A
:10BA6000307800F001002870716A6962317D2975B3
:10BA70003920805D00F0010039214855BDE8FE8382
:10BA800070B505462C68E06F10B12846E16F884715
:10BA9000204606F016FC70BD2DE9F04104460E4626
:10BAA000254604F13C07D4F87880B3B242463946C3
:10BAB0002846FFF708FEA06FFEF71EFDBDE8F081E7
:10BAC00070B50446204605F038FD002020614FF493
:10BAD000807060611B4860601B48A0601B48E0608C
:10BAE000802006F0BEFB05460DB900BFFEE705B994
:10BAF00070BD0020E867A86715492846FFF73AFBA4
:10BB0000134905F13C00FFF735FB256000BFEFE767
:10BB10002DE9F04105460E46174698462C68A66763
:10BB20003C223946204611F07BFF3C22414604F17D
:10BB30003C0011F075FF3C223946A06F11F070FFF8
:10BB4000BDE8F08199BA00080715010881BA00081C
:10BB50005C2C002010B5044654480068844202D88A
:10BB60005348006810BD514804605148006860B9EE
:10BB7000204606F076FB4E4908600846006808B982
:10BB800000BFFEE74A480068ECE7214648480068E5
:10BB900006F0CEFB464908600846006808B900BFB9
:10BBA000FEE743480068DDE710B54148006840B152
:10BBB0003F48006806F085FB00203D4908603B498E
:10BBC000086010BD10B503460BB9002010BD082B4E
:10BBD00007DA581E374C54F82000405C5043000AE6
:10BBE000F4E7012000EB410050435C0090FBF4F0CF
:10BBF000C0B2EBE72DE9F84F82460E4614461F46C9
:10BC0000DDF82C804FF0000B002C03DA4FF0010B15
:10BC1000604204B2002517E0424629462046FFF75D
:10BC2000D1FF8146BBF1000F03D0A8EB090000F063
:10BC3000FF09701901B2CDF800903A4650460A9BB0
:10BC400000F078F8681C05B2A542E5DBBDE8F88F86
:10BC50002DE9F84F06468A4614461F46DDF82C802B
:10BC60004FF0000B002C03DA4FF0010B604204B2DE
:10BC7000002517E0424629462046FFF7A3FF8146EC
:10BC8000BBF1000F03D0A8EB090000F0FF09711908
:10BC900008B2CDF800903A4651460A9B00F04AF8A7
:10BCA000681C05B2A542E5DBBDE8F88F0401002061
:10BCB000A00100200801002007B581B0BDF80800F0
:10BCC000C00AC2F1FF014843BDF80410C90A01FBD4
:10BCD0000200010ABDF8000061F3CF200090BDF81A
:10BCE0000800C0F34510C2F1FF014843BDF804103D
:10BCF000C1F3451101FB0200010ABDF8000061F328
:10BD00004A100090BDF8080000F01F00C2F1FF01CA
:10BD10004843BDF8041001F01F0101FB0200010AB5
:10BD2000BDF8000061F304000090BDF80010084663
:10BD300004B000BD2DE9FF4F83B004460D46174601
:10BD4000DDF84080B8F1100F02DA07B0BDE8F08FDF
:10BD5000B8F1FB0F01DD4FF0FF08B7F90000A0427A
:10BD60000BDCB7F90400A04207DBB7F90200A842D8
:10BD700003DCB7F90600A84200DAE6E7FEF7ADFDFE
:10BD80008146484605F014FA064606F1100000F018
:10BD90008EFC8246308A201A04B2708A281A05B2B4
:10BDA000D9F8140078B1CDF80880BDF81800ADF8C6
:10BDB00004000095B16823460FFA8AF24846D9F884
:10BDC00014C0E0471FE000200290D6F808B005FB41
:10BDD0000A400BEB400B0298A0B9B8F1FF0F04D159
:10BDE000BDF81800ABF800000CE0BBF800004246BC
:10BDF000014600900698FFF75FFF0190BDF8040030
:10BE0000ABF8000000BF00BF9FE72DE9FF4F83B0F4
:10BE1000064688461446DDF84090FEF75EFD8246F1
:10BE2000DAF8140000B3B4F9005018E0B4F9027065
:10BE30000FE0CDF80890BDF81800ADF804000097A9
:10BE40002B46424631465046DAF814C0E047781C8B
:10BE500007B2B4F90600B842EBDA681C05B2B4F9CF
:10BE60000400A842E2DA71E0B4F9020000FB08F035
:10BE700006EB4006B9F1FF0F2FD1B4F9005006E0F0
:10BE800006EB4500BDF818100180681C05B2B4F936
:10BE90000400A842F4DAB4F9000006EB400BA088D5
:10BEA0002188401A401C400000B2029006EB480670
:10BEB0006088401C07B20BE0B4F9001006EB4100AB
:10BEC0005946029A11F025FD06EB4806781C07B288
:10BED000B4F90600B842EFDA38E04FF0000B00206A
:10BEE0000290029801904A4601990698FFF7E4FEF5
:10BEF0000090B4F9027024E0B4F9005019E0BBF1ED
:10BF0000000F14D136F81500BDF80410884209D08E
:10BF100006EB4500008801904A4601990698FFF714
:10BF2000CBFE009006EB4500BDF800100180681CB8
:10BF300005B2B4F90400A842E1DA06EB4806781C21
:10BF400007B2B4F90600B842D6DA00BF07B0BDE8C0
:10BF5000F08F2DE9FF4F85B0804689461D46102D94
:10BF600002DA09B0BDE8F08FFB2D00DDFF254A465F
:10BF7000414603A805F0CEFC074607B9F1E7FEF7F6
:10BF8000ACFC8346584605F013F90446BDF80C0096
:10BF9000218A401A00B2ADF80400BDF80E10608A84
:10BFA000081A00B2ADF80600BDF81000218A401A48
:10BFB00000B2ADF80800BDF81210608A081A00B28D
:10BFC000ADF80A00D4F808A004F1100000F06FFBEF
:10BFD0000646BDF8060010FB06F00AEB400A009585
:10BFE000A06801AA3146079BFFF70FFF00BFB8E723
:10BFF0002DE9FF4F9DB00C46FEA000681C90FEA0EE
:10C0000000681B90FDA30FCB17AD0FC52B98102810
:10C0100002DA21B0BDE8F08F2B98FB2801DDFF206C
:10C020002B901F9800B9F4E7002315A9DDE91F0242
:10C03000F9F7AAFF1490149800B9EAE71D98008850
:10C040009DF95810084405B21F98017A407A091AE0
:10C050001D98408808449DF85710401A9DF95910C2
:10C06000401A06B29DF85A00012806D0022809D0CD
:10C0700004280CD0082814D10EE00DF1700B80209C
:10C0800013900FE00DF16C0BC02013900AE00DF13E
:10C090005C0BF020139005E04FF0000BFF20139095
:10C0A00000E0B6E700BFDDE91F01F9F765FF824652
:10C0B000BAF1000F00D1ACE79DF856002844B4F95E
:10C0C000001088420EDBB4F90400A8420ADB9DF898
:10C0D00057003044B4F90210884203DBB4F906007B
:10C0E000B04200DA95E7FEF7F8FB1190119805F0E1
:10C0F0005FF8804608F1100000F0D9FA1090D8F8E7
:10C1000008709DF85600C0100D909DF8560000F084
:10C11000070018B10D98401CC0B20D909DF8560054
:10C120009DF85A1010FB01F00C90B4F90000A842E1
:10C1300001DC002002E0B4F90000401B00B20B90CB
:10C140009DF856002844B4F90410884202DC9DF89A
:10C15000560003E0B4F90400401B401C00B20A90F2
:10C16000B4F90200B04201DC002002E0B4F90200A0
:10C17000801B00B209909DF857003044B4F90610B6
:10C18000884202DC9DF8570003E0B4F90600801BEA
:10C19000401C00B20890B8F91200311A109801FB47
:10C1A0000050B8F91010401A07EB4007109A0B998D
:10C1B000099800FB021007EB40070C9909984843C7
:10C1C0009DF85A200B9901FB0200079007980AEB93
:10C1D000D00A079800F007090020049009980E90F3
:10C1E000A7E0139840FA09F012900B980F9080E0A6
:10C1F000C9F108009DF85A10421A9AF800001299E5
:10C200000840104106900698D0B32B98FF280AD119
:10C210009DF85A00082801D1069802E006981BF8FC
:10C22000000005900FE09DF85A00082804D12B99D2
:10C2300006984843001205E006981BF800002B9969
:10C2400048430012059011984069D0B105980290BA
:10C25000BDF8A800ADF804000E988119B8F81200D6
:10C26000081A00B200900F982844B8F81020801ADD
:10C2700003B2D8F808101198D0F814C0109AE0470B
:10C280001BE03888BDF8A810884216D00598FB2816
:10C2900003DDBDF8A80038800FE0059810280CDDFC
:10C2A000049850B9388802900146059A2A98FFF7F9
:10C2B00003FD0390BDF80C003880BF1C9DF85A00A8
:10C2C000C0F1080048450ADD9DF85A0048441FFAAD
:10C2D00080F99DF85A1012980841129005E04FF02D
:10C2E0000009139812900AF1010A0F98401C00B23D
:10C2F0000F900A990F988842FFF67AAF9DF8561072
:10C300000A98091A0B9808449DF85A1000FB0190EE
:10C310001FFA80F90AEBE90A09F00709DDE90A01C9
:10C32000411A1098401A07EB40070E98401C00B2C3
:10C330000E9008990E988842FFF653AF00BF68E64A
:10C340002DE9FE430546884616461F46FF2F05D1B8
:10C3500072004146284611F0DCFA17E0002412E092
:10C3600005EB44000088019008EB440000883A4641
:10C3700000900199FFF7A0FC029005EB4400BDF886
:10C3800008100180641CB442EAD300BFBDE8FE83FC
:10C390002DE9FF4F8FB090461298102802DA13B0A3
:10C3A000BDE8F08F1298FB2801DDFF2012900DA848
:10C3B000DDE90F1205F0AEFA0C900C9800B9EEE72B
:10C3C0001D9808B1032000E0022082460F9800F07B
:10C3D0006EF90B900F98B0F90200BDF93610884243
:10C3E00016DABDF936100F98B0F90200081A0B9949
:10C3F00048430BE000FF00000055AAFF0011223364
:10C40000445566778899AABBCCDDEEFF00FB0A880D
:10C410000F98B0F90000BDF93410884207DABDF971
:10C4200034100F98B0F90000081A00FB0A88FEF7D4
:10C4300054FA8146484604F0BBFE0746BDF8340076
:10C44000398A401A00B2ADF83400BDF83610788A47
:10C45000081A00B2ADF83600BDF83800398A401A23
:10C4600000B2ADF83800BDF83A10788A081A00B268
:10C47000ADF83A0007F1100000F019F90A90BD6814
:10C48000BDF836100A9811FB00F005EB4005BDF928
:10C49000340005EB40050DA800F009F909900020D3
:10C4A00008901C9800284AD11D98002847D112985E
:10C4B000FF2844D11F98002841D1D9F8140040B377
:10C4C000BDF9364020E0002616E006FB0A80008811
:10C4D000079012980290BDF81C00ADF8040000947B
:10C4E000BDF83400304403B2B968D9F814C04846E6
:10C4F0000A9AE047701C06B209988642E5DB0B9861
:10C5000000FB0A88601C04B2BDF93A00A042DADAE6
:10C51000CBE0BDF936400DE041462846129B099A12
:10C52000FFF70EFF0B9800FB0A880A9805EB400501
:10C53000601C04B2BDF93A00A042EDDAB5E000207B
:10C54000079007980690DDE91E020699FFF7B4FBF5
:10C550000590BDF93640A2E0002694E0DDF848B031
:10C5600006FB0A8004901D9888B104990A784978DE
:10C5700002EB012189B203910499887800B980E027
:10C58000FF2803D000FB0BF14FEA112B02E00498C7
:10C59000008803901C9830B1BDF80C00B9F81C104D
:10C5A000884200D16DE01F98D0B3BDF81800BDF8E7
:10C5B0000C10884207D003980690DDE91E02069908
:10C5C000FFF77AFB0590D9F8140088B1CDF808B0D0
:10C5D000BDF81400ADF804000094BDF834003044F8
:10C5E00003B2B968D9F814C048460A9AE04747E050
:10C5F000BBF1FF0F04D1BDF8140025F816003FE091
:10C6000005EB460000885A46014601900598FFF761
:10C6100053FB029005EB4600BDF8081001802FE0A7
:10C62000FFE7D9F8140088B1CDF808B0BDF80C00C8
:10C63000ADF804000094BDF83400304403B2B9688A
:10C64000D9F814C048460A9AE04719E0BBF1FF0F39
:10C6500005D105EB4600BDF80C10018010E00898EC
:10C6600070B905EB460000885A46014601900398D0
:10C67000FFF722FB029005EB4600BDF80810018091
:10C6800000BF701C06B209988642FFF667AF0B9890
:10C6900000FB0A880A9805EB4005601C04B2BDF94E
:10C6A0003A00A042BFF658AF00BF00BF77E6014690
:10C6B00088880A88801A401C00B270470146002012
:10C6C0000C290FD006DC02290AD0052907D00B2936
:10C6D0000CD106E00D2906D00E2907D104E000BFD9
:10C6E00000BF00BF00BF00BF012001E0002000BF6D
:10C6F00000BF704701460020CA1E082A0CD2DFE89E
:10C7000002F0050B0B040607080900BF00BF00BFBD
:10C7100000BF00BF012001E0002000BF00BF704744
:10C720002DE9FF4F8FB0064692461D46DDF870B0EA
:10C7300032460DA8109905F0EDF80C900C9818B938
:10C74000012013B0BDE8F08FBBF1FF0F02D1332001
:10C75000405D04E03320405D00FB0BF000120B90C5
:10C760002946504603F08CFD04460CB90020E8E74A
:10C77000217C01F01F00FFF7BDFF8046217C01F006
:10C780001F00FFF79BFF0746E069B8B1FF23FD4A92
:10C790003046109903F018FD00204FF6FF71CDE9E7
:10C7A0000201CDE904100146E069FF23F54ACDE915
:10C7B00000013046109900F053FC6FE0606970B1E1
:10C7C0003220405D0390288EADF80800CDE9008747
:10C7D000626930460B9B1099FFF7DAFD5EE00DA809
:10C7E00000F00FFC0A900DA800F00BFC00EB4000DD
:10C7F0000390FFF7AFF9099007A80D9901600E9912
:10C80000416000BF012105F051F8BDF834003188C6
:10C81000401A00B20690BDF836007188401A00B286
:10C820000590BDF93600049032E00998009020464A
:10C830000A9BDDE9052104F0A5F98146B9F1010F54
:10C8400004D0204604F0B8F900207AE73220405D99
:10C850000390288EADF80800CDE9008707A80B9B50
:10C86000099A1099FFF794FDBDF81E00401C00B214
:10C87000ADF81E00BDF82200401C00B2ADF8220049
:10C880000598401C00B205900498401C00B204902A
:10C89000BDF93A1004988142C7DA00BF012050E781
:10C8A0002DE9F04387B006460F4615469846DDF859
:10C8B0003890C5B9FF23B34A3946304603F084FCAB
:10C8C00000204FF6FF71CDE90201CDE90410AEA1C1
:10C8D000FF23AC4ACDE900103946304600F0C0FBDA
:10C8E00007B0BDE8F08343462A4639463046CDF8C6
:10C8F0000090FFF715FF0446B4B9FF23A14A39465B
:10C90000304603F061FC00204FF6FF71CDE90201D3
:10C91000CDE904109CA1FF239A4ACDE900103946C5
:10C92000304600F09DFBDBE700BFD9E70146002061
:10C930000F291DD2DFE801F008091C1C0B0E0C109A
:10C940001316191114171A0000BF002012E000BFBF
:10C9500010200FE018200DE000BF01200AE000BF0A
:10C96000022007E000BF042004E000BF082001E02F
:10C97000002000BF00BF70472DE9FE4304460D466E
:10C9800016461F4600200290029801902068C0F3CE
:10C990008A20A84204DC2068C0F38A20451E02E0F9
:10C9A000002D00DA00252068B6EB505F04DB012182
:10C9B0002068C1EB505602E0002E00DA0026A36882
:10C9C000207800F01F00042809D0207800F01F0014
:10C9D000062804D0207800F01F00052813D1217804
:10C9E00001F01F00FFF7A2FF4FEAE0082068C0F344
:10C9F0008A20704300FB08F005FB080903EB0900DF
:10CA00000088019088E0207800F01F00072819D1E5
:10CA1000083305F00700ED102268C2F38A22D21D08
:10CA2000D21002FB06515A5CC0F107084FF0010C0E
:10CA30000CFA08FC02EA0C02C0F1070C42FA0CF2F4
:10CA4000019269E0207800F01F00082819D1103306
:10CA5000AA07500FAD102268C2F38A22D21C92108E
:10CA600002FB06515A5CC0F106084FF0030C0CFAA9
:10CA700008FC02EA0C02C0F1060C42FA0CF2019228
:10CA80004AE0207800F01F00092819D14033EA0756
:10CA9000500F6D102268C2F38A22521C521002FB02
:10CAA00006515A5CC0F104084FF00F0C0CFA08FC58
:10CAB00002EA0C02C0F1040C42FA0CF201922BE0E3
:10CAC000207800F01F000A2809D103F5806321684F
:10CAD000C1F38A2101FB0650195C01911CE020780A
:10CAE00000F01F000B280ED0207800F01F000C284B
:10CAF00009D0207800F01F000D2804D0207800F025
:10CB00001F000E2808D117B1388E019004E00020D4
:10CB100000900098019000BFBDF804100846BDE8E1
:10CB2000FE832DE9FF4303461868C0F38A2088423C
:10CB300004DC1868C0F38A20411E02E0002900DAF4
:10CB400000211868B2EB505F04DB01251868C5EBC3
:10CB5000505202E0002A00DA00229C68187800F0A7
:10CB60001F00052814D11868C0F38A20504300EB39
:10CB7000400001EB41068519A81C205C04B0BDE80B
:10CB8000F08300005C2C00204E6F0A646174610029
:10CB9000187800F01F000B281BD101F00705C91001
:10CBA0001868C0F38A20C01DC01000FB0216A05DEB
:10CBB000C5F107084FF0010C0CFA08FC00EA0C0064
:10CBC000C5F1070C40FA0CF70FB10020D6E7FF20A3
:10CBD000D4E7187800F01F000C281CD1F9A00068D9
:10CBE00003908807450F89101868C0F38A20C01C7D
:10CBF000801000FB0216A05DC5F106084FF0030C83
:10CC00000CFA08FC00EA0C00C5F1060C40FA0CF71F
:10CC100003A8C05DB2E7187800F01F000D2826D1E8
:10CC20000FF2A439D9E901C8D9F80000D9F80C905D
:10CC3000CDE901C8CDF80C900090C807450F491008
:10CC40001868C0F38A20401C401000FB0216A05D4B
:10CC5000C5F104084FF00F0C0CFA08FC00EA0C00B8
:10CC6000C5F1040C40FA0CF71DF8070086E71878A8
:10CC700000F01F000E2806D11868C0F38A2000FBC0
:10CC80000215605D7AE700BFFF2077E72DE9FF47D7
:10CC900005460E461746AC68287800F01F000428A9
:10CCA00004D0287800F01F00062815D1297801F05B
:10CCB0001F00FFF73BFE4FEAE0082868C0F38A2018
:10CCC000784300FB08F006FB080904EB0900424624
:10CCD00003A910F01EFE94E0287800F01F0005283C
:10CCE00016D1297801F01F00FFF720FE4FEAE00877
:10CCF0002868C0F38A20784300FB08F006FB080987
:10CD0000A8F1010204EB090003A910F002FE78E08B
:10CD1000287800F01F0007281DD1083406F007010D
:10CD2000F6102A68C2F38A22D21DD21002FB0760D5
:10CD3000225CC1F1070C012303FA0CF39A4322543D
:10CD4000BDF80C2002F00102C1F107039A40235CF8
:10CD50001A43225455E0287800F01F0008281DD1FE
:10CD60001034B207510FB6102A68C2F38A22D21CBF
:10CD7000921002FB0760225CC1F1060C032303FA48
:10CD80000CF39A432254BDF80C2002F00302C1F1C7
:10CD900006039A40235C1A43225432E0287800F0BC
:10CDA0001F0009281DD14034F207510F76102A6860
:10CDB000C2F38A22521C521002FB0760225CC1F1AE
:10CDC000040C0F2303FA0CF39A432254BDF80C20F1
:10CDD00002F00F02C1F104039A40235C1A4322546B
:10CDE0000FE0287800F01F000A280AD104F58064BB
:10CDF0002968C1F38A2101FB0760BDF80C1021549A
:10CE000000BFBDE8FF872DE9F04304460D461746F5
:10CE10001E46A368207800F01F00052813D1217852
:10CE200001F01F00FFF782FD4FEAE0082068C0F321
:10CE30008A20784300FB08F005FB080909EB08008D
:10CE4000401E1E547DE0207800F01F000B2820D1EA
:10CE5000F61105F00701ED102268C2F38A22D21DF7
:10CE6000D21002FB07501A5CC1F107084FF0010C09
:10CE70000CFA08FC22EA0C021A5406F00102C1F175
:10CE8000070C02FA0CF213F800C042EA0C021A5422
:10CE900057E0207800F01F000C2820D1B611AA0717
:10CEA000510FAD102268C2F38A22D21C921002FBED
:10CEB00007501A5CC1F106084FF0030C0CFA08FC8D
:10CEC00022EA0C021A5406F00302C1F1060C02FA1F
:10CED0000CF213F800C042EA0C021A5431E0207838
:10CEE00000F01F000D2820D13611EA07510F6D10F8
:10CEF0002268C2F38A22521C521002FB07501A5CAD
:10CF0000C1F104084FF00F0C0CFA08FC22EA0C02E5
:10CF10001A5406F00F02C1F1040C02FA0CF213F8D5
:10CF200000C042EA0C021A540BE0207800F01F0007
:10CF30000E2806D12168C1F38A2101FB07501E5437
:10CF400000BFBDE8F08317B583B0037803F01F037B
:10CF50000B2B01D1012912DC037803F01F030C2BEA
:10CF600001D103290BDC037803F01F030D2B01D142
:10CF70000F2904DC037803F01F030E2B01D106B048
:10CF800010BD059B0193BDF80430DB0ADB008DF872
:10CF90000230BDF80430C3F345139B008DF8013017
:10CFA000BDF80430DB061B0E8DF80030FF238DF832
:10CFB0000330009B0293826802EB8103029C1C6099
:10CFC00000BFDCE70055AAFF001122334455667705
:10CFD0008899AABBCCDDEEFF0146032001B970475A
:10CFE0000A461378202B04DB13787F2B01DC012009
:10CFF00005E01378802B01DB022000E0002000BF59
:10D00000EDE7014688880A88801A401C00B2704704
:10D0100001460020302905DB392903DCA1F130026B
:10D02000D0B21CE0612902DBA1F12002D1B2A1F152
:10D030004102062A10D2DFE802F0030507090B0DB2
:10D040000A200BE00B2009E00C2007E00D2005E092
:10D050000E2003E00F2001E0002000BF00BF70475A
:10D060002DE9FF4FA7B082461446DDF8E480DDE9E4
:10D070003476606A269006F0020020B9504600F02F
:10D080005AFA259010E047F61841B4F92A008DE8C5
:10D090004300B4F92830394609A8626A05F09FFCBC
:10D0A000BDF92400259000BF00BF2698007A618D4D
:10D0B000084400B2249000202390BAF80000ADF894
:10D0C0008800BAF80200ADF88A0000202190209074
:10D0D000369870B13698B0F9000021903698B0F9C2
:10D0E00002002090BDF88A102098084400B2ADF8E4
:10D0F0008A000025681E1F90B8F1000F24D02098E8
:10D1000010BBBAF9020000281EDABAF90210D8F8EA
:10D110000800401A002805DDBAF90210D8F8080006
:10D12000401A04E0BAF90200D8F80810401A24990D
:10D130004900C1F58061884203DD4FF0FF30C8F837
:10D140000000D8F800001F90B8F1000F0BD01F9816
:10D15000002808DB1F9DBDF88A00B8F804100844B9
:10D1600000B2ADF88A000096B4F928207819DDE9FC
:10D17000253105F0ACFB00EB05092EE04D4600968D
:10D18000B4F928207819DDE9253105F0A0FB8144A8
:10D19000BDF88A102498084400B2ADF88A00B8F1AE
:10D1A000000F15D0BDF98A0010F5806F10DBD8F89C
:10D1B000000000280CDAC8F80050BDF98A00BAF95E
:10D1C0000210401AC8F80400BAF90200C8F80800B2
:10D1D000785D10B92BB0BDE8F08FBDF98A102498A6
:10D1E00001442898B0F902008142C7DB06F0040030
:10D1F000D0B10096B4F92830A9EB050291B27819A4
:10D20000269A05F01EFB2390504600F094F92399CE
:10D21000A0EB010B0BEBDB70BDF8881001EB60009D
:10D2200000B2ADF8880018E006F00800A8B100963A
:10D23000B4F92830A9EB050291B27819269A05F0C5
:10D2400000FB2390504600F076F92399401ABDF870
:10D250008810084400B2ADF888002A98FF2802D14F
:10D260002C20005D04E02C20005D2A994843001228
:10D270001E9000201D901B90B2490AA8FDF77AFF6E
:10D28000608CADF82A000AA8BDF82A10ADF82C1061
:10D290004BE1369830B1BDF888102198084400B2AF
:10D2A000ADF8880000201D901C95E5E01CA93846CB
:10D2B000A54A1268904709901C9978180021A24A43
:10D2C00012689047089006F00100002877D09FA0D0
:10D2D00001780998814213D11D9828B91C9880B211
:10D2E0001B9001201D90C7E01D98012802D100204D
:10D2F0001D9005E01D98022802D100201D90BBE082
:10D300001D9801285BD10998202857D1DDE91B0120
:10D31000081A07284ED11B98384401680591808867
:10D32000ADF8180000208DF81A009DF81500FFF7E1
:10D330006FFE83469DF81400FFF76AFE0BEB0010AA
:10D3400004909DF81700FFF763FE83469DF81600D2
:10D35000FFF75EFE0BEB001003909DF81900FFF73E
:10D3600057FE83469DF81800FFF752FE0BEB0010A6
:10D370000290049BD8B2039BD9B2029BDAB24FEA67
:10D38000D20CBDF804306CF3040301934FEA910C06
:10D39000BDF804306CF34A1301934FEAD00CBDF88A
:10D3A00004306CF3CF230193BDF804C063461A9395
:10D3B00002E004E0208C1A9002201D905CE0206ABC
:10D3C00007901D98022801D11A980790DDE90821DD
:10D3D0002698F8F7E8FD00B219904FF6FF713798DC
:10D3E000884230D0389888422DD03846584A1C9907
:10D3F0001268904783463798834523DD38988345E4
:10D4000020DCBDF88800ADF81400BDF88A00ADF846
:10D410001600BDF8881019980144208D0844401E5C
:10D4200000B2ADF81800BDF88A1024980844401ED8
:10D4300000B2ADF81A000AAA05A81E9B289902F0AE
:10D44000C3FE00BF00BF1E980190BDF81C00ADF8E0
:10D45000000022A8099B269A2899FEF7C9FD199871
:10D46000002808DDBDF88810228D19981044084462
:10D4700000B2ADF8880000BF1C984845FFF416AF15
:10D480004D460096B4F928207819DDE9253105F0DC
:10D490001EFA8144BAF80000ADF8880006F00400D6
:10D4A000D0B10096B4F92830A9EB050291B27819F1
:10D4B000269A05F0C6F92390504600F03CF82399CF
:10D4C000A0EB010B0BEBDB70BDF8881001EB6000EB
:10D4D00000B2ADF8880018E006F00800A8B1009688
:10D4E000B4F92830A9EB050291B27819269A05F013
:10D4F000A8F92390504600F01EF82399401ABDF871
:10D500008810084400B2ADF88800BDF88A1024984D
:10D51000084400B2ADF88A00BDF98A102898B0F925
:10D520000600814200DD55E600BF785D00287FF4EB
:10D53000B0AE00BF4EE6014688880A88801A401CBB
:10D5400000B27047982C0020CC010020230000007E
:10D55000D801002007B581B0BDF80800C00AC2F1AB
:10D56000FF014843BDF80410C90A01FB0200010A8B
:10D57000BDF8000061F3CF200090BDF80800C0F3B3
:10D580004510C2F1FF014843BDF80410C1F3451135
:10D5900001FB0200010ABDF8000061F34A1000908F
:10D5A000BDF8080000F01F00C2F1FF014843BDF8BC
:10D5B000041001F01F0101FB0200010ABDF8000088
:10D5C00061F304000090BDF80010084604B000BDEF
:10D5D00030B50346022B04D1FE48405C5043001294
:10D5E00030BD032B04D1FC48405C50430012F7E7E8
:10D5F000042B04D1F948405C50430012F0E7C1EB22
:10D60000C105581EB5FBF0F0C4B2F548005D5043AB
:10D61000000AE5E72DE9F04104460D461646FDF700
:10D620005CF9804603F0A4FD0746B4EB650F04DB0C
:10D63000C5F34F040CB1601E84B2B4EB660F04DB7B
:10D64000C6F34F040CB1601E84B2002C01DDE01B58
:10D6500084B22046BDE8F0810FB5A3B02598C088FC
:10D6600080B22290FDF739F9079003F081FD2190F7
:10D670002598B0F90C002090259840891F90259896
:10D68000807B1E902698FF2802D12598C07B04E05D
:10D690002598C07B2699484300121D902098401E73
:10D6A00000B22090219818B12098401E00B220901E
:10D6B000239802F0D6FD1C90239802F0D9FD1B9010
:10D6C000DDE91B212298FFF7A5FF2290239801880E
:10D6D000229801442198084400B2ADF868002398CC
:10D6E0004188229801442198084400B2ADF86A00AC
:10D6F00023980188229801442198084400B2ADF88B
:10D7000064002398C1882298091A2198081A00B247
:10D71000ADF86600239881882298091A2198081A82
:10D7200000B2ADF860002398418822980144219806
:10D73000084400B2ADF86200239881882298091A43
:10D740002198081A00B2ADF85C002398C18822988D
:10D75000091A2198081A00B2ADF85E00229802B2A8
:10D7600015A916A804F0CEF920992298401A00B203
:10D7700012901298002801DA0020129013A914A820
:10D78000129A04F0BFF900200D900C90229800B27C
:10D790000B9000200A90099020992298401A00B21C
:10D7A0000890FDE3BDF95200BDF95010884209DA36
:10D7B000BDF85800BDF85010401A00B20F900F98F5
:10D7C0000E900AE0BDF85800BDF85A10401A00B299
:10D7D0000F900F98401E00B20E90219800287DD027
:10D7E000BDF958100B98814279D0BDF95A000C90C0
:10D7F000DDE90C01401A00B207900B98ADF8180053
:10D800000D98ADF81A00002005902EE10798012828
:10D8100006DD1D9A05990798FFF7DAFE049008E0E7
:10D820001D9A05990798FEF7CDF91D99081AC0B2FF
:10D8300004901E9800F00100D8B31E9800F0080074
:10D84000B8B304980090BDF85E00BDF81A1001440A
:10D850000598084400B20290BDF85C00BDF81810AD
:10D860000844401C00B2019025984089034603906B
:10D87000249ADDE90101FEF75DFA04980090BDF8F5
:10D880005E00BDF818100844401C00B20290BDF8BC
:10D890005C00BDF81A1001440598084400B20190DC
:10D8A0002598408903460390249ADDE90101FEF79B
:10D8B00041FA1E9800F00100E8B31E9800F0040041
:10D8C000C8B304980090BDF86600BDF8181008446D
:10D8D000401C00B20290BDF8640001E054E1CFE0CA
:10D8E000BDF81A10494201440598081A00B2019087
:10D8F0002598408903460390249ADDE90101FEF74B
:10D9000019FA04980090BDF86600BDF81A10014499
:10D910000598084400B20290BDF86400BDF81810E4
:10D9200049420844401E00B20190259840890346B0
:10D930000390249A00E003E0DDE90101FEF7FAF923
:10D940001E9800F00200E0B31E9800F00400C0B37F
:10D9500004980090BDF86A00BDF81A1049420144CD
:10D960000598081A00B20290BDF86800BDF81810BA
:10D9700049420844401E00B2019025984089034660
:10D980000390249ADDE90101FEF7D4F90498009090
:10D99000BDF86A00BDF8181049420844401E00B2A4
:10D9A0000290BDF86800BDF81A104942014405987C
:10D9B000081A00B201902598408903460390249AE2
:10D9C00000E003E0DDE90101FEF7B4F91E9800F084
:10D9D000020007E07A0802087C0802087F080208B3
:10D9E00083080208E8B31E9800F00800C8B3049842
:10D9F0000090BDF86200BDF8181049420844401E6E
:10DA000000B20290BDF86000BDF81A1001440598FC
:10DA1000084400B201902598408903460390249A57
:10DA2000DDE90101FEF786F904980090BDF8620077
:10DA3000BDF81A10494201440598081A00B2029034
:10DA4000BDF86000BDF818100844401C00B20190F9
:10DA50002598408903460390249ADDE90101FEF7E9
:10DA600069F90598401C00B205900799059888420D
:10DA7000FFF6CCAEBDF958000B900C980D9000BF8E
:10DA8000BDF95010089881427ED0BDF95A00099026
:10DA9000DDE90901401A00B207900898ADF81800B6
:10DAA0000A98ADF81A00002005904BE1079801286C
:10DAB00009DD1D9A05990798FFF78AFD1D99081A37
:10DAC000C0B2049005E01D9A05990798FEF77AF810
:10DAD00004901E9800F00100F8B11E9800F00800B4
:10DAE000D8B104980090BDF85E00BDF81A1001444A
:10DAF0000598084400B20290BDF85C00BDF818100B
:10DB00000844401E00B201902598408903460390C6
:10DB1000249ADDE90101FEF70DF91E9800F00100DD
:10DB200000B31E9800F00400E0B104980090BDF826
:10DB30006600BDF818100844401E00B20290BDF8FF
:10DB40006400BDF81A10494201440598081A00B251
:10DB500001902598408903460390249ADDE901014C
:10DB6000FEF7E8F81E9800F0020018B31E9800F0C7
:10DB70000400F8B104980090BDF86A00BDF81A10CE
:10DB800049420144059800E0E7E0081A00B202901B
:10DB9000BDF86800BDF8181049420844401C00B2A6
:10DBA00001902598408903460390249ADDE90101FC
:10DBB000FEF7C0F81E9800F0020000B31E9800F0B7
:10DBC0000800E0B104980090BDF86200BDF818109C
:10DBD00049420844401C00B20290BDF86000BDF804
:10DBE0001A1001440598084400B201902598408914
:10DBF00003460390249ADDE90101FEF79BF8BDF985
:10DC00001800401EBDF91A200599114488427DD0A4
:10DC10001E9800F00100F8B11E9800F00800D8B17D
:10DC200004980090BDF85E00BDF818100844401E2E
:10DC300000B20290BDF85C00BDF81A1001440598CE
:10DC4000084400B201902598408903460390249A25
:10DC5000DDE90101FEF76EF81E9800F0010000B347
:10DC60001E9800F00400E0B104980090BDF8660032
:10DC7000BDF81A1001440598084400B20290BDF89E
:10DC80006400BDF8181049420844401C00B20190DD
:10DC90002598408903460390249ADDE90101FEF7A7
:10DCA00049F81E9800F0020008B31E9800F0040026
:10DCB000E8B104980090BDF86A00BDF81810494218
:10DCC0000844401C00B20290BDF86800BDF81A106C
:10DCD000494201440598081A00B2019025984089EC
:10DCE00003460390249ADDE90101FEF723F81E980C
:10DCF00000F0020050B11E9800F0080030B1049806
:10DD00000090BDF86200BDF81A1000E016E049422C
:10DD100001440598081A00B20290BDF86000BDF8F1
:10DD200018100844401E00B201902598408903460F
:10DD30000390249ADDE90101FDF7FCFF0598401CE2
:10DD400000B20590079905988842FFF6AFAEBDF97D
:10DD50005000089009980A9000BF1E9800F001003A
:10DD6000F0B31E9800F00800D0B3BDF85C00BDF819
:10DD7000581001440E98081A00B2ADF84000BDF8E2
:10DD80005C00BDF85810084400B2ADF84400BDF87E
:10DD90005E00BDF85A10084400B2ADF84200BDF86C
:10DDA0005E00BDF85A10084400B2ADF8460010A855
:10DDB0001D9B1F9A2499FEF7CCF8BDF85C00BDF8B6
:10DDC0005A10084400B2ADF84000BDF85C00BDF840
:10DDD0005A10084400B2ADF84400BDF85E0000E0FF
:10DDE00015E0BDF8581001440F98081A00B2ADF8BC
:10DDF0004200BDF85E00BDF85810084400B2ADF80E
:10DE0000460010A81D9B1F9A2499FEF7A2F81E98A1
:10DE100000F00100F0B31E9800F00400D0B3BDF88C
:10DE20006400BDF85A104942084400B2ADF8400001
:10DE3000BDF86400BDF85A104942084400B2ADF87C
:10DE40004400BDF86600BDF8581001440E98081A49
:10DE500000B2ADF84200BDF86600BDF858100844A5
:10DE600000B2ADF8460010A81D9B1F9A2499FEF73A
:10DE700070F8BDF86400BDF858104942084400B27B
:10DE8000ADF84000BDF86400BDF8581049420144A7
:10DE90000F9800E019E0084400B2ADF84400BDF866
:10DEA0006600BDF85A10084400B2ADF84200BDF853
:10DEB0006600BDF85A10084400B2ADF8460010A83C
:10DEC0001D9B1F9A2499FEF744F81E9800F002004B
:10DED000E8B31E9800F00400C8B3BDF96600BDF9B0
:10DEE0005A100844BDF96A10BDF95A205242114433
:10DEF00088422BDDBDF86800BDF85810494208443F
:10DF000000B2ADF84000BDF86800BDF858104942B5
:10DF100001440E98084400B2ADF84400BDF86A0010
:10DF2000BDF85A104942084400B2ADF84200BDF8AD
:10DF30006A00BDF85A104942084400B2ADF84600E4
:10DF400010A81D9B1F9A2499FEF703F800E02DE00E
:10DF5000BDF86800BDF85A104942084400B2ADF857
:10DF60004000BDF86800BDF85A104942084400B2AC
:10DF7000ADF84400BDF86A00BDF8581049420844A5
:10DF800000B2ADF84200BDF86A00BDF85810494231
:10DF900001440F98084400B2ADF8460010A800E014
:10DFA0007DE01D9B1F9A2499FDF7D3FF1E9800F07A
:10DFB0000200E8B31E9800F00800C8B3BDF8600086
:10DFC000BDF85A10084400B2ADF84000BDF860003A
:10DFD000BDF85A10084400B2ADF84400BDF8620024
:10DFE000BDF858104942084400B2ADF84200BDF8EF
:10DFF0006200BDF85810494201440E98084400B22E
:10E00000ADF8460010A81D9B1F9A2499FDF7A1FFAB
:10E01000BDF95E00BDF95A100844BDF96210BDF9A2
:10E020005A205242114488422BDDBDF8600000E0C6
:10E0300027E0BDF8581001440F98081A00B2ADF857
:10E040004000BDF86000BDF85810084400B2ADF8BB
:10E050004400BDF86200BDF85A104942084400B2BD
:10E06000ADF84200BDF86200BDF85A1049420844BC
:10E0700000B2ADF8460010A81D9B1F9A2499FDF729
:10E0800068FF15A916A803F050FDBDF95200BDF9AF
:10E090005010884203DA13A914A803F046FDBDF915
:10E0A0005A00BDF9581088427FF77CAB21980028B0
:10E0B0007DD0BDF95A000C90DDE90C01401A00B288
:10E0C00007900B98ADF818000D98ADF81A000020D5
:10E0D00005901AE11D9A05990798FDF773FD1D99A2
:10E0E000081AC0B204901E9800F00100D8B31E9820
:10E0F00000F00800B8B304980090BDF85E00BDF8C9
:10E100001A1001440598084400B20290BDF85C0062
:10E11000BDF818100844401C00B2019025984089B1
:10E1200003460390249ADDE90101FDF703FE0498FC
:10E130000090BDF85E00BDF818100844401C00B205
:10E140000290BDF85C00BDF81A100144059808441F
:10E1500000B201902598408903460390249ADDE996
:10E160000101FDF7E7FD1E9800F00100F0B31E98D5
:10E1700000F00400D0B304980090BDF86600BDF82C
:10E1800018100844401C00B20290BDF86400BDF8AD
:10E190001A10494201440598081A00B201902598C6
:10E1A000408903460390249ADDE9010100E0AEE2D4
:10E1B000FDF7C0FD04980090BDF86600BDF81A1088
:10E1C00001440598084400B20290BDF86400BDF80F
:10E1D000181049420844401E00B201902598408919
:10E1E00003460390249ADDE9010100E001E0FDF718
:10E1F000A1FD1E9800F00200F0B31E9800F004008C
:10E20000D0B304980090BDF86A00BDF81A104942D6
:10E2100001440598081A00B20290BDF86800BDF8E4
:10E22000181049420844401E00B2019025984089C8
:10E2300003460390249ADDE90101FDF77BFD049874
:10E240000090BDF86A00BDF8181049420844401E0D
:10E2500000B20290BDF86800BDF81A1049420144AE
:10E260000598081A00B2019025984089034603904A
:10E27000249ADDE9010100E001E0FDF75BFD1E9855
:10E2800000F00200E8B31E9800F00800C8B304983C
:10E290000090BDF86200BDF8181049420844401EC5
:10E2A00000B20290BDF86000BDF81A100144059854
:10E2B000084400B201902598408903460390249AAF
:10E2C000DDE90101FDF736FD04980090BDF862001C
:10E2D000BDF81A10494201440598081A00B202908C
:10E2E000BDF86000BDF818100844401C00B2019051
:10E2F0002598408903460390249ADDE90101FDF742
:10E3000019FD0598401C00B20590079905988842B0
:10E31000FFF6E0AEBDF91800BDF91A10401A00284A
:10E3200005DDBDF91800BDF91A10401A04E0BDF969
:10E330001A00BDF91810401A079988427ED10B982F
:10E34000ADF818000B98ADF81A001D984010049015
:10E350001E9800F00100E0B11E9800F00800C0B166
:10E3600004980090BDF85E00BDF81810084400B293
:10E370000290BDF85C00BDF81A10084400B201908C
:10E380002598408903460390249ADDE90101FDF7B1
:10E39000D1FC1E9800F00100E8B11E9800F00400C6
:10E3A000C8B104980090BDF86600BDF81A10084482
:10E3B00000B20290BDF86400BDF81810494208444C
:10E3C00000B201902598408903460390249ADDE924
:10E3D0000101FDF7AFFC1E9800F00200F0B11E989D
:10E3E00000F00400D0B104980090BDF86A00BDF8B8
:10E3F00018104942084400B20290BDF86800BDF808
:10E400001A104942084400B20190259840890346F9
:10E410000390249ADDE90101FDF78CFC1E9800F0C1
:10E420000200F8B11E9800F00800D8B104980090DE
:10E43000BDF86200BDF81A10494200E013E008443C
:10E4400000B20290BDF86000BDF81810084400B298
:10E4500001902598408903460390249ADDE9010143
:10E46000FDF768FC00BFBDF9520009900898ADF8AF
:10E4700018000A98ADF81A00DDE90901401A00B247
:10E480000790002005903CE11D9A05990798FDF73B
:10E4900099FB04901E9800F00100F8B11E9800F05E
:10E4A0000800D8B104980090BDF85E00BDF81A10BD
:10E4B00001440598084400B20290BDF85C00BDF824
:10E4C00018100844401E00B2019025984089034668
:10E4D0000390249ADDE90101FDF72CFC1E9800F061
:10E4E000010000B31E9800F00400E0B10498009011
:10E4F000BDF86600BDF818100844401E00B2029036
:10E50000BDF86400BDF81A10494201440598081A84
:10E5100000B201902598408903460390249ADDE9D2
:10E520000101FDF707FC1E9800F0020008B31E98D9
:10E5300000F00400E8B104980090BDF86A00BDF84E
:10E540001A10494201440598081A00B20290BDF819
:10E550006800BDF8181049420844401C00B2019000
:10E560002598408903460390249ADDE90101FDF7CF
:10E57000E1FB1E9800F0020000B31E9800F00800B6
:10E58000E0B104980090BDF86200BDF8181049424F
:10E590000844401C00B20290BDF86000BDF81A109B
:10E5A00001440598084400B201902598408903462B
:10E5B0000390249ADDE90101FDF7BCFBBDF91800C9
:10E5C000401EBDF91A200599114488427ED01E983C
:10E5D00000F00100F8B11E9800F00800D8B10498CE
:10E5E0000090BDF85E00BDF818100844401E00B24F
:10E5F0000290BDF85C00BDF81A100144059808446B
:10E6000000B201902598408903460390249ADDE9E1
:10E610000101FDF78FFB1E9800F0010000B31E986A
:10E6200000F00400E0B104980090BDF86600BDF869
:10E630001A1001440598084400B20290BDF8640025
:10E64000BDF8181049420844401C00B201902598BA
:10E65000408903460390249ADDE90101FDF76AFB36
:10E660001E9800F0020008B31E9800F00400E8B104
:10E6700004980090BDF86A00BDF81810494208449B
:10E68000401C00B20290BDF86800BDF81A10494263
:10E6900001440598081A00B2019025984089034664
:10E6A0000390249ADDE90101FDF744FB1E9800F078
:10E6B000020058B11E9800F0080038B1049800908C
:10E6C000BDF86200BDF81A10494200E015E00144AF
:10E6D0000598081A00B20290BDF86000BDF8181045
:10E6E0000844401E00B201902598408903460390DB
:10E6F000249ADDE90101FDF71DFB0598401C00B2DD
:10E700000590079905988842FFF6BEAE00BF27B076
:10E7100000BD2DE9FF4F87B004469146B9F80600C9
:10E720001FFA80F8FCF7D9F8009002F021FD0746A7
:10E73000204601F096FD0690204601F099FD0590D7
:10E74000B9F90C600A98FF2802D199F80F0004E08B
:10E7500099F80F000A9948430012049099F80E5056
:10E76000B9F80A0003904FF0000BDA46701E06B2AB
:10E770004046DDE90521FEF74DFF8046B04506DA4B
:10E78000A6EB0800C01B0FFA80FBB24603E008EBC3
:10E7900007000FFA80FAB9F8060000287ED105F0CC
:10E7A000020098B12088ADF80400A088ADF80800F8
:10E7B0006088ADF806006088304400B2ADF80A0009
:10E7C00001A8DDE903230899FDF7C3FB05F0080064
:10E7D00028B3A088801B00B2ADF80400A088ADF873
:10E7E0000800B4F9021005F0020008B1701C00E046
:10E7F0000020084400B2ADF80600B4F9061005F098
:10E80000010008B1701C00E00020081A00B2ADF849
:10E810000A0001A8DDE903230899FDF79AFB05F03A
:10E82000040028B32088ADF804002088304400B2EA
:10E83000ADF80800B4F9021005F0020008B1701C30
:10E8400000E00020084400B2ADF80600B4F906105C
:10E8500005F0010008B1701C00E00020081A00B2A9
:10E86000ADF80A0001A8DDE903230899FDF771FB63
:10E8700005F00100A8B12088ADF80400A088ADF82B
:10E880000800E088801B00B2ADF80600E088ADF813
:10E890000A0001A8DDE90323089900E004E0FDF780
:10E8A00058FB0BB0BDE8F08F0AF101000FFA80FAB7
:10E8B00005F0020028B16088504400B2ADF80600AF
:10E8C00004E06088404400B2ADF8060005F00100A5
:10E8D00030B1E088A0EB0A0000B2ADF80A0005E014
:10E8E000E088A0EB080000B2ADF80A0005F00400D3
:10E8F00070B12088ADF80400BDF80400304400B2C7
:10E90000ADF8080001A8DDE903230899FDF721FB14
:10E9100005F0080070B1A088ADF80800BDF8080047
:10E92000801B00B2ADF8040001A8DDE903230899BB
:10E93000FDF70FFB20885044A0EB0B0000B2ADF8B0
:10E940000400A088A0EB0A00584400B2ADF808000B
:10E9500005F0020068B16088ADF8060060883044B8
:10E9600000B2ADF80A0001A8DDE903230899FDF71C
:10E97000F0FA05F0010070B1E088ADF80A00BDF8CA
:10E980000A00801B00B2ADF8060001A8DDE90323F0
:10E990000899FDF7DEFABBF1000F7DD005F002000B
:10E9A000E8B105F00400D0B12088ADF8040020885B
:10E9B0004044384400B2ADF8080060884044401C30
:10E9C000384400B2ADF806006088304400B2ADF8BB
:10E9D0000A0001A8DDE903230899FDF7BAFA05F05A
:10E9E0000200F0B105F00800D8B1A088A0EB080043
:10E9F000C01B00B2ADF80400A088ADF80800608824
:10EA00004044401C384400B2ADF8060060883044F1
:10EA100000B2ADF80A0001A8DDE903230899FDF76B
:10EA200098FA05F00100F0B105F00400D8B1208893
:10EA3000ADF8040020884044384400B2ADF8080026
:10EA4000E088801B00B2ADF80600E088A0EB08006B
:10EA5000401EC01B00B2ADF80A0001A8DDE9032387
:10EA60000899FDF776FA05F00100A8B105F0080055
:10EA700090B1A088A0EB0800C01B00B2ADF8040064
:10EA8000A088ADF80800E088801B00B2ADF8060051
:10EA9000E088A0EB080000E00AE0401EC01B00B2C6
:10EAA000ADF80A0001A8DDE903230899FDF751FA42
:10EAB000B9F80600002863D105F00600A8B1208847
:10EAC000ADF804002088384400B2ADF80800608832
:10EAD000ADF806006088384400B2ADF80A0001A81D
:10EAE000DDE903230899FDF734FA05F00A00A8B11F
:10EAF000A088C01B00B2ADF80400A088ADF80800E3
:10EB00006088ADF806006088384400B2ADF80A00AD
:10EB100001A8DDE903230899FDF71BFA05F00500BC
:10EB2000A8B12088ADF804002088384400B2ADF8C0
:10EB30000800E088C01B00B2ADF80600E088ADF820
:10EB40000A0001A8DDE903230899FDF702FA05F0A0
:10EB50000900A8B1A088C01B00B2ADF80400A088CD
:10EB6000ADF80800E088C01B00B2ADF80600E088F0
:10EB7000ADF80A0001A8DDE903230899FDF7E9F9DA
:10EB800000BF8EE60FB5A9B02B98C08880B2289040
:10EB9000FBF7A3FE0B9002F0EBFA27902B9840882E
:10EBA00026902B98808825902C98FF2802D12B98AE
:10EBB000007A04E02B98007A2C99484300122390A5
:10EBC000299801F055FB2190299801F04AFB2090EB
:10EBD000DDE920122898FEF71DFD2890299801886C
:10EBE000289801442798084400B2ADF87C00299881
:10EBF0004188289801442798084400B2ADF87E0067
:10EC000029980188289801442798084400B2ADF853
:10EC100078002998C1882898091A2798081A00B2FC
:10EC2000ADF87A00299881882898091A2798081A37
:10EC300000B2ADF8740029984188289801442798BB
:10EC4000084400B2ADF87600299881882898091AFE
:10EC50002798081A00B2ADF870002998C188289842
:10EC6000091A2798081A00B2ADF87200289802B263
:10EC700012A913A802F046FFBDF87200BDF84E10AD
:10EC8000084400B20090BDF87000BDF84C10084474
:10EC900000B20B90BDF87A00BDF84E10084400B2E7
:10ECA0000A90BDF87800BDF84C104942084400B203
:10ECB0000990014616A8DDE90A2302F0EAFDBDF835
:10ECC0007200BDF84C10084400B20090BDF870000E
:10ECD000BDF84E10084400B20B90BDF87A10BDF894
:10ECE0004C00084400B20A90BDF87800BDF84E1000
:10ECF0004942084400B20990014614A8DDE90A23FC
:10ED000002F0C7FDBDF87600BDF84E104942084438
:10ED100000B20090BDF87400BDF84C10084400B279
:10ED20000B90BDF87E00BDF84E104942084400B279
:10ED30000A90BDF87C00BDF84C104942084400B26E
:10ED40000990014618A8DDE90A2302F0A2FDBDF8EA
:10ED50007600BDF84C104942084400B20090BDF85E
:10ED60007400BDF84E10084400B20B90BDF87E0050
:10ED7000BDF84C104942084400B20A90BDF87C002E
:10ED8000BDF84E104942084400B2099001461AA845
:10ED9000DDE90A2302F07DFD0020119010902898F3
:10EDA00000B20F908AE2279800287DD0BDF94C1060
:10EDB0000F988142F9D0BDF94E001090DDE91001A5
:10EDC000401A00B207900F98ADF818001198ADF8EE
:10EDD0001A000F992898401AC0EB00212198B1FB26
:10EDE000F0F0C0B22290229ADDE92501FEF7B2FBD5
:10EDF0000E90229ADDE92510FEF7ACFB0D90002065
:10EE00000590F8E00798012806DD239A05990798F0
:10EE1000FEF7DEFB049008E0239A05990798FCF7BB
:10EE2000D1FE2399081AC0B2049004980090BDF84E
:10EE30007200BDF818100844401C00B20390BDF8E1
:10EE40007000BDF81A1001440598084400B2029001
:10EE50000D9B2A9A0399FCF76DFF04980090BDF86A
:10EE60007A00BDF818100844401C00B20390BDF8A9
:10EE70007800BDF81A10494201440598081A00B2FA
:10EE800002900D9B2A9A0399FCF754FF0498009076
:10EE9000BDF87E00BDF8181049420844401E00B27B
:10EEA0000390BDF87C0000E0B0E0BDF81A104942C4
:10EEB00001440598081A00B202900E9B2A9A039901
:10EEC000FCF738FF04980090BDF87600BDF81810E4
:10EED00049420844401E00B20390BDF87400BDF8DA
:10EEE0001A1001440598084400B202900E9B2A9A19
:10EEF0000399FCF71FFF11992898411A05980844B7
:10EF0000C0EB00212198B1FBF0F0C0B22290229A10
:10EF1000DDE92510FEF71EFB0C9004980090BDF86B
:10EF20007210BDF81A0001440598084400B203901D
:10EF3000BDF87000BDF818100844401C00B20290E3
:10EF40000C9B2A9A0399FCF7F5FE04980090BDF8F3
:10EF50007A00BDF81A1001440598084400B20390E5
:10EF6000BDF87810BDF8180040420844401E00B2B9
:10EF700002900C9B2A9A0399FCF7DCFE229ADDE9A9
:10EF80002501FEF7E7FA0C9004980090BDF87E008A
:10EF9000BDF81A10494201440598081A00B20390BE
:10EFA000BDF87C00BDF8181049420844401E00B26C
:10EFB00002900C9B2A9A0399FCF7BCFE04980090DF
:10EFC000BDF87610BDF81A00404201440598081AB1
:10EFD00000B20390BDF87410BDF818000844401C3E
:10EFE00000B202900C9B2A9A0399FCF7A3FE0598A5
:10EFF000401C00B20590079905988842FFF602AFC1
:10F00000BDF94C000F901098119000BF00200B909C
:10F010000A9009900890BDF94E10BDF97A00084495
:10F02000BDF95A10884201D001200990BDF94C1059
:10F03000BDF97A000844BDF95210884201D0012080
:10F040000890BDF94E004042BDF97E100844BDF95C
:10F050006210884201D001200A90BDF94C00404264
:10F06000BDF97E100844BDF96A10884201D0012024
:10F070000B900B9808B3BDF89800BDF89410884227
:10F0800002D12698249012E02998B0F90600BDF923
:10F090006A10401AC0EB00212198B1FBF0F0C0B219
:10F0A0002290229ADDE92510FEF754FA24901AA83E
:10F0B000DDE923322A99FCF74CFF0A9808B3BDF822
:10F0C0009800BDF89410884202D12698249012E04E
:10F0D0002998B0F90610BDF96200081AC0EB0021AA
:10F0E0002198B1FBF0F0C0B22290229ADDE9251000
:10F0F000FEF730FA249018A8DDE923322A99FCF7AC
:10F1000028FF099808B3BDF89800BDF8941088420C
:10F1100002D12698249012E02998B0F90610BDF982
:10F120005A00081AC0EB00212198B1FBF0F0C0B2E0
:10F130002290229ADDE92510FEF70CFA249016A8F9
:10F14000DDE923322A99FCF704FF089808B3BDF8DB
:10F150009800BDF89410884202D12698249012E0BD
:10F160002998B0F90600BDF95210401AC0EB0021F1
:10F170002198B1FBF0F0C0B22290229ADDE925106F
:10F18000FEF7E8F9249014A8DDE923322A99FCF768
:10F19000E0FEBDF87210BDF84E00084400B20090C9
:10F1A000BDF87000BDF84C10084400B20790BDF8DF
:10F1B0007A10BDF84E00084400B20690BDF87810F1
:10F1C000BDF84C004042084400B20590014616A824
:10F1D000DDE9062302F05DFBBDF87210BDF84C00BE
:10F1E000084400B20090BDF87000BDF84E1008440D
:10F1F00000B20790BDF87A10BDF84C00084400B288
:10F200000690BDF87810BDF84E004042084400B2A8
:10F210000590014614A8DDE9062302F03AFBBDF88B
:10F220007610BDF84E004042084400B20090BDF890
:10F230007400BDF84C10084400B20790BDF87E0081
:10F24000BDF84E104942084400B20690BDF87C005B
:10F25000BDF84C104942084400B20590014618A878
:10F26000DDE9062302F015FBBDF87600BDF84C1071
:10F270004942084400B20090BDF87400BDF84E1039
:10F28000084400B20790BDF87E00BDF84C1049421A
:10F29000084400B20690BDF87C00BDF84E1049420B
:10F2A000084400B2059001461AA8DDE9062302F0E1
:10F2B000F0FA12A913A802F038FC00BF13A802F05C
:10F2C00029FC00287FF46FADBDF89800BDF89410BC
:10F2D000884202D12698249012E02998B0F90600BD
:10F2E000BDF96A10401AC0EB00212198B1FBF0F083
:10F2F000C0B22290229ADDE92510FEF72BF9249066
:10F300001AA8DDE923322A99FCF723FEBDF96A0029
:10F31000BDF96210884221D0BDF89800BDF8941064
:10F32000884202D12698249012E02998B0F906006C
:10F33000BDF96210401AC0EB00212198B1FBF0F03A
:10F34000C0B22290229ADDE92510FEF703F924903D
:10F3500018A8DDE923322A99FCF7FBFDBDF89800D7
:10F36000BDF89410884202D12698249012E0299882
:10F37000B0F90600BDF95A10401AC0EB00212198DF
:10F38000B1FBF0F0C0B22290229ADDE92510FEF721
:10F39000E1F8249016A8DDE923322A99FCF7D9FD7B
:10F3A000BDF95200BDF95A10884221D0BDF898101D
:10F3B000BDF89400814202D12698249012E0299849
:10F3C000B0F90600BDF95210401AC0EB0021219897
:10F3D000B1FBF0F0C0B22290229ADDE92510FEF7D1
:10F3E000B9F8249014A8DDE923322A99FCF7B1FD7D
:10F3F000279800287ED02998018828980844801CE6
:10F4000000B2ADF86800299881882898081A801EF3
:10F4100000B2ADF86C0029984088ADF86A002998D0
:10F420004088ADF86E002B984088089002461AA8D4
:10F43000239B2A99FCF78DFD2998C088ADF86A00B6
:10F440002998C088ADF86E002B98808808900246F5
:10F450001AA8239B2A99FCF77CFDBDF94E00109059
:10F46000DDE91001401A00B20B900F98ADF82800AA
:10F470001198ADF82A000F992898401AC0EB002186
:10F480002198B1FBF0F0C0B22290229ADDE925016B
:10F49000FEF760F80D90229ADDE92510FEF75AF884
:10F4A0000E9000200990EEE0239A09990B98FCF742
:10F4B00089FB2399081AC0B2089008980090BDF8FB
:10F4C0007200BDF828100844401C00B20790BDF837
:10F4D0007000BDF82A1001440998084400B2069053
:10F4E0000E9B2A9A0799FCF725FC08980090BDF816
:10F4F0007A0000E058E1BDF828100844401C00B232
:10F500000790BDF87810BDF82A00404201440998E0
:10F51000081A00B206900E9B2A9A0799FCF70AFC7B
:10F5200008980090BDF87E00BDF8281049420844B4
:10F53000401E00B20790BDF87C10BDF82A00404282
:10F5400001440998081A00B206900D9B2A9A07995F
:10F55000FCF7F0FB08980090BDF87600BDF8281085
:10F5600049420844401E00B20790BDF87410BDF82F
:10F570002A0001440998084400B206900D9B2A9A7B
:10F580000799FCF7D7FB11992898411A0998084464
:10F59000C0EB00212198B1FBF0F0C0B22290229A7A
:10F5A000DDE92510FDF7D6FF0C9008980090BDF816
:10F5B0007200BDF82A1001440998084400B207906F
:10F5C000BDF87010BDF828000844401C00B2069039
:10F5D0000C9B2A9A0799FCF7ADFB08980090BDF8A0
:10F5E0007A00BDF82A1001440998084400B2079037
:10F5F000BDF87800BDF8281049420844401E00B20A
:10F6000006900C9B2A9A0799FCF794FB229ADDE955
:10F610002501FDF79FFF0C9008980090BDF87E1023
:10F62000BDF82A00404201440998081A00B2079028
:10F63000BDF87C00BDF8281049420844401E00B2C5
:10F6400006900C9B2A9A0799FCF774FB0898009087
:10F65000BDF87600BDF82A10494201440998081AFD
:10F6600000B20790BDF87400BDF828100844401C93
:10F6700000B206900C9B2A9A0799FCF75BFB09984D
:10F68000401C00B209900B9909988842FFF60CAF14
:10F69000BDF92800BDF92A10401A002805DDBDF982
:10F6A0002800BDF92A10401A04E0BDF92A00BDF96E
:10F6B0002810401A0B99884275D10F98ADF8280090
:10F6C0000F98ADF82A000F98C0EB00212198B1FBEC
:10F6D000F0F0C0B22290229ADDE92501FDF73AFF51
:10F6E0000E90229ADDE92510FDF734FF0D90239846
:10F6F0004010089008980090BDF87200BDF82810DE
:10F70000084400B20790BDF87010BDF82A00084404
:10F7100000B206900D9B2A9A0799FCF70BFB0898FC
:10F720000090BDF87A00BDF82A10084400B2079096
:10F73000BDF87800BDF828104942084400B2069090
:10F740000D9B2A9A0799FCF7F5FA08980090BDF8E6
:10F750007E00BDF828104942084400B20790BDF869
:10F760007C00BDF82A104942084400B206900E9B66
:10F770002A9A0799FCF7DEFA08980090BDF87600FF
:10F78000BDF82A104942084400B20790BDF8741031
:10F79000BDF82800084400B206900E9B2A9A0799EB
:10F7A000FCF7C8FA00BF00BF2DB000BD2DE9FF4F28
:10F7B00089B0044615469A46E88886B2FBF78DF86C
:10F7C000074601F0D5FC089068880790A888069045
:10F7D000204600F04DFD8046204600F042FD04909A
:10F7E000BAF1FF0F01D1287A03E0287A00FB0AF072
:10F7F00000120390424630460499FDF70BFF06467F
:10F8000008EBD871B6EB610F02DD0DB0BDE8F08FEB
:10F810002088ADF80400A088ADF80800BDF81C00F1
:10F82000BDF8181088422DD16088304400B2ADF880
:10F830000600E088801B00B2ADF80A00E888D0B16D
:10F84000089860B1BDF80600801C00B2ADF8060053
:10F85000BDF80A00801E00B2ADF80A000BE0BDF84A
:10F860000600401C00B2ADF80600BDF80A00401EBC
:10F8700000B2ADF80A0001A8039B079A0A99FCF7A9
:10F8800068FB43E0608830440FFA80F9E088801B11
:10F890000FFA80FBE88890B1089840B109F10200A6
:10F8A0000FFA80F9ABF102000FFA80FB07E009F1D3
:10F8B00001000FFA80F9ABF101000FFA80FBB9F1FA
:10F8C000000F01DA4FF000094F461CE0ADF806705A
:10F8D000ADF80A70B4F90600BDF90610401AC0EB85
:10F8E0000020B0FBF8F0C0B20590DDE905210798D3
:10F8F000FDF730FE009001A8039B009A0A99FCF7DF
:10F9000028FB781C07B25F45E0DD00BF00BF7CE745
:10F910002DE9FF4F95B082461646FAF7DEFF814685
:10F9200001F026FC1490B6F90650B6F91270504654
:10F9300000F097FC1390504600F09AFC1290A8B289
:10F94000DDE91221FDF766FE05B2149800EB4000D8
:10F95000284405B21498384407B2281D20F003004B
:10F960001190119840001190F81C00F0FC001090CC
:10F9700010981090DDE910218818FCF7EBF80F9033
:10F98000DDF83C80DDF83C80119808EB000B2A463E
:10F990000DA90EA802F0B6F80FE0BDF83800BDF9C9
:10F9A0003A1028F81100BDF83A00BDF9381028F8CF
:10F9B00011000DA90EA802F0B8F80EA802F0AAF8DE
:10F9C0000028EAD11898FF2801D1307A03E0307A74
:10F9D0001899484300120C90002409E0381B0C9938
:10F9E00048434008B0FBF7F00BF80400601C04B279
:10F9F000BC42F3DBBAF80000284400B2ADF81C00AA
:10FA0000BAF80600401B401C1499401A00B2ADF829
:10FA10001E00BAF80400401B00B2ADF81800BAF896
:10FA20000600401B401C1499401A00B2ADF81A00A1
:10FA300000246BE0BDF81C00001B00B2ADF82C00E8
:10FA4000BDF81E0038F81410084400B2ADF82E00BE
:10FA5000BDF81800204400B2ADF82800BDF81A0027
:10FA600038F81410084400B2ADF82A000CB9002090
:10FA700005E0601E38F9100038F91410401A00B281
:10FA800003904FF000093DE0039818B91BF80900F6
:10FA9000049009E01BF809100398A9EB00001BF87B
:10FAA000000008444008049004980090328A0292B2
:10FAB000BDF92E10BDF92C001346169AFCF73AF941
:10FAC000BDF82E00401C00B2ADF82E00BDF9280094
:10FAD000BDF91C1088420BDD04980090328A029216
:10FAE000BDF92A10BDF928001346169AFCF722F931
:10FAF000BDF82A00401C00B2ADF82A0009F101004F
:10FB00001FFA80F9B945BFDB601C04B2AC4291DD3D
:10FB1000BDF81C00401C00B2ADF82000BDF81E006E
:10FB2000284400B2ADF82200BDF81800401E00B213
:10FB3000ADF82400BDF82200ADF8260000200590A5
:10FB400019E005981BF80030308A0246049008A896
:10FB50001699FCF7FEF9BDF82200401C00B2ADF882
:10FB60002200BDF82600401C00B2ADF82600059822
:10FB7000401C80B205900598B842E2DB19B0BDE8A0
:10FB8000F08F2DE9F04F8DB004468B46174699460D
:10FB9000FAF7A3FE019001F0EBFA0546B7F906600B
:10FBA000B7F912000C90204600F05BFB0B9020464A
:10FBB00000F05EFB0A90B0B2DDE90A21FDF72AFDF4
:10FBC00006B2701906B2A088401C401B00B2ADF806
:10FBD000200060883044284400B2ADF82200BDF80F
:10FBE0002000ADF82400E088801B401B00B2ADF877
:10FBF00026002088401E284400B2ADF81800608816
:10FC00003044284400B2ADF81A00BDF81800ADF831
:10FC10001C00E088801B401B00B2ADF81E0020884D
:10FC20003044284400B2ADF810006088401E2844DB
:10FC300000B2ADF81200A088801B401B00B2ADF8E6
:10FC40001400BDF81200ADF8160020883044284496
:10FC500000B2ADF80800E088401C401B00B2ADF8CF
:10FC60000A00A088801B401B00B2ADF80C00BDF854
:10FC70000A00ADF80E004FF0010855E019F808A091
:10FC8000388A534602465946019008A8FCF761F9A4
:10FC9000BDF82000401C00B2ADF82000BDF82400E3
:10FCA000401C00B2ADF82400388A5346024659463B
:10FCB000019006A8FCF74DF9BDF81800401E00B2EF
:10FCC000ADF81800BDF81C00401E00B2ADF81C00D5
:10FCD000388A534602465946019004A8FCF739F980
:10FCE000BDF81200401E00B2ADF81200BDF81600BB
:10FCF000401E00B2ADF81600388A534602465946F7
:10FD0000019002A8FCF725F9BDF80A00401C00B2DA
:10FD1000ADF80A00BDF80E00401C00B2ADF80E00B0
:10FD200008F101000FFA80F80C988045A6DD0DB0AF
:10FD3000BDE8F08F2DE9FF4F99B080469146FAF764
:10FD4000CCFD039001F014FA8246B9F90650B9F9D6
:10FD50001270404600F085FA1890404600F088FA8C
:10FD60001790A8B2DDE91721FDF754FC05B205EBA9
:10FD70000A0005B27800401C00B21690E819001D78
:10FD800020F0030015901598400015901698C01C9F
:10FD900020F003001490149880001490E819001DBE
:10FDA00020F00300139013981390DDE914210A4406
:10FDB00013995018FBF7CEFE1290129E129E1598C2
:10FDC00030441190DDE914100844129E3044109024
:10FDD000304615990DF09BFE2A460EA90FA801F09A
:10FDE00091FE0FE0BDF83C00BDF93E1026F8110071
:10FDF000BDF83E00BDF93C1026F811000EA90FA871
:10FE000001F093FE0FA801F085FE0028EAD11C98AE
:10FE1000FF2802D199F8080004E099F808001C991D
:10FE2000484300120D9000240EE01698001B0D9917
:10FE300049004843010216984043B1FBF0F1119884
:10FE400040F82410601C04B216988442EDDBB8F828
:10FE50000400401BA0EB0A0000B2ADF82000B8F887
:10FE60000600401BA0EB0A0000B2ADF82200B8F873
:10FE70000400401BA0EB0A0000B2ADF81C00B8F86B
:10FE800002002844504400B2ADF81E00B8F800004B
:10FE90002844504400B2ADF81800B8F80600401BE2
:10FEA000A0EB0A0000B2ADF81A00B8F80000284430
:10FEB000504400B2ADF81400B8F802002844504491
:10FEC00000B2ADF81600002420E100200490834623
:10FED00044E00022794208B22DE02318002B06DA14
:10FEE00036F81430EB1AA3EB0B0319B20DE023180C
:10FEF000AB4200DD21E0231836F8133036F814C089
:10FF0000A3EB0C03A3EB0B0319B27B42994204DA77
:10FF1000F84201D1012304930FE0B94203DD119BA4
:10FF20001B681A4405E0A7EB010C119B53F82C3019
:10FF30001A44411C08B2B842CFDD00BFC2F3072308
:10FF4000109901F80B30049921B10BF101011FFA4E
:10FF500081FB06E00BF101001FFA80FBE819584510
:10FF6000B7DA00BF36F81400BDF81C100844401C76
:10FF700000B2ADF83000BDF81E00001B00B2ADF8B5
:10FF8000320036F81400BDF820100844401C00B2BE
:10FF9000ADF82C00BDF82200204400B2ADF82E00D0
:10FFA000BDF8140036F81410401A401E00B2ADF827
:10FFB0002800BDF81600001B00B2ADF82A00BDF8FD
:10FFC000180036F81410401A401E00B2ADF8240094
:10FFD000BDF81A00204400B2ADF8260001200390BD
:10FFE00087E0BDF92800BDF91410884214DABDF984
:10FFF0002A00BDF9161088420EDA03991098405C69
:020000040801F1
:100000000090B9F810200292BDF92A10BDF928001D
:1000100013461A9AFBF78EFEBDF92400BDF918109D
:10002000884214DABDF92600BDF91A1088420EDDA7
:1000300003991098405C0090B9F810200292BDF925
:100040002610BDF9240013461A9AFBF773FEBDF97A
:100050003000BDF91C10884214DDBDF93200BDF935
:100060001E1088420EDA03991098405C0090B9F88F
:1000700010200292BDF93210BDF9300013461A9AD1
:10008000FBF758FEBDF92C00BDF92010884214DDA5
:10009000BDF92E00BDF9221088420EDD039910989B
:1000A000405C0090B9F810200292BDF92E10BDF905
:1000B0002C0013461A9AFBF73DFEBDF82C00401C9D
:1000C00000B2ADF82C00BDF82400401E00B2ADF81F
:1000D0002400BDF83000401C00B2ADF83000BDF87F
:1000E0002800401E00B2ADF828000398401C80B2E2
:1000F000039003985845FFF674AF2CB94A46404622
:10010000109B1A99FFF73DFD601C04B2E819A0424C
:10011000BFF6DBAE1DB0BDE8F08F2DE9FC4706460B
:100120000F4615469846B5F90640304600F099F856
:100130008146304600F09CF88246A0B252464946BD
:10014000FDF768FA04B23146684600F085F8BDF85C
:100150000000204400B2ADF80000BDF80400001B10
:1001600000B2ADF804006946384601F080FC08B1E1
:10017000BDE8FC873146684600F06EF8BDF8020025
:10018000204400B2ADF80200BDF80600001B00B22A
:10019000ADF806006946384601F069FC00B1E7E7B2
:1001A000287D012806D143462A4639463046FFF7C6
:1001B000C1FD07E0287D28B943462A463946304626
:1001C000FFF7A6FB00BFD3E72DE9F04105460E4639
:1001D00014461F46284600F04BF8012804DB284649
:1001E00000F03FF8012801DABDE8F081608A28B10B
:1001F0003B46224631462846FFF78FFF31462846C8
:1002000001F018FC00B9EFE7207A10280DDD3B461D
:10021000224631462846FFF7C9FAE08828B13B4616
:10022000224631462846FEF7ADFCA08990B1A07B5E
:1002300080B1E07B10280DDB3B4622463146284644
:10024000FEF767FAE08828B13B4622463146284649
:10025000FDF702FA00BFC7E70A6802604A68426019
:100260007047014688880A88801A401C00B270478F
:100270000146C8884A88801A401C00B270470000B6
:100280002DE9F047074689467C48008810B90020D0
:10029000BDE8F0877A480668002514E005EB850084
:1002A00006EBC000406A774988420ADD05EB85000D
:1002B00006EBC000406A401E05EB850106EBC1015C
:1002C0004862681C85B26D4800888542E6DB0024E0
:1002D000002518E005EB850006EBC0004068B84239
:1002E0000FD105EB850006EBC004616AA0690844E4
:1002F0006062606AB0F57A7F02DD4FF47A70606206
:1003000005E0681C85B25D4800888542E2DB00BFDD
:10031000002C44D1344601250DE005EB850006EBA9
:10032000C000406A616A884203DA05EB850006EB8B
:10033000C004681C85B2514800888542EDDB6068C6
:1003400010B1204600F038FC00F0F9FF8246002092
:10035000A0614A463946204600F0D4FB8046B8F1F9
:10036000000F0FD1204600F027FC242120460DF07D
:10037000F0FB282120460DF0ECFB4FF000406062BE
:10038000002085E700206062A06918B9504600F09F
:10039000E1FFA061A06908B90120A06100BF20466B
:1003A00076E770B5064636480568002423E004EB7E
:1003B000840005EBC0004068B04200D0CEB904EB29
:1003C000840005EBC000406828B104EB840105EB14
:1003D000C10000F0F1FB04EB840105EBC100242116
:1003E0000DF0B7FB04EB840105EBC10028210DF0F3
:1003F000B0FB601C84B2214800888442D7DB70BD0A
:1004000070B505461E48006830B10020FFF7C9FFEF
:100410001B48006801F055FF05EB8501C80001F09D
:1004200020FF174908600846006808B900BFFEE7CA
:100430001348006818B900201049088070BD0F48A3
:100440000580002413E004EB84010D4A126802EBDE
:10045000C10024210DF07DFB04EB8401084A1268E1
:1004600002EBC10028210DF074FB601C84B203482C
:1004700000888442E7DB00BFE0E70000280100209D
:10048000980100200100008070B506460D462C6AD8
:100490004CB1206810B1206801F013FF204601F034
:1004A00010FF0020286270BDC16070472DE9FF4F2A
:1004B00087B004460E469046217C01F01F00FCF7F1
:1004C00035FA8346012000FA0BF0401E80B20690F8
:1004D0000027B9460025207C00F01F00072806D021
:1004E000082819D009282DD00A284CD140E02069CD
:1004F000C0F38A20C710208AC0F3822008B1781C7C
:1005000007B207FB08F000EBE6000544083506F0EB
:100510000700C0F1070936E02069C0F38A20871080
:10052000208AC0F3812008B1781C07B207FB08F0CD
:1005300000EBA6000544103506F003000621A1EBF0
:10054000400920E02069C0F38A204710208AC0F3C8
:10055000802008B1781C07B207FB08F000EB6600AA
:100560000544403506F001000421A1EB80090AE0B2
:100570002069C0F38A2707FB0860054405F58065FC
:100580004FF0000900BF00BF206A059000200490D2
:10059000207B20B9606881682944049104E0002030
:1005A00004900BB0BDE8F08F0020039014980190E8
:1005B0004FF0000A25E0DDE90310415C069800FADF
:1005C00009F0084040FA09F0029005980168029885
:1005D00001EB4001019800EB4A0009880180A9EB7A
:1005E0000B004FFA80F9B9F1000F06DACBF10800E1
:1005F0004FFA80F90498401C04900AF101000FFAA8
:1006000080FA0A988245D6DB0120CAE72DE9FF4F20
:100610008DB004460D469146FAA000680C90FAA0F1
:1006200000680B90F9A30FCB07AE0FC6A068008E31
:100630000690002710E0BDF81800C1B207EB470292
:100640001A988154BDF81800020A07EB4700401CB5
:100650001A990A54781C07B210988742EBDB0020E5
:100660000590217C01F01F00FCF760F98246012112
:1006700001FA0AF0401E80B2049000264FF00008F4
:100680004FF0000B207C00F01F000B2806D00C2838
:100690001AD00D282FD00E284DD143E02069C0F389
:1006A0008A20C610208AC0F3822008B1701C06B2CE
:1006B00006FB09F000EBE500804405F00700C0F1FF
:1006C000070B0CA8059036E02069C0F38A2086103D
:1006D000208AC0F3812008B1701C06B206FB09F025
:1006E00000EBA500804405F003000621A1EB400BC0
:1006F0000BA805901FE02069C0F38A204610208ACD
:10070000C0F3802008B1701C06B206FB09F000EBB4
:100710006500804405F001000421A1EB800B07A8CF
:10072000059008E02069C0F38A2606FB0950804442
:100730004FF0000B00BF00BF00200390207B20B9CA
:10074000606881684144039104E00020039011B087
:10075000BDE8F08F00200290002728E0DDE90210BC
:10076000415C049800FA0BF0084040FA0BF001904D
:10077000207C00F01F000E2801D1019902E00199B0
:100780000598415C07EB4700801C1A9A1154ABEBAB
:100790000A004FFA80FBBBF1000F06DACAF108002D
:1007A0004FFA80FB0398401C0390781C07B2109806
:1007B0008742D3DB0120CAE730B50546039C002001
:1007C00030BD2DE9F84F82460C4616461F46DDE93E
:1007D0000A854FF00009207C00F01F00042809D092
:1007E000207C00F01F00052804D0207C00F01F00B2
:1007F00006280BD1207B012845D143463A46314695
:1008000020460095FFF7D8FF81463CE0207C00F0B1
:100810001F000B280ED0207C00F01F000C2809D0F0
:10082000207C00F01F000D2804D0207C00F01F0069
:100830000E2808D143463A46314620460095FFF738
:10084000E5FE81461FE0207C00F01F0007280ED047
:10085000207C00F01F00082809D0207C00F01F0039
:10086000092804D0207C00F01F000A2808D1434644
:100870003A46314620460095FFF718FE814602E0D1
:100880000020BDE8F88F4846FBE7816070472DE9FE
:10089000FC5F80460C46207B012802D10020BDE889
:1008A000FC9F207C00F01F05042D03D0052D01D0F6
:1008B000062D0AD1207B20B9606880686061012024
:1008C000EDE7002060610120E9E7072D05D0082D44
:1008D00003D0092D01D00A2D5AD12846FCF726F85D
:1008E0008146012000FA09F7206A60B9042001F06E
:1008F000B8FC2062206A18B9206A08B900BFFEE778
:100900000021206A0160266A780001F0AAFC3060AC
:10091000207B012801D10020C1E762689168002294
:1009200010462EE001EB800A9AF8022001EB800AC3
:100930009AF8013011F820C04FEADC0BBDF800A096
:100940006BF3040ACDF800A04FEA930BBDF800A0AA
:100950006BF34A1ACDF800A04FEAD20BBDF800A005
:100960006BF3CF2ACDF800A0BDF800B0DA46CDF881
:1009700004A0326802EB4002BDF804301380421C30
:100980001046B842CED300BF00206061012086E748
:100990000B2D05D00C2D03D00D2D01D00E2D03D124
:1009A0000020606101207AE721464046FFF76CFD98
:1009B000002074E7416070472DE9F04107460D467D
:1009C00014462846FCF708FB06463EBB287800F094
:1009D0001F01042901DB0E2902DD0020BDE8F081A2
:1009E0002868820A206862F3942020602868420DFB
:1009F000206862F35F5020602878226860F3040268
:100A0000226021E000FF00000055AAFF0011223300
:100A1000445566778899AABBCCDDEEFFFFE7022E2E
:100A200010D10121206861F3942020602068C0F378
:100A3000140000F500102060206820F01F000B302B
:100A4000206001E00020C9E70120C7E7016070478E
:100A500010B5644801F0B8F904460CB900BFFEE7D0
:100A60000CB9002010BD002020606060A060E06034
:100A70002046F7E710B510215A4801F06CF9FFF74E
:100A8000E7FF04461CB90CB900BFFEE710BDAFF28A
:100A9000D7012046FFF7DAFFAFF20D212046FFF71E
:100AA00089FFAFF2E1212046FFF7EFFEAFF22761A9
:100AB0002046FFF7F9FC00BFE8E72DE9F0410646C4
:100AC0000D46286820F0E00028600027454801F026
:100AD000A5F9044610E00027206840B12A463146B7
:100AE0002046236898470746012F00D106E021469B
:100AF0003C4801F0F4F90446002CECD100BF384624
:100B0000BDE8F0812DE9F04104460F469046C4F857
:100B1000088067603846FCF75FFA20730020206287
:100B20000026304801F07AF9054620E0286808B12F
:100B3000686800B916E004F11002394628462B68AF
:100B400098470646012E00D00CE00020E06160616D
:100B50002560214628466A6890470646012E00D146
:100B600007E000BF29461F4801F0B9F90546002DEE
:100B7000DCD100BF1EB9242120460CF0EAFF30462C
:100B8000BDE8F0812DE9FC4704460D4616461F4698
:100B9000DDF828804FF000092068806848B1CDE971
:100BA0000078206833462A462146D0F808C0E0473E
:100BB00081464846BDE8FC8710B50446206830B140
:100BC0002068C06818B120682146C268904710BDEF
:100BD00010B504462146034801F091F9204601F082
:100BE00070FB10BDCC2E0020024610880B88C01A66
:100BF00070472DE9FC4780460E4616B90020BDE837
:100C0000FC87D8F80C406069B04201D1A069F6E7D2
:100C10000025AEE005EB8501A06850F82100301AF0
:100C2000019005EB8501A06800EB810080880199A7
:100C3000884200D29BE0002705EB8501A06800EB0D
:100C40008100807C00F0030040B905EB8501A068BD
:100C500000EB8100C0880199471884E005EB85010D
:100C6000A06800EB8100807C00F0030001280FD118
:100C700005EB8502A16801EB8201C86805EB8502DE
:100C8000A16801EB8201C988019A825C8F186AE031
:100C900005EB8501A06800EB8100807C00F003007B
:100CA000022827D1AA48009005EB8503A06800EB35
:100CB0008300028A05EB8503A06800EB8300022312
:100CC000816801A802F01EF98146B9F1000F10D029
:100CD00005EB8502A16801EB82018968A9EB01009F
:100CE000400805EB8502A16801EB8201C9880F1855
:100CF00000BF38E005EB8501A06800EB8100807C37
:100D000000F0030003282ED19148009005EB8503E5
:100D1000A06800EB8300028A05EB8503A06800EB66
:100D200083000223816801A802F0ECF88146B9F142
:100D3000000F17D005EB8503A26802EB83029268CF
:100D4000A9EB0200400805EB8503A26802EB8302D1
:100D5000D16805EB8503A26802EB8302D2880B5CA5
:100D6000D71800BF00BF6661A761384647E7681C17
:100D700085B2608AC0F30900A8423FF74BAF6661B5
:100D80000020A06100BF3AE72DE9F0410546884602
:100D9000EE6841462846FFF72CFF074617B90020AA
:100DA000BDE8F081706800EBC7042CB130682168A1
:100DB000C1F313010844F3E70020F1E730B5024620
:100DC00014460B4620881D88A84203D020881D8821
:100DD000401B30BD60885D88401BFAE730B5024695
:100DE00014460B4620781D78A84203D020781D7841
:100DF000401B30BD60785D78401BFAE72DE9FC5F51
:100E000080460D461646D8F80C704FF0000A788AD6
:100E1000C0F34030002841D1FC68A068C0F30160F5
:100E2000D8B9D4F8009005EB062080B2019049486B
:100E30000090A06820F07F420223494601A802F0FA
:100E400061F88346BBF1000F06D0ABEB0900400808
:100E5000616811F900A000BF1FE0A068C0F3016045
:100E600001281AD1D4F8009005EB062001903A48E9
:100E70000090A06820F07F420423494601A802F0B8
:100E800041F88346BBF1000F06D0ABEB0900000927
:100E9000616811F900A000BF00BF13E0F868436863
:100EA000595D43689A5D00290BDD002A09DD531E58
:100EB0004C1E90F80DC004FB0C330468E35C4FFA41
:100EC00083FA00BF5046BDE8FC9F2DE9FF5F8046D6
:100ED0000C46D8F80C6040460299FFF78AFE074698
:100EE0001FB9002004B0BDE8F09F4FF00009F06882
:100EF00070B140460399FFF77CFE8346BBF1000FBB
:100F000005D05A4639464046FFF778FF814600BF74
:100F1000706800EBC7052868010D308A00FB09F0F6
:100F200001EB201A0AF108004FEA101AA4F800A0F9
:100F30006879E0702879A070A8792071E87940B2CA
:100F40006071708AC0F38220A0710120CAE700009E
:100F5000E90B0108DD0D0108BD0D010838B5044697
:100F6000202120460CF0F5FD0020E060F0202080DC
:100F70004FF4A070608000206060A06820F0020044
:100F8000A060A74800680090BDF80000A083A0689A
:100F900020F00100401CA0600020606138BD2DE9F8
:100FA000F04104460F4615461E461C2120460CF013
:100FB000D0FD276065602068A060E660BDE8F08134
:100FC00070B50546974800F0FFFE044624B90CB9F9
:100FD00000BFFEE7002070BD2022294620460CF00D
:100FE0001FFD202104F59E700CF0B3FD4FF48071BD
:100FF00004F13C000CF08BFD442104F1240000F0CE
:10100000AAFE8948006808B98748046086480668CF
:1010100004600020C4F85C0100210846F8F796FA45
:10102000206300210846F8F791FA60630021084622
:10103000F8F78CFAA0637D49606BF9F734FA7B49C5
:10104000A06BF9F730FA206BF8F77CF87648066069
:10105000234603221E21764801F087FB2062206A86
:1010600008B900BFFEE7206A08B90020B3E7206A8C
:1010700001F09AFB2046AEE76B480068704700B568
:10108000014611B9FFF7F8FF014611B94FF4A070FE
:1010900000BD087AC0F3400010B9B1F90200F7E7CB
:1010A000B1F90000F4E700B5014611B9FFF7E4FF1C
:1010B000014609B9F02000BD087AC0F3400010B91C
:1010C000B1F90000F7E7B1F90200F4E72DE9F041CA
:1010D00004460E462022314620460CF0A1FC04F1C5
:1010E000240000F09BFE054612E02046FFF7C7FFF4
:1010F00007462046FFF7D7FF80463A464146284636
:10110000F9F72FF9294604F1240000F0E8FE05461E
:10111000002DEAD1BDE8F0814349086070472DE910
:10112000F04105460026FFF7A7FFA84200D101269F
:10113000002000F0CCF8044608E0E068A84201D1A5
:101140000020E060204600F0C2F80446002CF4D1F4
:101150002946344800F0D3FE284601F0B2F82EB1FB
:10116000304800F05BFE0746FFF7D6FFBDE8F08190
:1011700000B5014611B9FFF77FFF014609B900200C
:1011800000BD087A00F00100FAE74168896921F0A2
:10119000010142689161704710B504461CB92148AD
:1011A00000F03CFE10BD21461E4800F098FEF9E715
:1011B0000146486870470146B1F85C01C0F3090078
:1011C0007047B0F85C21C2F309028A4203DA0022B8
:1011D000C0F85C2106E0B0F85C21C2F30902521AA3
:1011E000C0F85C21704701464868006820B1486833
:1011F000406808B1012070470020FCE700B50246B6
:101200001088518810FB01F31046FFF7ECFF28B15E
:101210005068C068984201D1012000BD0020FCE761
:101220007C610008842E002084010020A82B00206F
:1012300031AE000810B504461C2120460CF089FC94
:10124000002020700A202075142060754FF4C870AB
:10125000E0826420208310BD70B50546E86810B9AF
:10126000FFF70AFFE860E86808B9002070BD2D4864
:1012700000F0AAFD044624B90CB900BFFEE7002027
:10128000F4E75C2120460CF064FC1C222946204631
:101290000CF0C6FB94F84C0020F00200801C84F88F
:1012A0004C00002020656065A065234603221E21B6
:1012B0001D4801F05AFA20612046D7E770B5044670
:1012C0000D461C22294620460CF0AAFB70BD10B525
:1012D00004461CB9134800F0A1FD10BD2146114879
:1012E00000F0FDFDF9E770B504460D46002600202C
:1012F00028606860A860E8602078012804D1208C0C
:101300002880608C688004E02078022801D1606A1F
:101310006860606820B129462046626890470646AA
:10132000304670BD902E0020438E00080021104AE8
:1013300011701049096801440E4A1160704700BFDE
:1013400001210B4A11700B490868114609780029E0
:10135000F6D0704710B50346FFF7F1FF04469C42F4
:1013600001D3E31A01E05B422344184610BD00009C
:101370008C0100208801002010B58AB0044694F842
:101380002000C0F3400020B994F8200000F00100D4
:1013900070B194F82000C0F34000F0B994F8200038
:1013A00000F00100C8B194F82000C0F38000A0B1A3
:1013B0002422214601A80CF033FB2146FD4800F011
:1013C0009EFD204600F07DFF0120FB490870049837
:1013D00010B101A8049988471FE0E08B404200B299
:1013E000608394F8200000F00100B0B194F8201060
:1013F000C1F3800119B9A18B494209B2618310344C
:10140000217C8908C943227C61F38202227420680E
:10141000616821606060103C00BFE74800780AB056
:1014200010BD2DE9F0410746E24800F0F7FC044604
:1014300008E0206A20F0080020622146DD4800F024
:101440004EFD0446002CF4D1DC480068FFF782FF13
:101450000646D84800F0E2FC04463CE00020D649AD
:10146000087094F82000C0F3C00038BB206A20F058
:10147000080008302062608B304400B26083B4F909
:101480001A0000281ADBB4F91A00218B884202DD09
:10149000208B00B260832046A168884705466068BB
:1014A00018B129B2D4E900029047B4F91A00218B8F
:1014B000884202DB2046FFF75FFF00BFBE4800788E
:1014C00020B1BC4800F0AAFC044604E02146B9481B
:1014D00000F005FD0446002CC0D1FFF730FFB749EE
:1014E0000860BDE8F08110B52421B24800F033FC5B
:1014F000FFF725FFB1490860002303221E21B048F1
:1015000001F033F910BD10B50146088BB1F91A404E
:10151000A04202D14FF4806205E0B1F91A008002C6
:101520000C8B90FBF4F2D1E90440001B00FB02F3AA
:101530009B120869034418B210BD10B5044624215B
:1015400020460CF006FB4FF4FA7020830020206147
:1015500064206061AFF25100A06010BD2DE9F04140
:1015600007460D464FF00008924800F057FC04462D
:1015700017E021468F4800F0B2FC06462068B842CA
:101580000ED16068A84200D055B92146894800F0C4
:10159000B6FC204600F095FE012087490870804681
:1015A0003446002CE5D14046BDE8F08170B50546D3
:1015B000686818B1D5E90001FFF7D0FF7D4800F059
:1015C00003FC04460CB900BFFEE704B970BD95F8F2
:1015D000200020F0040085F820002422294620461F
:1015E0000CF01EFA606820B1238A19B2D4E9000217
:1015F000904701207049087000BFE7E770B50025EB
:101600006C4800F00BFC044606E0681C85B22146DD
:10161000684800F064FC0446002CF6D12846691C9A
:101620008DB270BD30B504460B46981A002801DD16
:10163000981A00E0D01A05464FF47A70684390FB80
:10164000F4F1B1F5803F01D34FF6FF7101B9491CA8
:1016500088B230BDF8B50446208BB4F91A10884220
:1016600002D14FF4806505E0B4F91A008002218BA5
:10167000B0FBF1F54FF4806001231A460021009081
:10168000284600F05AFD0746D4E90410401A00FB32
:1016900007F6B6122069064430B2F8BDF8B5044624
:1016A000208BB4F91A10884202D14FF4806505E00E
:1016B000B4F91A008002218BB0FBF1F54FF4806081
:1016C000431E1A4600210090284600F036FD0746CA
:1016D000D4E90410401A00FB07F6B612206906444C
:1016E00030B2F8BDF8B50446208BB4F91A10884220
:1016F00002D14FF4806505E0B4F91A008002218B15
:10170000B0FBF1F54FF480604FF467736422002161
:101710000090284600F011FD0746D4E90410401A55
:1017200000FB07F6B6122069064430B2F8BDF8B5E2
:101730000446208BB4F91A10884202D14FF4806518
:1017400005E0B4F91A008002218BB0FBF1F54FF4EB
:10175000806040F214534FF4167200210090284626
:1017600000F0EBFC0746D4E90410401A00FB07F632
:10177000B6122069064430B2F8BD2DE9F84305469B
:10178000288BB5F91A10884202D14FF4806405E025
:10179000B5F91A008002298BB0FBF1F4D5E90410E9
:1017A000461AB4F5CC7F0DD240F6C4106043840ACB
:1017B0004BE00000B42E0020940100209001002096
:1017C00023140108B4F5CC7F0DD340F26620844287
:1017D00009D2A4F5CC7404EB8404C4F5806406201B
:1017E00096FBF0F631E040F2662084420BD340F2E3
:1017F0003330844207D2A4F2662404EB840406202A
:1018000096FBF0F621E040F2333084420ED3B4F57B
:10181000667F0BD8A4F2333404EB84004400C4F593
:101820008064F11706EB11710E110EE0B4F5667FBE
:101830000BD9B4F5806F08D8A4F2993404EB840076
:101840004400F11706EB11710E11B4F5806F01D948
:101850004FF4806400204FF448734FF480621146C7
:101860000090204600F069FC804608FB06F7BF1296
:101870006869C71B38B2BDE8F8830146B1F91A00A0
:101880000A8B904202DB888A00B27047088A00B255
:10189000FBE710B5029C018042808380C48010BDAC
:1018A00002880A44521E12B28280704742880A445B
:1018B000521E12B2C2807047F0B503460C46154660
:1018C00000BF98881988401A401C00B2064600BF25
:1018D000D8885988401A401C00B207461C805D8099
:1018E00031461846FFF7DCFF39461846FFF7DEFFA2
:1018F000F0BD10B50146B1F90420B1F90030D21A9B
:10190000521CB1F90630B1F902401B1B5B1C02FBF3
:1019100003F010BD30B50346B1F90040B2F90050F4
:10192000AC4202DDB1F9004001E0B2F900401C8098
:10193000B1F90240B2F90250AC4202DDB1F9024005
:1019400001E0B2F902405C80B1F90440B2F9045000
:10195000AC4202DAB1F9044001E0B2F904409C80E3
:10196000B1F90640B2F90650AC4202DAB1F90640CC
:1019700001E0B2F90640DC800120B3F90040B3F980
:101980000450AC4205DCB3F90240B3F90650AC4256
:1019900000DD002030BD10B5B1F90030B2F90040D3
:1019A000A34202DAB1F9003001E0B2F9003003805D
:1019B000B1F90230B2F90240A34202DAB1F90230C1
:1019C00001E0B2F902304380B1F90430B2F90440C9
:1019D000A34202DDB1F9043001E0B2F904308380A2
:1019E000B1F90630B2F90640A34202DDB1F9063082
:1019F00001E0B2F90630C38010BD10B502460020E8
:101A0000B1F90030B2F90040A34212DBB1F9003065
:101A1000B2F90440A3420CDCB1F90230B2F9024041
:101A2000A34206DBB1F90230B2F90640A34200DC62
:101A3000012010BD0246B2F90000B1F9043098420D
:101A400013DCB2F90400B1F9003098420DDBB2F9B1
:101A50000200B1F90630984207DCB2F90600B1F98C
:101A60000230984201DB012070470020FCE710B5EE
:101A700002460020B2F90030B1F90040A34212DB67
:101A8000B2F90230B1F90240A3420CDBB2F90430E2
:101A9000B1F90440A34206DCB2F90630B1F90640C0
:101AA000A34200DC012010BD70B50546EC68D4E906
:101AB00000108847204600F004FC70BD2DE9F0417D
:101AC00006460F46082000F0CCFB044614B900205F
:101AD000BDE8F081234605220021094800F045FEBB
:101AE000054625B9204600F0ECFB0020F0E7266013
:101AF0006760EC60284600F060FE0120E8E7000027
:101B0000A91A0108028000234380C2F101031BB21D
:101B10000B8070470146B1F90200B1F900209042F4
:101B200001DC012070470020FCE74288521C12B201
:101B30004280B1F90020002A07DC0B88428852005D
:101B4000521C1A4412B20A800CE00288521E12B2D1
:101B5000028042880388D21A5200521C0B881A4411
:101B600012B20A80704718B50346D408BDF80000C9
:101B700064F3040000908C08BDF8000064F34A1080
:101B80000090DC08BDF8000064F3CF200090BDF8A1
:101B90000040204618BD2DE9F04F85B082468946A9
:101BA0001446CAEB0A204FF4B471B0FBF1F01FFAEF
:101BB00080FAC9EB0920642190FBF1F000F0FF09E5
:101BC000C4EB042090FBF1F0C4B2B9F1000F0ED1C8
:101BD000254626462746224621462046FFF7C3FFD4
:101BE0000090BDF80010084605B0BDE8F08F2B202E
:101BF0009AFBF0F0C0B204902B21049810FB01F086
